:020000040000FA
:1080000030590020D5800000F1800000CB5B0100DA
:108010000000000000000000000000000000000060
:10802000000000000000000000000000F5800000DB
:108030000000000000000000F7800000690202005C
:10804000FB800000FB800000E9CC0100F5CC0100C2
:108050003DC700007D080200E50E0200F10E02009F
:10806000E16E0100E96E010029E9010031E901003A
:108070003D5C0100455C0100650802006D080200DE
:1080800075080200B36D0100850802008D0802002A
:1080900095080200D9CC010023450200F9DC01005B
:1080A000898C0000E1CC0100553802005D380200E7
:1080B0000F700100AB6D010019D4000089BB0000F6
:1080C0000348854600F09CFD004800477B8C00007B
:1080D0003059002009480A4A002100A1814200D9F4
:1080E00002440848084A0260084880470848004798
:1080F000FEE7FEE7FEE7FEE7FEE7FEE70000002002
:108100000000000008ED00E0008000008D07020084
:10811000C180000030B50B4601460020202201241A
:1081200009E00D46D5409D4205D31D469540491BAB
:108130002546954040191546521E002DF1DC30BDF4
:1081400070B500242546002801DA012440420029A8
:1081500001DA01254942FFF7DDFFAC4200D0404281
:10816000002C00D0494270BDF0B51FB40646002077
:1081700082B005464024019100901BE001992246FF
:108180000F46304600F036FC049A059B801A994150
:1081900010D310461946224600F01CFC361A8F41B7
:1081A0000197224601200021009F00F013FC38189F
:1081B0004D4100902046641E0028DFDC019B0098A2
:1081C0002946324607B0F0BD38B50446C0681821CC
:1081D000401E4843A16840183C214843616840184C
:1081E0003C2148432168451860690C2148432169B6
:1081F00040186921C900401A3021FFF7A1FF114A38
:1082000050434219084600921A2902DB0E495118C0
:1082100000910C21FFF794FF0C4A5043009A8018FC
:1082200000900B4806E0491E425C074B5A43009BF6
:10823000D21800920029F6DC2146684600F006FCC0
:10824000009838BD801F8607805101008033E1010E
:1082500020CA020003460B439B0703D009E008C96C
:10826000121F08C0042AFAD203E00B780370401CE6
:10827000491C521EF9D27047D2B201E00270401C74
:10828000491EFBD270470022F6E710B513460A4696
:1082900004461946FFF7F0FF204610BD421E5378F2
:1082A000521C002BFBD10B781370491C521C002B65
:1082B000F9D17047421C0178401C0029FBD1801A7B
:1082C000704703460A780270401C491C002AF9D105
:1082D000184670470321001D401E037812021A43FE
:1082E000491EF9D510467047034610B508330722DA
:1082F000040E090221435B1E1C7800022043521E1B
:10830000F6D510BD034603220870000A491C521E10
:10831000FAD51846704770B504460D46072310700D
:108320000E06000A3043090A521C5B1EF7D5204690
:10833000294670BDF8B502464A40D40F42004B00B2
:1083400052085B089A4202D20246084611464A0089
:1083500023D0C30D4A00DDB2120EAD1A202D35DA3E
:1083600049020126490AF6058A19002C00D052421A
:1083700020214F1B1146B9402A411018C20D9A42C4
:1083800021D0002C17D0012D08DCDA05801AD20F7D
:108390008019D207DBB200F09BFBF8BDDA05801A2A
:1083A000012340001B06C01880185A428018CA0FCB
:1083B0001043490007E04908C2071143DA05801A53
:1083C00080194008801800F07BFBF8BD6100012295
:1083D000511A001BF7E70122D2075140AAE70122F8
:1083E000D2075040A6E7024670B54A40D30FDB07DC
:1083F00040002DD04A002AD0010E140E00021202B5
:108400000919400A520A8418E50104465443000A37
:10841000120A2E045043A4194219200CC543AA186D
:10842000120C0125AD03521C521912047F39240489
:1084300000D0521C104301D44000491EC2B20C06A9
:10844000C0092018401C4008802A02D003E0002008
:1084500070BD40084000002900DA0020184370BDBC
:1084600070B502464A40D50F40004A00ED0740086B
:108470005208002814D0002A12D0C40DD30D410296
:108480000120C0055202490A520AE41A09181218BA
:108490007D34914201D3641C00E04900002C01DAD4
:1084A000002070BD0023914201D3891A0343400884
:1084B00049000028F7D100290AD0914202D10121B8
:1084C000C90705E0914201D2012101E00121C94320
:1084D000E005C018401900F0F3FA70BDF0B507468A
:1084E0000846584087B0C00F049048000E46590017
:1084F00040084908BC1A884105D2384631461E4614
:1085000017460B4602465800400810434CD0300D29
:10851000039040055900400D490D0590401A029006
:10852000402872DA18030121000B09050843019065
:1085300004980092002805D00199524200208841F9
:1085400000920190029840210A1A0199009800F0C7
:1085500041FA05460C466B4607CB00F05CFAC019A1
:108560007141039A0E0D0023D71756401A467A40E0
:10857000164344D0049A002A2DD0029A012A039A65
:1085800015DC1205C01A914101263605001C714107
:10859000D20F059ED2070093019202962A462346E7
:1085A00000F0DCFA07B0F0BD38463146FAE71605B0
:1085B000224A0F46B218C01AB74101210905001C12
:1085C0004F4100187F41114618187941E20F1043BE
:1085D0006D19644113E0E2076D0815436408C20792
:1085E0001443039A01261205C01A91413605001C56
:1085F0007141CE07400830434908C01851412A460E
:10860000234600F09EFACDE7FFE7049801224000E0
:10861000C117121A00238B4104983146C417381A27
:10862000A141EEE730B40124E407634030BC55E7D4
:1086300030B40124E407614030BC4FE70000E0FFA4
:10864000F0B51FB488B00B990998002448400999E7
:10865000C00F490049080991C0070B9900904900D3
:1086600049080B9109990898A64608431CD00B9914
:108670000A98084318D0099801244000420D480088
:10868000410D099824050003000B204309900B9825
:108690000003000B20430B9050181C494018002287
:1086A00001901446104605E0002001460DB0F0BDD3
:1086B000032801DA034600E003239C46C11A0AAEF0
:1086C0000AE05F0008ADED5B4F00F75B7D430027DC
:1086D000AA187C41491C5B1E6145F2DD410004ABD8
:1086E0005A522104120C0A43240C401C0828DFDBD8
:1086F000019802900099704601910090059B049AA0
:108700000799069800F02AFAD0E700000DFCFFFF59
:10871000F0B50C465C4085B0E40FE40703944C00D0
:1087200000266408590094464908024602962243EE
:1087300021D062460A431ED06200570D4A000E0344
:108740002303550D012402462C492405781B1B0BDD
:10875000360B401823432643614600901C46501AAE
:10876000B44103D30098401C009002E09218009896
:108770005B41002803DA0020014605B0F0BD00206F
:10878000012109050746864611E064461D46141B73
:10879000B54106D36546521BB341744607430C43AB
:1087A000A646CD0740084908284392185B41054674
:1087B0000D43EAD11046184313D060461946504085
:1087C0007140084306D06046101AB34106D2012218
:1087D000002306E000220123DB0702E00122D2434E
:1087E0005310009874460105381C6141029C039D9A
:1087F0000019694100F0A5F9BFE70000FD03000082
:10880000C217C10F504010B54018CA079623002167
:1088100000F05EF910BD10B500229623114600F05D
:1088200057F910BD0EB5C217C10F5040CA07401806
:108830000021054B0293019200910A460B4600F07D
:108840008DF903B000BD0000330400000EB50549EA
:108850000291002100910A460B46019100F07EF939
:1088600003B000BD33040000410040020122400A71
:10887000D205090E80187F2901DA00207047962959
:1088800003DC9622511AC8407047963988407047D9
:1088900041000A0E40020121400AC90510B54018E6
:1088A0007F2A02DA0020014610BD0021962A03DC4F
:1088B00096239A1AD04010BD963A00F08BF810BD5E
:1088C0004A0009030123090B1B051943094B10B585
:1088D000520D9A4201DA002010BD064B34339A4201
:1088E00003DC9A1A00F086F810BD0349511888403D
:1088F00010BD0000FF030000CDFBFFFFC20FD20739
:10890000400040080BD0C10D0723DB01C91840020D
:108910000905400A1143C20840071143704700206F
:108920000146704710B5002904DB0124E4074042EA
:108930008C412146002B04DB1C460123DB075242FD
:10894000A3418B4200D1824210BD000010B5002926
:1089500004DB0124E40740428C412146002B04DB68
:108960001C460123DB075242A341994200D19042A9
:1089700010BD0000CB0FDB07490010B549080246C7
:108980000A4307D00A0D07240903E401090B121B4F
:10899000002A01DC002010BDC900440F0C43C100B7
:1089A000E018D205801800F08BF810BD0122D20724
:1089B000002800DB101A002900DB511A81427047A1
:1089C0000122D207002800DB101A002900DB511A0F
:1089D0008842704710B5202A04DB0146203A9140B6
:1089E000002010BD914020239C1A0346E340194308
:1089F000904010BD10B5202A04DB0846203AD04034
:108A0000002110BD0B46D340D0402024A21A914033
:108A10000843194610BD10B5202A06DBCB170846BF
:108A2000203A1041C1170B4306E00B461341D040DA
:108A30002024A21A91400843194610BD10B50249DE
:108A400000F004F810BD00000049002070B50C468D
:108A500000683C21FFF75EFB21603C21FFF75AFBD9
:108A600061601821FFF756FB0546A1600721001D34
:108A7000FFF750FBA1610F48A90008180E49FFF746
:108A800049FB0246443288086261E0613B2802D318
:108A9000910700D0401C0021084B0A462161995CD7
:108AA000814203D8401A521C2261F8E7401CE06062
:108AB000204670BD6C0B0000B50500002CCA0200FA
:108AC000002904DA401C490001D1400840007047E9
:108AD00070B40024050C05D11024000402D1002933
:108AE00021D01124050E01D100020834050F01D157
:108AF0000001241D850F01D18000A41C002801DB8A
:108B00004000641C002908D020252E1B0D46F5408E
:108B1000A14000D001212943084301061B1B000A84
:108B2000DB1D02D5002070BC7047DB0518188018CB
:108B30000029F8DA401C4900F5D170BC400840001B
:108B4000704710B5002B08DA0024401C61419218D0
:108B50005B411A4301D14008400010BDF0B51FB47D
:108B600082B005460C0003D008461CF071F802E004
:108B70001CF06EF820300246009021462846FFF790
:108B800029FF049B059A04460F46184311430843E6
:108B900014D0184610431BD0009840210A1A1846DA
:108BA0000599FFF727FF05460E46009A0599049898
:108BB000FFF710FF084305D0012004E020463946A6
:108BC00007B0F0BD0020C11705430E432C433743C7
:108BD00000990E986305401A7905E40A00220C43B7
:108BE000FD0A0A3002D500200146E9E70105101907
:108BF00069410C9C0D9D00196941FFF7A2FFDFE759
:108C0000064C0125064E05E0E36807CC2B430C3CDF
:108C100098471034B442F7D3FFF756FA38CC020025
:108C200058CC020070B58C180578401C6B075B0FA0
:108C300001D10378401C2A1106D10278401C03E0C0
:108C400006780E70401C491C5B1EF9D12B0705D419
:108C50000023521E0DD40B70491CFAE70378401C08
:108C6000CB1A921C03E01D780D70491C5B1C521E30
:108C7000F9D5A142D8D3002070BD10B517F086FDFC
:108C800021F01CFE002010BD10B5C046C046C046F5
:108C9000C04610BDF7B58AB00D460595059D28461E
:108CA000E917090F09180905090E0491002728E0A2
:108CB000002407E0380101190A98405C694608550C
:108CC000601CC4B2102CF5DB002605E00C98805D1A
:108CD00006A98855701CC6B2102EF7DB012206A922
:108CE00068461CF0E3F8002407E06846015D38019F
:108CF00002190A988154601CC4B2102CF5DB781C50
:108D0000C7B204988742D3DB0DB0F0BDFFB58DB07C
:108D100014460D98002802D0012854D154E025466D
:108D20002C462046E917090F09180911491C0905A5
:108D30000E0C301BC0B2089008980790E8B206905D
:108D400007E0069A0E99079888540698401CC0B20E
:108D500006900698B042F4DB002005902CE0002736
:108D600008E005980001C1190E98405C01A9C8559A
:108D7000781CC7B2102FF4DB002705E01098C05D07
:108D800009A9C855781CC7B2102FF7DB002209A922
:108D900001A81CF08BF8002708E001A8C15D059828
:108DA0000001C2190E988154781CC7B2102FF4DB51
:108DB0000598401CC0B20590F117090F89190A11D6
:108DC00005998A42CBDC53E025462C462046E9171C
:108DD000090F09180911491C09050E0C301BC0B2F6
:108DE000089008980790069507E0069A0E9907984C
:108DF00088540698401C80B206900698B042F4DB76
:108E0000002005902CE0002708E005980001C1191A
:108E10000E98405C01A9C855781CC7B2102FF4DB2E
:108E2000002705E01098C05D09A9C855781CC7B295
:108E3000102FF7DB002209A901A81CF037F8002742
:108E400008E001A8C15D05980001C2190E9881547F
:108E5000781CC7B2102FF4DB0598401CC0B20590F7
:108E6000F117090F89190A1105998A42CBDC00BF55
:108E700000BF11B0F0BD0000FEB51746002400256C
:108E8000002600200290019000BF27E0A0002549A5
:108E9000085800280DD0A00008584B21C90088426E
:108EA00007D2A0001F490958029808180290701CA8
:108EB000C6B2A0001C49085800280DD0A0000858D0
:108EC0004B21C900884207D2A000174909580198D0
:108ED00008180190681CC5B2601CC4B2BC42D5DB46
:108EE000002D08D029460198FFF714F90F4900908A
:108EF000FFF708FA03E00D490020FFF703FA002E00
:108F000009D031460298FFF705F90849091F00907A
:108F1000FFF7F8F904E00549091F0020FFF7F2F90F
:108F2000FEBD0000401A0020581A00207C1A0020C4
:108F300010B50446454800780A3803001BF09FFE30
:108F40000B070D17212B353F49535F697F002B2CF1
:108F500002D10B203D49087075E0432C03D10C2051
:108F60003A49087002E00A20384908706BE0452C45
:108F700003D10D203549087002E00A2033490870FA
:108F800061E0522C03D10E203049087002E00A2023
:108F90002E49087057E0452C03D10F202B4908704B
:108FA00002E00A20294908704DE0472C03D1102027
:108FB0002649087002E00A202449087043E03A2C50
:108FC00003D111202149087002E00A201F490870CE
:108FD00039E0202C03D112201C49087002E00A203D
:108FE0001A4908702FE0302C05DB332C03DC1320EA
:108FF0001649087002E00A201449087023E02C2C5E
:1090000003D114201149087002E00A200F490870AA
:1090100019E020463038C1B2012022F05DFB312C2E
:1090200001D0352C07D10320C04309490875002021
:109030000649087002E00A200449087003E00A208B
:109040000249087000BF00BF10BD00000C070020DF
:109050006334002010B50446384800780A3803000D
:109060001BF00DFE09060C16202A343E48526600FD
:109070002B2C02D10B20314908705DE0432C03D129
:109080000C202E49087002E00A202C49087053E099
:10909000472C03D10D202949087002E00A202749F6
:1090A000087049E0412C03D10E202449087002E0E9
:1090B0000A20224908703FE0542C03D10F201F4999
:1090C000087002E00A201D49087035E0542C03D1D5
:1090D00010201A49087002E00A20184908702BE095
:1090E0003A2C03D111201549087002E00A201349D7
:1090F000087021E0202C03D112201049087002E0F2
:109100000A200E49087017E020463038C1B202200C
:1091100022F0E2FA312C07D10320C0430849087538
:1091200000200649087002E00A200449087003E0A4
:109130000A200249087000BF00BF10BD0C070020C4
:10914000633400202B4909780A2902D00B2944D125
:1091500012E00021284A117030280CDB39280ADC83
:1091600011460A780978491C234B19702349885401
:109170000B21204A11703AE030280ADB392808DC3C
:109180001D490A780978491C1B4B19701B498854E2
:1091900022E04B280DD10021174A117000221749F7
:1091A000CA730A21134A11700321C943144A117565
:1091B00012E0114909780F2904DB0321C943104A41
:1091C000117503E00221C9430D4A117500220B49B4
:1091D000CA730A21074A117009E00A21054A117071
:1091E0000021054A1170C91E054A117500BF00BF54
:1091F000704700000C070020430700206C29002066
:109200006334002070B50446B24800780A38030081
:109210001BF035FD2C171D27313B455B6597A1AB36
:10922000B5BBC9E0F8FEEDECEBEAEAEAEAEAEAEA05
:10923000EAEAEAEAEAEAEAEAEAEAEAEAEA6F7983E1
:109240008DEA2B2C02D10B20A24908703FE14D2C56
:1092500003D10C209F49087002E00A209D49087044
:1092600035E1492C03D10D209A49087002E00A200B
:10927000984908702BE1502C03D10E2095490870B5
:1092800002E00A209349087021E14C2C03D10F2001
:109290009049087002E00A208E49087017E1572CA7
:1092A00006D100218C48817210208A4908700BE099
:1092B000452C06D1012188488172322085490870E9
:1092C00002E00A208349087001E1522C03D11120E9
:1092D0008049087002E00A207E490870F7E0492CB6
:1092E00003D112207B49087002E00A2079490870F6
:1092F000EDE0582C03D133207649087002E00A20B3
:1093000074490870E3E0452C03D13420714908709A
:1093100002E00A2071490870D9E0432C03D13520BE
:109320006C49087002E00A206A490870CFE0552CA9
:1093300003D112206749087002E00A2065490870CD
:10934000C5E0542C03D113206249087002E00A20C2
:1093500060490870BBE0452C03D114205D490870BA
:1093600002E00A205B490870B1E03A2C03D11520D5
:109370005849087002E00A2056490870A7E0302CCE
:1093800002D1162053490870A1E02C2C0AD11720D5
:10939000504908700020504988710A214E48001F2A
:1093A000FEF771FF93E02C2C10D0302C11DB392C00
:1093B0000FDC4948807909280BDA474881798079A0
:1093C000401C454A9071101F445402E01820414946
:1093D00008707CE02C2C14D13F48807A002809D1F9
:1093E00019203C4908700CE070E027E01CE015E013
:1093F0000EE007E03848807A012802D11A2035496A
:10940000087064E02C2C02D11A20324908705EE00A
:109410002C2C02D11B202F49087058E02C2C02D193
:109420001C202C49087052E02C2C06D11D20294903
:10943000087000212A488172C17248E02C2C3BD070
:109440000D2C39D02649C87A897A000208430121B7
:109450008902884228DA20480838FEF73BFF451C7D
:109460001D4908392846FEF74DFF302C01DB392C09
:1094700007DD412C01DB462C03DD612C25DB662C4E
:1094800023DC1748C17A807A09020143144AD07A52
:10949000927A00021043401C82B211488272120A72
:1094A000C2720C30445410E000210D488172C17228
:1094B0000A200849087008E0002007494872012086
:1094C0002039C8750A200349087000E000BF00BFBA
:1094D00070BD000051070020833400200C070020DD
:1094E000632E002000B52F4909780A390B001BF0C4
:1094F000C6FB08050B151F29333D47522B2802D107
:109500000B21284A11704AE0432803D10C21254A37
:10951000117002E00A21234A117040E0532803D160
:109520000D21204A117002E00A211E4A117036E016
:10953000432803D10E211B4A117002E00A21194A67
:1095400011702CE04F2803D10F21164A117002E050
:109550000A21144A117022E04E2803D11021114A29
:10956000117002E00A210F4A117018E0202803D17F
:1095700011210C4A117002E00A210A4A11700EE012
:10958000312804D10321C943074A117502E00A2199
:10959000044A117003E00A21024A117000BF00BFA3
:1095A00000BD00000C0700206334002000B54249D4
:1095B00009780A390B001BF062FB0A06101A242EE8
:1095C00038424A5D6A782B2803D10B213A4A117040
:1095D00002E00A21384A11706BE0432803D10C21C4
:1095E000354A117002E00A21334A117061E05328B4
:1095F00003D10D21304A117002E00A212E4A117068
:1096000057E0512803D10E212B4A117002E00A21A4
:10961000294A11704DE03A2803D10F21264A1170D2
:1096200002E00A21244A117043E0202803D11021CE
:10963000214A117002E00A211F4A117039E00146E7
:1096400030391E4A117011211B4A117031E02C284B
:1096500003D11221184A11700BE0184909780A2227
:1096600051430246303A8918144A11701221124AA5
:1096700011701EE04F2809D113210F4A11700F49B4
:1096800009781F2902DD00210C4A117011E04B28D6
:1096900007D10321C9430A4A11750A21064A1170EC
:1096A00002E00A21044A117003E00A21024A117003
:1096B00000BF00BF00BD00000C0700201207002003
:1096C0006334002070B50446D04800780A3803009F
:1096D0001BF0D5FA0C070D17212B353E5F80A0C07B
:1096E000E0F32B2C02D10B20C84908708BE1432CEE
:1096F00003D10C20C549087002E00A20C349087054
:1097000081E1432C03D10D20C049087002E00A20FA
:10971000BE49087077E14C2C03D10E20BB4908707C
:1097200002E00A20B94908706DE14B2C03D10F20EB
:10973000B649087002E00A20B449087063E1222C9F
:1097400005D11020B14908700020B14908705AE1D4
:109750002F2C10D0302C1BDB392C19DCAC480078B6
:109760000A214843AA490870204630380978401831
:10977000A74908700CE0A649097808466430A54955
:10978000FEF7C0FD0020A249087011209F49087013
:1097900039E12F2C10D0302C1BDB392C19DC9C48E4
:1097A00000780A2148439A490870204630380978E1
:1097B0004018974908700CE095490978481E95496A
:1097C000091FFEF79FFD00209149087012208F4964
:1097D000087018E12C2C10D0302C1ADB392C18DC36
:1097E0008B4800780A214843894908702046303860
:1097F00009784018864908700BE086490839844882
:109800000078FEF77FFD00208149087013207F4912
:109810000870F8E03A2C10D0302C1ADB392C18DC08
:109820007B4800780A21484379490870204630383F
:1098300009784018764908700BE076490C3974486D
:109840000078FEF75FFD00207149087014206F4911
:109850000870D8E03A2C10D0302C1ADB392C18DCE8
:109860006B4800780A21484369490870204630381F
:1098700009784018664908700BE066491039644859
:109880000078FEF73FFD00206149087015205F4910
:109890000870B8E0222C11D0302C0DDB392C0BDCF9
:1098A0005B4800780A2148435949087020463038FF
:1098B0000978401856490870A0E0A0E055491439CD
:1098C00053480078FEF71EFD5248FEF703FD05469B
:1098D000643D50492846FEF715FD4E48001FFEF72F
:1098E000F9FC451C4B49091F2846FEF70BFD49486A
:1098F0001438FEF7EFFC05460A21FEF721FC0601AD
:1099000044481438FEF7E6FC05460A21FEF718FC29
:109910000E4341498E713F481038FEF7DBFC054687
:109920000A21FEF70DFC06013A481038FEF7D2FC7A
:1099300005460A21FEF704FC0E4337494E713548AF
:109940000C38FEF7C7FC05460A21FEF7F9FB0601B5
:1099500030480C38FEF7BEFC05460A21FEF7F0FB46
:109960000E432D490E712B480838FEF7B3FC05460F
:109970000A21FEF7E5FB060126480838FEF7AAFC97
:1099800005460A21FEF7DCFB0E4323498E70214871
:10999000001FFEF79FFC05460A21FEF7D1FB0601DA
:1099A0001C48001FFEF796FC05460A21FEF7C8FB7F
:1099B0000E4319494E701748FEF78CFC05460A21E4
:1099C000FEF7BEFB06011348FEF784FC05460A219C
:1099D000FEF7B6FB0E4310490E70084600782328A8
:1099E00002DB084614F061FE0020094908700A20D5
:1099F000064908700320C0430849087503E00A209F
:109A00000249087000BF00BF70BD0000450700207C
:109A100046070020E134002047070020633400207F
:109A20002E4909780A2906D00B290ED00C2916D008
:109A30000D294DD11CE0492803D10B21274A117073
:109A400002E00A21254A117046E0442803D10C2186
:109A5000224A117002E00B21204A11703CE03A28A2
:109A600005D100211E4A11700D211C4A117033E0EE
:109A7000522823D04B2814D0302801DB392803DDAD
:109A8000412824DB462822DC1549097815291EDAED
:109A900013490A780978491C114B197011498854E7
:109AA00015E000210E4A117000220E490A75111F9F
:109AB0000D4A11750A21094A117008E00021084A6F
:109AC0001170C91E084A11750A21044A117003E079
:109AD0000A21024A117000BF00BF70470C07002026
:109AE0004E0700207C2900206334002000B5344953
:109AF00009780A390B001BF0C2F807050F19232D4E
:109B000037415D002B2803D10B212D4A117002E053
:109B10000A212B4A117051E0432803D10C21284A15
:109B2000117002E00A21264A117047E0472803D14C
:109B30000D21234A117002E00A21214A11703DE0F3
:109B4000532803D10E211E4A117002E00A211C4A3B
:109B5000117033E04E2803D10F21194A117002E031
:109B60000A21174A117029E03A2803D11021144A1A
:109B7000117002E00A21124A11701FE04B280CD02C
:109B8000302816DB392814DC0E490A780978491C7C
:109B90000C4B19700C4988540BE00021094A1170D4
:109BA0000A21074A117000220749CA73111F074A88
:109BB000117503E00A21024A117000BF00BF00BD09
:109BC0000C070020440700205C290020633400209B
:109BD00000B53D4909780A390B001BF050F80A0618
:109BE000101A242E384248525C6E452803D10B21AE
:109BF000354A117002E00A21334A117061E056289B
:109C000003D10C21304A117002E00A212E4A117052
:109C100057E0452803D10D212B4A117002E00A219B
:109C2000294A11704DE04E2803D10E21264A1170A9
:109C300002E00A21244A117043E0542803D10F2185
:109C4000214A117002E00A211F4A117039E03A28B6
:109C500003D110211C4A117002E00A211A4A117026
:109C60002FE0302802D11121174A117029E02C2849
:109C700003D11221144A117002E00A21124A117014
:109C80001FE0312803D113210F4A117002E00A218D
:109C90000D4A117015E0352807D10321C9430B4A3D
:109CA00011750A21084A117006E00221C943074ACA
:109CB00011750A21044A117003E00A21024A117049
:109CC00000BF00BF00BD00000C070020633400206F
:109CD00010B50446314800780A2804D00B280FD06C
:109CE0000C2855D12DE02C2C06D10B202B490870C7
:109CF00000202B49088002E00A20284908704BE028
:109D00002C2C1AD0302C1BDB392C19DC2448008871
:109D10000A214843224908802046303809884018E3
:109D20001F490880084600881A2809D10C201B49C1
:109D3000087000201A49088002E00A2017490870BC
:109D40002AE00D2C20D0302C21DB392C1FDC1448CC
:109D500000880A2148431249088020463038098883
:109D600040180F49088020F017F90D4909888842EA
:109D70000DD1232005F07AFA0320C0430949087564
:109D80000A200649087002E00A200449087003E02E
:109D90000A200249087000BF00BF10BD0C07002058
:109DA000520700206334002000B5344909780A398D
:109DB0000B001AF064FF0906101A242E384248528C
:109DC0006000452803D10B212C4A117002E00A21C2
:109DD0002A4A117050E0562803D10C21274A1170ED
:109DE00002E00A21254A117046E0452803D10D21E1
:109DF000224A117002E00A21204A11703CE04E28EC
:109E000003D10E211D4A117002E00A211B4A117074
:109E100032E0542803D10F21184A117002E00A21C0
:109E2000164A117028E03A2803D11021134A117004
:109E300002E00A21114A11701EE0302802D11121DE
:109E40000E4A117018E02C2803D112210B4A117010
:109E500002E00A21094A11700EE0362807D10321D9
:109E6000C943074A11750021044A117002E00A2112
:109E7000024A117000E000BF00BF00BD0C070020C7
:109E80006334002070B50446564800780A38030051
:109E90001AF0F5FE0805A10F19232D3A59A14E2CF1
:109EA00003D10C204F49087002E00A204D49087088
:109EB00095E04E2C03D10D204A49087002E00A209B
:109EC000484908708BE04D2C03D10E20454908709D
:109ED00002E00A204349087081E0492C03D10F2099
:109EE0004049087002E00A203E49087077E03A2CA9
:109EF00006D100213C48817110203A49087002E0E7
:109F00000A20384908706AE02C2C14D0302C19DB58
:109F1000392C17DC34488079092808DA32488179ED
:109F20008079401C304A9071101F44540AE0002090
:109F30002D49887106E000212C488172C1721120E0
:109F4000284908704BE02C2C3BD00D2C39D02749E8
:109F5000C87A897A0002084301218902884228DAF6
:109F600021480838FEF7B6F9451C1F49083928462C
:109F7000FEF7C8F9302C01DB392C07DD412C01DB61
:109F8000462C03DD612C25DB662C23DC1748C17AC7
:109F9000807A09020143154AD07A927A000210436E
:109FA000401C82B211488272120AC2720C304454B0
:109FB00010E000210D488172C1720A200949087021
:109FC00008E00020084948720120203988750A20DD
:109FD0000449087003E00A200249087000BF00BF6E
:109FE00070BD00000D07002083340020632E002088
:109FF00000B54B4909780A390B001AF040FE0D08EC
:10A000000E1826303A444E58626C76808A003A2800
:10A0100002D10B21424A11707FE0202803D10C218C
:10A020003F4A117002E00A213D4A117075E0522842
:10A0300003D10D213A4A117006E00221C943394A81
:10A0400011750A21364A117067E0452803D10E21A7
:10A05000334A117002E00A21314A11705DE047284D
:10A0600003D10F212E4A117002E00A212C4A1170EF
:10A0700053E0492803D11021294A117002E00A2136
:10A08000274A117049E0532803D11121244A117045
:10A0900002E00A21224A11703FE0542803D1122124
:10A0A0001F4A117002E00A211D4A117035E045284F
:10A0B00003D113211A4A117002E00A21184A1170C3
:10A0C0002BE0522803D11421154A117002E00A2115
:10A0D000134A117021E0452803D11521104A11704F
:10A0E00002E00A210E4A117017E0442803D116211C
:10A0F0000B4A117002E00A21094A11700DE04B2849
:10A1000006D10321C943074A11750A21044A117077
:10A1100003E00A21024A117000BF00BF00BD000029
:10A120000C0700206334002000B5264909780A395D
:10A130000B001AF0A4FD07050B11171D2329410080
:10A14000542802D10B211F4A117039E0492802D14D
:10A150000C211C4A117033E04E2802D10D21194AFE
:10A1600011702DE0442802D10E21164A117027E00B
:10A170003A2802D10F21134A117021E0202802D180
:10A180001021104A11701BE0332804D10321C94368
:10A190000D4A11750CE0362804D10321C9430A4A3F
:10A1A000117505E0312803D10221C943064A117512
:10A1B0000A21044A117003E00A21024A117000BF0B
:10A1C00000BF00BD0C0700206334002010B504461A
:10A1D000304800780A3803001AF051FD07050F19BE
:10A1E000232D37415600542C03D10B2029490870E8
:10A1F00002E00A20274908704AE0492C03D10C20CC
:10A200002449087002E00A202249087040E04E2CE0
:10A2100003D10D201F49087002E00A201D49087073
:10A2200036E0442C03D10E201A49087002E00A20BF
:10A23000184908702CE03A2C03D10F2015490870FA
:10A2400002E00A201349087022E0202C03D11020DC
:10A250001049087002E00A200E49087018E0342CFA
:10A260000AD1232005F002F80320C0430A490875EB
:10A270000A200849087006E00220C0430649087514
:10A280000A200449087003E00A200249087000BF50
:10A2900000BF10BD0C0700206334002070B50446D9
:10A2A000F84800780A3803001AF0E9FC120A154A47
:10A2B0007EB0B9E1F8F6F5F4F3F2F1F0EFEEEDEC83
:10A2C0002C2C07D10020F0490870F04908800B20A1
:10A2D000EC4908705EE22C2C1DD100200021EB4AD5
:10A2E000118000BF0CE0E94909880A225143E74A7E
:10A2F0001180E749095C12888918E44A1180401CE2
:10A30000E14909788842EEDB0021DF4A11700C2117
:10A31000DC4A117013E0DC4800780A280CDA204689
:10A320003038C1B2DA48D84A12788154D648007819
:10A33000401CD549087002E00020D2490870EDE3C6
:10A340002C2C1DD100200021D24A116000BF0CE04E
:10A35000D04909680A225143CE4A1160CC49095CB0
:10A3600012688918CB4A1160401CC7490978884295
:10A37000EEDB0021C44A11700D21C24A117012E0B7
:10A38000C14800780A280BDA20463038C049BE4A56
:10A3900012788854BC480078401CBB49087002E021
:10A3A0000020B8490870B9E32C2C1AD100200021F4
:10A3B000B94A118000BF0CE0B74909880A2251430D
:10A3C000B54A1180B249095C12888918B24A1180D5
:10A3D000401CAD4909788842EEDB0E21A94A117074
:10A3E00013E0A948007805280CDA20463038C1B2BD
:10A3F000A748A54A12788154A3480078401CA24976
:10A40000087002E000209F49087087E3222C05D1E4
:10A4100000209D4908700F209A4908707EE3222C85
:10A4200013D100250A219D48FDF72DFF00BF04E050
:10A430009748405D994948556D1C9348007885427E
:10A44000F6DB10208F49087010E08F4800780A284A
:10A4500009DA8F488C49097844548B480078401CAD
:10A460008949087002E000208649087056E32C2CC8
:10A4700007D100208449087085490870112081495E
:10A4800008704BE346E39CE28CE280E256E24AE24B
:10A4900013E280E108E17EE072E0FFE72E2C57D165
:10A4A00079480078012804D1794840787C490880AF
:10A4B0003AE075480078022809D1754840780A21A9
:10A4C0004843734989784018754908802CE06E48E4
:10A4D000007803280FD16E484078642148436C49C6
:10A4E00089780A22514340186949C978401800B256
:10A4F0006B49088018E064480078042814D1644847
:10A5000040787D21C90048436149897864225143DC
:10A5100041185F48C0780A22504308185C490979FD
:10A52000401800B25E4908805D4800880A2148430F
:10A5300000B25B49088056480078012804D10846DB
:10A540000088404200B2088012204E49087016E090
:10A550002D2C03D101204E49087010E04A480078A4
:10A5600004280CDA20463038C1B247480078401C35
:10A57000474A115444480078401C43490870CDE2D2
:10A580002C2C07D100204049087041490870132045
:10A590003C490870C2E22C2C5CD13B480078012871
:10A5A00004D13B4840783F4908803AE0364800787B
:10A5B000022809D1364840780A214843344989782D
:10A5C0004018384908802CE02F48007803280FD124
:10A5D0002F484078642148432D4989780A22514305
:10A5E00040182B49C978401800B22E49088018E05D
:10A5F00025480078042814D1254840787D21C900D9
:10A600004843234989786422514341182048C0783F
:10A610000A22504308181E490979401800B22149FE
:10A620000880204800880A21484300B21D4908805C
:10A6300017480078012804D108460088404200B23B
:10A6400008800020104908701149087014200D4935
:10A65000087016E02D2C03D101200D49087010E080
:10A660000948007804280CDA20463038C1B2064880
:10A670000078401C064A115403480078401C0249E7
:10A6800008704BE20C07002015070020200700206F
:10A69000F93400202407002028070020043500207A
:10A6A0002A0700202C0700202C2C5CD1FE480078C3
:10A6B000012804D1FD484078FD4908803AE0FA4875
:10A6C0000078022809D1F94840780A214843F7491F
:10A6D00089784018F64908802CE0F3480078032870
:10A6E0000FD1F248407864214843F04989780A2222
:10A6F00051434018ED49C978401800B2EC49088030
:10A7000018E0E9480078042814D1E84840787D2111
:10A71000C9004843E5498978642251434118E34818
:10A72000C0780A2250430818E0490979401800B25D
:10A73000DF490880DE4800880A21484300B2DC492E
:10A740000880DA480078012804D108460088404291
:10A7500000B208800020D4490870D4490870152040
:10A76000D449087016E02D2C03D10120CF49087080
:10A7700010E0CD48007804280CDA20463038C1B209
:10A78000C9480078401CC94A1154C7480078401C89
:10A79000C5490870C2E12C2C73D1C3480078012848
:10A7A0000BD1C2484078C4490880084600880A2175
:10A7B000484300B2C04908804FE0BB4800780228F7
:10A7C00010D1BA4840780A214843B84989784018DE
:10A7D000B9490880084600880A21484300B2B649B2
:10A7E00008803AE0B0480078032816D1AF48407896
:10A7F00064214843AD4989780A2251434018AB4946
:10A80000C978401800B2AC490880084600880A217F
:10A81000484300B2A84908801FE0A34800780428F4
:10A820001BD1A24840787D21C90048439F498978BF
:10A830006422514341189D48C0780A2250430818A9
:10A840009A490979401800B29B4908800846008857
:10A850000A21484300B298490880944800780128AA
:10A8600005D195480088404200B2934908800020F5
:10A870008D4908708D49087016208E4908701BE0BC
:10A88000FFE72D2C03D101208849087014E0864889
:10A89000007804280DDA20463038C1B2834A824855
:10A8A0000078401C115480480078401C7E49087094
:10A8B00002E00A207F49087030E12C2C1FD10020D3
:10A8C00000217E4A118000BF0CE07C4909880A22E1
:10A8D00051437A4A11807549095C12888918774A70
:10A8E0001180401C704909788842EEDB00216E4AD5
:10A8F00011706E4A117017216E4A117012E06A4889
:10A90000007804280BDA204630386849664A127805
:10A91000885465480078401C6349087002E00A20AA
:10A9200064490870FAE0222C07D100205E490870C3
:10A930005E49087018205F490870EFE0222C14D19E
:10A94000002000BF04E05949095C5D4A1154401CD5
:10A95000554909788842F6DB0021534A1170534A61
:10A9600011701921534A117010E04F4800780A28DD
:10A9700009DA4E484C49097844544B480078401C49
:10A980004949087002E000204A490870C6E02C2CB2
:10A9900007D1002044490870444908701A204549ED
:10A9A0000870BBE02C2C07D140480078454908804E
:10A9B0001B204049087003E0204630383B490870AE
:10A9C000ACE02D2C03D1012038490870A1E0302CD7
:10A9D00017DB392C15DC3448007804280DDA2046C2
:10A9E0003038C1B2314A30480078401C11542E48EA
:10A9F0000078401C2C4908708BE00A202D49087013
:10AA000087E02948007801280BD1284840782E4952
:10AA10000880084600880A21484300B22A49088075
:10AA200013E02148007802280FD1204840780A21FD
:10AA300048431E4989784018234908800846008801
:10AA40000A21484300B220490880174800780328AB
:10AA500016D11648407864214843144989780A225F
:10AA6000514340181149C978401800B2164908806E
:10AA7000084600880A21484300B21349088032E0A2
:10AA80000948007804282ED1084840787D21C90063
:10AA90004843064989786422514341180348C078E5
:10AAA0000A225043081811E015070020F93400204D
:10AAB0002E0700200C07002030070020320700205E
:10AAC0000E3500203407002036070020144909798C
:10AAD000401800B213490880084600880A214843FC
:10AAE00000B2104908800E480078012805D10D48B1
:10AAF0000088404200B20B49088000200A490870D3
:10AB0000074908700A20094908700320C043084912
:10AB1000087503E00A200549087000BF00BF70BD3A
:10AB2000F934002036070020150700200C0700200C
:10AB3000633400202A4909780A2906D00B290AD053
:10AB40000C291ED00D2945D125E04F2802D10B211B
:10AB5000234A117042E04B2806D10121214A11708D
:10AB60000C211F4A11700BE0522806D100211D4A0A
:10AB700011700C211A4A117002E00A21184A117052
:10AB80002CE00D2803D10D21154A117002E00A2195
:10AB9000134A117022E00A2818D1124909780029B5
:10ABA00004D00321C943104A117503E00221C943AF
:10ABB0000D4A11750D49097A0B2903D10A21084A5A
:10ABC000117006E00021064A117002E00A21044AD1
:10ABD000117003E00A21024A117000BF00BF7047E4
:10ABE0000C0700204207002063340020632E002061
:10ABF00000B5224909780A390B001AF040F8080517
:10AC00000B11171D23292F392B2802D10B211B4A89
:10AC1000117031E0512802D10C21184A11702BE03B
:10AC2000492802D10D21154A117025E04F2802D183
:10AC30000E21124A11701FE0502802D10F210F4A35
:10AC4000117019E0452802D110210C4A117013E04F
:10AC50004E2802D11121094A11700DE03A2803D182
:10AC60000321C943064A11750A21044A117003E001
:10AC70000A21024A117000BF00BF00BD0C0700206E
:10AC8000633400200E4909780A2902D00B2911D11A
:10AC900005E0572802D10B21094A11700EE04E2819
:10ACA00004D10321C943074A117502E00A21044A6D
:10ACB000117003E00A21024A117000BF00BF704703
:10ACC0000C07002063340020144909780A2904D0B5
:10ACD0000B2908D00C291BD10FE0452802D10B21EC
:10ACE0000E4A117018E0452803D10C210B4A11704F
:10ACF00002E00A21094A11700EE0502804D1032114
:10AD0000C943074A117502E00A21044A117003E0A1
:10AD10000A21024A117000BF00BF70470C070020D3
:10AD20006334002000B5634909780A390B0019F033
:10AD3000A6FF0B07111B252F39434D697394BB00E8
:10AD4000222803D10B215B4A117002E00A21594AE3
:10AD50001170ADE0722803D10C21564A117002E047
:10AD60000A21544A1170A3E0652803D10D21514AEC
:10AD7000117002E00A214F4A117099E0632803D153
:10AD80000E214C4A117002E00A214A4A11708FE0EC
:10AD9000762803D10F21474A117002E00A21454A63
:10ADA000117085E0222803D11021424A117002E07F
:10ADB0000A21404A11707BE02C2803D111213D4A21
:10ADC000117002E00A213B4A117071E000213A4AF9
:10ADD0009172D172394A1180302806D10121384A46
:10ADE00051721221334A11700BE0312806D1022131
:10ADF000334A517212212F4A117002E00A212D4A62
:10AE0000117055E02C2803D113212A4A117002E059
:10AE10000A21284A11704BE00A2810D030281BDB89
:10AE2000392819DC254909880A225143234A11800F
:10AE30000146303912888918204A11800CE01F49D8
:10AE4000098801229202914203DA1421194A1170F1
:10AE500002E00021174A11702AE0174AD17A927A4B
:10AE600009021143154A1288914212DA124AD17A24
:10AE7000937A0A021A43104BD97A9B7A0902194332
:10AE8000491C8BB20C498B721B0ACB720C31885453
:10AE900009E00321C9430A4A203A1175012191753D
:10AEA0000A21044A117003E00A21024A117000BF0E
:10AEB00000BF00BD0F070020632E002010070020F8
:10AEC0008334002010B50446484800780A3803004F
:10AED00019F0D5FE0B07111B252F39434D57616E15
:10AEE0008600442C03D10B204049087002E00A2060
:10AEF0003E49087078E0492C03D10C203B4908708A
:10AF000002E00A20394908706EE0532C03D10D206D
:10AF10003649087002E00A203449087064E0432C86
:10AF200003D10E203149087002E00A202F49087031
:10AF30005AE04F2C03D10F202C49087002E00A2060
:10AF40002A49087050E0562C03D110202749087078
:10AF500002E00A202549087046E0452C03D1112063
:10AF60002249087002E00A20204908703CE0522C77
:10AF700003D112201D49087002E00A201B49087005
:10AF800032E03A2C03D113201849087002E00A205D
:10AF90001649087028E02C2C09D1002014490870AB
:10AFA0000A211448FDF76FF91420104908701BE0BE
:10AFB0002C2C0CD00E4800780A2810D20C480178AE
:10AFC0000078401C0A4A10700A48445407E00320E5
:10AFD000C04308492B3908750A200449087003E06A
:10AFE0000A200249087000BF00BF10BD4F070020B3
:10AFF000500700208E340020014800787047000080
:10B000004100002003480078002801D1012070474A
:10B010000020FCE7400000200020044909780029B6
:10B0200001D1012000E00020704700004000002016
:10B0300070B555480078030019F021FE050405108D
:10B040002593A3009EE0012000F0CAFD002804D152
:10B050000EF0D3FF02204C49087093E04B48007873
:10B0600000F008F9012000F017F900F079F915F067
:10B0700001FE4749086015F0FDFD464908600320C0
:10B08000414908707EE0012000F022F9012855D1E5
:10B0900015F0F0FD3F49086015F0ECFD3C490968EA
:10B0A000401A3D49096888425AD3002400F01CF92F
:10B0B00004463A48406800193849486038480078E2
:10B0C000002803D108468460046013E03348806898
:10B0D000A04201D2204601E0304880682F498860B4
:10B0E00008460068A04201D9204601E02B480068CC
:10B0F0002A4908602A480078401CC0B228490870D4
:10B1000028490978884215DB0025244840682349EE
:10B110000968401A21498968451A22480078811E29
:10B120002846FCF7F7FF2049096808600420164903
:10B13000087002E002201449087011E015F09AFD31
:10B1400014490968401A64280AD900F00FF9174811
:10B150000078022108431549087004200A49087044
:10B1600010E000F0A1F800F047FC0021102015F0DD
:10B170000DFA01200E490968087000200249087084
:10B1800000E000BF00BF70BD400000205100002063
:10B1900054000020580000204800002054130020D4
:10B1A00050000020520000204400002041000020F8
:10B1B0004C00002010B500F077F800F01DFC0021D5
:10B1C000102015F0E3F910BDF8B505460C461646FB
:10B1D0001F46032C00D20324502C00D950241B49B5
:10B1E00006980860192D0ADD1948007801210843E6
:10B1F000174908700120154909680870F8BD1548FD
:10B200000760002011490968087013490870134944
:10B210004860086088600E4908701148057011493F
:10B220000C70114806600EF002FF0121102015F08D
:10B23000ADF900F0EBFB00F041F80121084614F0F5
:10B24000C9F901200949087000BFD7E74C00002068
:10B250004100002044000020500000205413002032
:10B260005100002052000020480000204000002033
:10B2700070470000014607484068FF22F1329043C2
:10B280000A01FF23F1331A401043024A50600020A4
:10B2900070470000002400400249496B8143014A85
:10B2A00051637047802400400348406840084000D4
:10B2B000014948607047000000240040034840688E
:10B2C00040084000401C014948607047002400408D
:10B2D00001460448006B0840002801D00120704757
:10B2E0000020FCE7802400400148006A704700000D
:10B2F0008024004010B50446002C01D1042010BD6C
:10B3000001201649486002201AF020FB6078A188CD
:10B310000843E188084361880843218908430F49AD
:10B32000496808430D494860084680680915884304
:10B33000217889020122920211400843074988605E
:10B340000846806804218843A17A890004221140BC
:10B350000843024988600020D1E700000024004033
:10B360000120014908607047C024004000200149C5
:10B3700008607047C024004030B50A4600210EE046
:10B38000D400A41A074D6419635C04785C4004700F
:10B390000478AA256C400470401C4C1CE1B20729BB
:10B3A000EEDB30BD54C80200F0B589B012F0C4FF26
:10B3B00010210840002810D0042012F0E5FFFB48BF
:10B3C0000088401CF9490880E1210901F7480088FC
:10B3D000FCF7B6FE88B2F549088012F0ADFF2021D7
:10B3E0000840002822D0052012F0CEFFF048007857
:10B3F000401CEF490870084600783C2816DB002006
:10B400000870EC48FCF766FFE12109014418E9499E
:10B410002046FCF777FFE748001DFCF75BFF04467A
:10B42000233CE449091D2046FCF76CFFE248007804
:10B43000002804D001280ED002287DD1A8E102F016
:10B44000A1FF002806D1D9480088DC490860012006
:10B45000D9490870CCE102F095FF01286DD1002197
:10B4600007910691D1480088D4490968884207D3DA
:10B47000CE480088D1490988401AD149088009E09E
:10B48000CA480088E12109014018CC490988401ABE
:10B49000CB49088008201EF055FD772807D1C84801
:10B4A00000884B21C9004018C54908800BE00820DE
:10B4B0001EF048FD552806D1C1480088E121C90089
:10B4C0004018BF4908800021082020F039F8B94809
:10B4D0000C30FCF7FFFEBA4909884418B5490C3115
:10B4E0002046FCF70FFFB348417C027C0802104362
:10B4F000401C81B2AF480174090A417407A80FF0DB
:10B50000CDF906A80FF0BCF90A216A461C20105E8E
:10B51000FCF716FE00B207900A216A461820105E5A
:10B52000FCF70EFE00B2069004201EF00BFD012871
:10B530003ED1A348008801E056E128E1FDF786F9F5
:10B54000A04AA14B01910090FDF77AF80591049073
:10B550009848001DFCF7BEFE0746FDF777F90391FA
:10B560000290059B049AFDF75DF80546FDF7A8F9E2
:10B5700004469049091DFCF7C5FE04F043FD002870
:10B5800015D192480078401C9049087007218F48D7
:10B590000078FCF7D5FDC8B28C49087008460178E0
:10B5A00002201FF0CDFF01210A201FF0C9FFEAE0B1
:10B5B00069461C20085E002821DA81480088FDF7D2
:10B5C00045F906467F4A824BFDF73AF804460D4698
:10B5D0007848001DFCF77EFE0646FDF737F9224647
:10B5E0002B4601910090FDF71DF803910290FDF7A5
:10B5F00067F97049091D0590FCF784FEC3E06946B0
:10B600001820085E7721C943884220DA6C480088F8
:10B61000FDF71CF906466B4A6D4BFDF711F80391D7
:10B6200002906448001DFCF755FE0646FDF70EF932
:10B6300001910090039B029AFCF7F4FF0446FDF78A
:10B640003FF95C49091D0590FCF75CFE9BE06946EB
:10B650001820085E7221C943884221DA58480088C0
:10B66000FDF7F4F85B4A5C4B01910090FCF7E8FFB2
:10B6700004460D464F48001DFCF72CFE0190FDF7D7
:10B68000E5F8064622462B46FCF7CCFF03910290D4
:10B69000FDF716F94749091D0590FCF733FE72E0E6
:10B6A00069461820085E6821C943884221DA444867
:10B6B0000088FDF7CBF80646424A5242474BFCF75A
:10B6C000BFFF019100903B48001DFCF703FE0646BA
:10B6D000FDF7BCF80446019B009AFCF7A3FF039119
:10B6E0000290FDF7EDF83349091D0590FCF70AFEBD
:10B6F00049E069461820085E5921C943884221DA89
:10B700002F480088FDF7A2F82E4A2F4B0191009098
:10B71000FCF796FF06460F462648001DFCF7DAFDAB
:10B720000190FDF793F8044632463B46FCF77AFF5A
:10B7300003910290FDF7C4F81E49091D0590FCF71E
:10B74000E1FD20E01E480088FDF780F806461D4A0E
:10B750005242234BFCF774FF019100901548001DE5
:10B76000FCF7B8FD0646FDF771F80446019B009A08
:10B77000FCF758FF03910290FDF7A2F80D49091D4F
:10B780000590FCF7BFFD02200B49087000BF2FE0B9
:10B7900001F004FA012808D1124B1822D0210548E3
:10B7A00001F060FC00200449087021E070050020D1
:10B7B00072050020C02600206105002064050020DD
:10B7C000740500203333333333331F4084050020A6
:10B7D00033B330406666666666662D40CCCC214049
:10B7E000CCCC1A406005002000205A49087000BFE8
:10B7F00000BF59480078002802D001284FD10BE043
:10B800000AF052FE002806D15448008854490860C6
:10B8100001205149087046E00AF046FE01283DD15A
:10B820004E4800884E490968884207D34B48008833
:10B830004B490988401A4B49088009E0474800886D
:10B84000E1210901401846490988401A4549088004
:10B85000454800684349098840184349086008463C
:10B8600000683C2817D9084600683C3808603F4803
:10B87000FCF730FD04463C343C492046FCF742FDD1
:10B880003A48001FFCF726FD0446153C3749091FBE
:10B890002046FCF737FD00202F49087003E0002008
:10B8A0002D49087000BF00BF31480078002802D041
:10B8B000012848D10BE018F07BFB002806D127486F
:10B8C00000882C4908600120294908703FE018F0E1
:10B8D0006FFB012836D12148008826490968884233
:10B8E00007D31E48008823490988401A1D4908804B
:10B8F00009E01A480088E121090140181D4909881A
:10B90000401A1849088019480838C17C827C08020E
:10B91000104314490988401881B2144808388174CA
:10B92000090AC174001DFCF7D5FC0E4909882A22BA
:10B930005143441A0D49091F2046FCF7E3FC00203F
:10B940000B49087003E000200949087000BF00BFE0
:10B9500009B0F0BD610500206205002070050020DF
:10B9600068050020740500206C050020C826002012
:10B97000850500208805002007480078002809D1A7
:10B9800006480078002805D105480078002801D134
:10B99000012070470020FCE76105002062050020BF
:10B9A00085050020014680200840002801D0084677
:10B9B0007047302905DB392903DC08463038C0B22E
:10B9C000F6E7612905DB662903DC08465738C0B273
:10B9D000EEE7412905DB462903DC08463738C0B2CB
:10B9E000E6E70846E4E701460A110A235A430B0733
:10B9F0001B0FD218D0B270470348006802210840DC
:10BA000001490860704700000024004010B5054857
:10BA100000680121084303490860022019F096FFDD
:10BA200010BD00000024004030B502460020140282
:10BA3000044D63191C68240C24048DB22C431C6033
:10BA400030BD0000000C004030B50246002014025A
:10BA5000044D63195C68240C24048DB22C435C6093
:10BA600030BD0000000C004010B5014600200B0264
:10BA7000014C1A19906810BD000C004030B5024608
:10BA800000201402024D63199C68996030BD0000CB
:10BA9000000C004070B5024600201402054D6319E9
:10BAA0001C6BAD14AC430D030126360335402C430B
:10BAB0001C6370BD000C004010B5014600200B0255
:10BAC000034C1A19D3685B085B005B1CD36010BD84
:10BAD000000C004010B5014600200B02034C1A195F
:10BAE000D3685B085B00D36010BD0000000C004011
:10BAF00070B503460A4600201C02224D6119CC682D
:10BB0000AD00AC4315782D030326360335402C4396
:10BB1000CC60CC6801256D02AC4355786D020126DE
:10BB2000760235402C43CC60CC687510AC439578D8
:10BB30002D02761035402C43CC60CC687025AC4388
:10BB4000D5782D01702635402C43CC60CC68082573
:10BB5000AC431579ED00082635402C43CC60CC6809
:10BB60000425AC435579AD00042635402C43CC6008
:10BB7000CC680225AC4395796D00022635402C43F4
:10BB8000CC6070BD000C004010B500F009F910BD8C
:10BB900070B5044600252C2C1BDA15F06BF8054611
:10BBA000A0000D490858A84203D8A00008582D1A33
:10BBB00006E0A000084908580021C943081A4519A1
:10BBC000A00006490858A84201D8002070BD0120F5
:10BBD000FCE70020FAE70000B00C0020600D002018
:10BBE00070B504460025182C1BDA15F043F80546FD
:10BBF000A0000D490858A84203D8A00008582D1AE3
:10BC000006E0A000084908580021C943081A451950
:10BC1000A00006490858A84201D8002070BD0120A4
:10BC2000FCE70020FAE70000F00B0020500C002099
:10BC30000148007870470000C803002010B506488E
:10BC4000FCF752FB054B064A43404A40134301D1DF
:10BC5000012010BD0020FCE70E1A0020B8A7F6E571
:10BC6000D4C3B2A101480078704700009C020020B4
:10BC700070B504460025002614F0FCFF064609486E
:10BC80000068351A0848844203D1A54201D3012037
:10BC900070BD0648844203D1A54201D30120F7E7D5
:10BCA0000020F5E71800002050C30000C02709005D
:10BCB0000148007870470000C9030020FFB583B039
:10BCC00006460F461C4638461EF072F9029005984B
:10BCD0001EF06EF901906078217800020843002878
:10BCE00006DD6078217800020843164988420FDBA0
:10BCF00060782178000208431249083188421EDD2D
:10BD000060782178000208430E490931884216DA2A
:10BD10006078217800020843B04203D009480F3010
:10BD200086420CD1A01C1EF043F9054602988542BC
:10BD300005D30198854202D8012007B0F0BD00204C
:10BD4000FBE70000F0FF00000148007870470000AA
:10BD5000520300200148006870470000540300208F
:10BD6000002002498872C87270470000172900201D
:10BD70000020014908707047F602002000200149A8
:10BD8000C87570476334002000200149087070476F
:10BD90009C020020002001490870704752030020D7
:10BDA00010B5012015F07EF801280DD115F074F8BA
:10BDB00057490860084600685649884205D115F081
:10BDC00087F8FF205449087096E0514800685149AF
:10BDD000884246D215F07CF850480078002803D0FD
:10BDE0004E48007801281ED101204C49087048496E
:10BDF0000968484A501A4949491CFCF783FA4849DE
:10BE0000C968491C4805400D4549C968C90AC902A5
:10BE10000143434AD16015F051F842480078401C74
:10BE20004049087068E03D48401CFCF753FA384927
:10BE30000968384A511A88420FD23949C968491CE1
:10BE40004805400D3649C968C90AC9020143344A48
:10BE5000D160FF20304908704EE0FF202E49087065
:10BE60004AE02B4800682B49884245D915F030F844
:10BE70002A480078002803D02848007802281ED1DC
:10BE800002202649087022490968224A881A234953
:10BE9000491CFCF737FA2249C968491E4805400D7C
:10BEA0001F49C968C90AC90201431D4AD16015F07A
:10BEB00005F81C480078401C1A4908701CE0174817
:10BEC000401CFCF707FA12490968124A891A88428D
:10BED0000FD21349C968491E4805400D1049C96869
:10BEE000C90AC90201430E4AD160FF200A490870FD
:10BEF00002E0FF2008490870022014F0D3FF012857
:10BF000004D114F0E5FFEE200349087010BD0000D5
:10BF10000403002000093D00FA020020FC0200207A
:10BF200000200040FB02002010B5002014F006FBAA
:10BF3000002014F017FB112014F076FB022014F0FF
:10BF400061FB0121022014F093F9022014F090FB10
:10BF5000042014F043FB0121002014F089F9002093
:10BF600014F086FB0121062002F098FE002002F06A
:10BF7000F9FE01211C2014F009FB10BD002001492D
:10BF800008707047C404002010B500F001F810BD1F
:10BF9000F8B5B3480078030018F071FE05040FD916
:10BFA000FEFDFC000020AF4908700120AC4908707C
:10BFB000FF202D301FF0D2FA50E119F073F900285C
:10BFC0007ED10D24A8480688A8480568002751E0BE
:10BFD000E85D0A2808DAE85D3030C2B22046611C0C
:10BFE0008CB2A3490A543EE0E85D642816DAE85DA5
:10BFF0000A21FCF7A5F83030C2B22046611C8CB291
:10C000009B490A54E85D0A21FCF79AF83031CAB21C
:10C010002046611C8CB296490A5424E0E85D6421F4
:10C02000FCF78EF83030C2B22046611C8CB29049C9
:10C030000A54E85D0A21FCF783F80A210090FCF716
:10C040007FF83031CAB22046611C8CB288490A544C
:10C05000E85D0A21FCF774F83031CAB22046611C51
:10C060008CB283490A542E222046611C8CB280492E
:10C070000A547F1C042FABDB601E84B222222046B0
:10C08000611C8CB27A490A542C222046611C8CB265
:10C0900077490A5477493046FCF752F83030C2B23B
:10C0A0002046611C8CB272490A5472493046FCF732
:10C0B00047F800917D21C9000098FCF741F800E0A5
:10C0C00044E03030C2B22046611C8CB268490A5448
:10C0D0007D21C9003046FCF733F8009164210098B7
:10C0E000FCF72EF83030C2B22046611C8CB2604999
:10C0F0000A5464213046FCF723F800910A21009885
:10C10000FCF71EF83030C2B22046611C8CB2584990
:10C110000A540A213046FCF713F83031CAB22046DF
:10C12000611C8CB252490A540D222046611C8CB20B
:10C130004F490A54122221464D4810F0C1F82320DD
:10C140001FF018FA02204649087000BF86E00EF082
:10C1500013FB001D002809D1424908700320404903
:10C160000870FF202D301FF0F9F926E019F09FF834
:10C17000002804D00EF000FBC01C00281DD1394857
:10C180000078401C3749087008460078012811DB08
:10C19000002002E05EE027E010E008703648FCF77F
:10C1A00099F8A521017000202D490870A820334975
:10C1B000087002E001202A4908704FE019F072F877
:10C1C000002810D12E480068FCF774F884B21B22B6
:10C1D00021462B48006810F073F802201FF0CAF9BE
:10C1E00004201F49087039E00EF0C6FA001D00282F
:10C1F0000DD11C4908702048FCF76CF8A321017090
:10C20000002017490870A9201C49087021E019F086
:10C210004EF800281DD113480078401C11490870C1
:10C220000846007801280DDB002008701248FCF752
:10C2300051F8A5210170002009490870A8200F4974
:10C24000087006E0032006490870FF202D301FF01B
:10C2500085F903E000200249087000BF00BFF8BD67
:10C26000960500204E060020A8050020A405002009
:10C270004F06002010270000912900208E05002085
:10C280008406002010B500F001F810BD70B5C1485B
:10C290000078002804D003280AD004287ED13CE18D
:10C2A0000320BC490870FF202D301FF057F96FE1C3
:10C2B00018F0F8FF002872D10824002504E0B648E1
:10C2C000405DB64948556D1C082DF8DBB44A517ADB
:10C2D000127A090211430846B249FBF731FF3030A8
:10C2E000C2B22046611C8CB2AC490A54AC4A517AA5
:10C2F000127A090211430846AA49FBF721FF0E46AC
:10C300007D21C9003046FBF71BFF3030C2B220460A
:10C31000611C8CB2A1490A54A14A517A127A0902CD
:10C32000114308467D21C900FBF70AFF0E46642130
:10C330003046FBF705FF3030C2B22046611C8CB29C
:10C3400096490A54964A517A127A090211430846CC
:10C350006421FBF7F5FE0E460A213046FBF7F0FE9E
:10C360003030C2B22046611C8CB28C490A548C4ACF
:10C37000517A127A0902114308460A21FBF7E0FEBE
:10C380003031CAB22046611C8CB284490A542C2236
:10C390002046611C8CB281490A5401E0F4E0BBE004
:10C3A000002545E07E48001DFBF794FF405D00112D
:10C3B0000A280CDB7A48001DFBF78CFF405D00115A
:10C3C00037302146621C94B2744A50540BE07448D2
:10C3D000001DFBF77FFF405D001130302146621CDD
:10C3E00094B26E4A50546E48001DFBF773FF405DD7
:10C3F0000007000F0A280DDB6948001DFBF76AFFE4
:10C40000405D0007000F37302146621C94B2634A3A
:10C4100050540CE06248001DFBF75CFF405D0007D4
:10C42000000F30302146621C94B25C4A50546D1C9F
:10C430005B49487A097A00020843A842B2DC5A48AC
:10C44000007B80210840002828D05748007B8007C7
:10C45000800F002822D02C222046611C8CB24F492C
:10C460000A5431222046611C8CB24C490A543022B5
:10C470002046611C8CB249490A542046611C8CB28A
:10C4800046490A540D222046611C8CB243490A5485
:10C490003722214641480FF013FF36E04248807AA8
:10C4A000552804D0404876308078552822D12C2257
:10C4B0002046611C8CB239490A5431222046611C45
:10C4C0008CB236490A5430222046611C8CB2334962
:10C4D0000A542046611C8CB230490A540D22204671
:10C4E000611C8CB22D490A54372221462B480FF08B
:10C4F000E7FE0AE00D222046611C8CB227490A544F
:10C500001622214625480FF0DBFE04201FF032F8EA
:10C5100004202049087000BF3AE00EF02DF9001DFC
:10C5200000280DD121490870A920214908701C4814
:10C53000FBF7D0FEA421017000201649087022E00C
:10C540000EF01AF9C01C002803D018F0B0FE002825
:10C5500019D116480078401C144908700846007824
:10C5600001280DDB002008700D48FBF7B3FEA52164
:10C570000170A8200E49087000200649087002E0EA
:10C5800004200449087003E000200249087000BF3D
:10C5900000BF70BD980500209AC802009B290020AA
:10C5A0009129002010270000842600208806002002
:10C5B0008E05002000200149087070479605002074
:10C5C00070B546480078002806D0012805D0032819
:10C5D00074D006287CD123E07EE000F0DFFA012849
:10C5E0001DD13F48007816280FD0DC223D493E4837
:10C5F000FBF730FE3D4BDC22012149023A4800F0B6
:10C6000031FD03203549087009E0384BDC223649FA
:10C610000120400200F0E0FC0620304908705BE099
:10C6200000F0BCFA012846D1002500242EE0A1002C
:10C630002D4A8818FBF74EFE0021C943884201D1DC
:10C64000002525E0A100284A8818FBF743FE06468E
:10C6500031462748FCF7AAF909D3A100224A8818D5
:10C66000FBF738FE06462349FCF7A0F901D2002566
:10C670000EE0A1001C4A8818FBF72CFE064600219C
:10C68000FCF794F900D00125601CC4B2372CCEDB36
:10C6900000BF002D0BD1DC2212491348FBF7DAFD55
:10C6A000124BDC22012149020F4800F0DBFC032081
:10C6B0000A49087000BF0FE000E009E000F06EFAE0
:10C6C000012804D10C49087000200449087003E0D7
:10C6D00000200249087000BF00BF70BD1605002091
:10C6E000F025002034C90200DB3C002015050020A5
:10C6F00000007A4400007AC4170500200146002992
:10C7000006D10D48407F012800D170470020FCE78A
:10C71000012906D10848807F012800D1F5E70020D3
:10C72000F3E7022906D10448C07F012800D1ECE7D5
:10C730000020EAE70020E8E73C29002010B5C046C9
:10C74000C04610BD10B507480078002808D106483B
:10C750000078002804D111F003F9012800D110BDA0
:10C760000020FCE7DD0B0020E80B002010B511F0E5
:10C7700001F90B48C079202802DB00210848C1716B
:10C7800007488079202802DB0021054881710220BA
:10C7900008F08EFB04460349FBF7B4FD10BD000012
:10C7A000B0260020DE0B002010B512F03BFB12F08B
:10C7B000C3F811F047F910BDF1B584B08F48007887
:10C7C000002801D105B0F0BD8D48FBF783FD441C66
:10C7D0008B492046FBF796FD8948FBF77BFD044615
:10C7E0001421FBF797FC012908D186490498FBF72F
:10C7F00089FD8449091D0498FBF784FD8148FBF7F6
:10C8000069FD044621460498FCF7DAF803D27D4915
:10C810000498FBF777FD7B48001DFBF75BFD0446A2
:10C8200021460498FCF7C2F804D27649091D049801
:10C83000FBF768FD72480830FBF74CFD05462946BA
:10C840000498FBF777FD04466D490831FBF75AFD64
:10C850006B48FBF73FFD04461421FBF75BFC032903
:10C8600008D26748FBF736FD04461421FBF752FC5B
:10C87000002936D16248FBF72DFD07466048FBF7DB
:10C8800029FD0646113614213046FBF743FC4000D3
:10C890003D1A2846FBF7BFFF04465948001DFBF729
:10C8A00019FD02905748001DFBF714FD0746554837
:10C8B000FBF710FD019052480830FBF70BFD00908C
:10C8C0000199FBF788FD06463946FBF784FD0546CE
:10C8D0000299FBF72FFD21460390FBF7C1FD049061
:10C8E00022E04748FBF7F6FC07464548FBF7F2FC19
:10C8F00014210390FBF70EFC40003E1A3046FBF774
:10C900008AFF04463E480830FBF7E4FC06463C48F4
:10C91000001DFBF7DFFC07463146FBF70BFD054624
:10C920002146FBF79DFD04903548FBF7D3FC0446F8
:10C930001421FBF7EFFB002927D13148001DFBF73D
:10C94000C9FC03902F48001DFBF7C4FC02902D4842
:10C95000FBF7C0FC07462A480830FBF7BBFC39460A
:10C960000190FBF738FD06460299FBF734FD0546BA
:10C970000399FBF7DFFC04462149091DFBF7C2FCC4
:10C980001F4908310020FBF7BDFC1D48FBF7A2FC46
:10C99000E121C900884217D919490020FBF7B2FCF0
:10C9A0001749091D0020FBF7ADFC1549083100208F
:10C9B000FBF7A8FC12490C310020FBF7A3FC10493F
:10C9C00010310020FBF79EFC049802F0E5F90446C4
:10C9D0000B492839FBF796FC09482838FBF77AFC05
:10C9E000044608493439FBF78DFC05482838FBF725
:10C9F00071FC044604F0A2FF00BFE3E67D030020C3
:10CA00007C1900204019002010B500F0C7F801285B
:10CA100007D105480078002801D1012010BD002071
:10CA2000FCE70020FAE700001405002010B54C4890
:10CA30000078030018F023F90A060711213141514B
:10CA40006171868E8AE000204649087001204649BF
:10CA5000087002204249087080E013F0B3FA4148A0
:10CA60000078012808D100203E49087001203E4985
:10CA7000087003203A49087070E0FFF7A1FD3948BB
:10CA80000078012808D10020364908700120364975
:10CA9000087004203249087060E002F0ADF93148B6
:10CAA0000078012808D100202E49087001202E4965
:10CAB000087005202A49087050E014F01FFA294830
:10CAC0000078012808D10020264908700120264955
:10CAD000087006202249087040E011F0DDFE214870
:10CAE0000078012808D100201E49087001201E4945
:10CAF000087007201A49087030E011F04DFD194800
:10CB00000078012808D10020164908700120164934
:10CB1000087008201249087020E000F03FF8012852
:10CB20000FD112480078162808D016200F49087037
:10CB30000F4B012200210D4800F094FA092008490A
:10CB400008700BE000F02AF8012802D10020044907
:10CB5000087003E000200249087000BF00BF10BD4C
:10CB6000140500201705002016050020F0250020E0
:10CB70001505002010B5FFF759FF00F087F810BD2C
:10CB800010B5044609F0C6FB012805D100F006F8EF
:10CB9000002801D0012010BD0020FCE703480078E8
:10CBA000002801D1012070470020FCE7040000208C
:10CBB00003480078002801D1012070470020FCE7DD
:10CBC0000400002000B585B0072103A818F0AEFED0
:10CBD0000C21684618F0AAFE002168464173817353
:10CBE000C1730174417403AA03210120000308F0FA
:10CBF00071FE002168464173012141740021C17317
:10CC0000017403AA0821402008F064FE03AA092148
:10CC1000402008F05FFE01220821402008F0A8FE15
:10CC200001220921402008F0A3FE00220321012057
:10CC3000000308F0B5FE11481149086001220421E3
:10CC4000104812F0DFFC102011F09EF813F066FC83
:10CC500000900D48019040216846017255214172B3
:10CC60000021817269460648006809F005F8012232
:10CC700002210C2000F0B2FA05B000BD0004004013
:10CC80003800002020200040A086010010B5C548D3
:10CC90000078030017F0F3FF0906071019C4E5FD3B
:10CCA000FCFBFA007CE10320BE49087010F028F874
:10CCB000BD4812F0EDFC73E10320BA49087010F092
:10CCC0003BF8B94812F0E4FC6AE1B748FEF7D0FF40
:10CCD000002859D0B548006808F0C5FFB44800786E
:10CCE00000283FD109F01EFB01281DD1B048007873
:10CCF000401CAF49087003F08DF900220621AD48B1
:10CD000012F080FC002203210120000308F048FEFD
:10CD100000220421A84812F075FCA34812F0B8FCC8
:10CD20000720A04908707AE0A1480078401CA0497B
:10CD3000087003F06FF9002206219E4812F062FC91
:10CD4000002203210120000308F02AFE0022042112
:10CD5000994812F057FC944812F09AFC0820914927
:10CD600008705CE000209249087003F053F900223B
:10CD700003210120000308F013FE8B4812F088FC09
:10CD80000420884908704AE009F0C4FA01282FD12C
:10CD900009F0C8FA01280BD103F03CF900208449BE
:10CDA0000870864812F074FC06207E49087036E050
:10CDB00013F060FF82490968401AC8282FD903F090
:10CDC00029F900207A49087000220621794812F0DA
:10CDD00019FC002203210120000308F0E1FD0022DC
:10CDE0000421754812F00EFC00206E49087016E010
:10CDF0007448008801280FD113F03CFF724909687C
:10CE0000401A7249884207D900206E4908800521DE
:10CE10006648006808F08CFF032062490870BFE094
:10CE20006148FEF725FF002817D0FFF7CBFE01224F
:10CE30000321100308F0B4FD012206215D4812F021
:10CE4000E1FB05215948006808F072FF564812F0CE
:10CE50001FFC05205349087002E004205149087066
:10CE60009EE05148FEF704FF00283CD04F48006880
:10CE7000406908281DD104214C48006808F058FF7B
:10CE8000002206214B4812F0BDFB03E084E067E07E
:10CE90004AE02CE0002203210120000308F080FD7D
:10CEA00000220421444812F0ADFB00203D490870E7
:10CEB0001CE047480078402188434549087000221B
:10CEC00006213C4812F09EFB0022032101200003B2
:10CED00008F066FD00220421374812F093FB002081
:10CEE0003049087002E005202E49087058E03348A8
:10CEF000FEF7BEFE002813D0002206212D4812F0B6
:10CF000081FB002203210120000308F049FD0022DB
:10CF10000421294812F076FB00202249087002E023
:10CF20000620204908703BE017F01EFD1E48FEF762
:10CF30009FFE002813D0FFF745FE012203211003B6
:10CF400008F02EFD012206211A4812F05BFB012297
:10CF50000421194812F056FB0220124908701FE004
:10CF600017F002FD1048FEF783FE002813D0FFF7EC
:10CF700029FE01220321100308F012FD01220621DF
:10CF80000C4812F03FFB012204210B4812F03AFB3F
:10CF900001200449087003E000200249087000BF26
:10CFA00000BF10BD04000020C02709003800002089
:10CFB00005000020080400402020004050C300006D
:10CFC000200000202E0000201C00002088130000FC
:10CFD0003600002070470000F8B505460F4614469D
:10CFE0001E46402016490870002030702819012183
:10CFF000C903884221DC002C1DDD881184421ADC23
:10D0000010480580104807601048048010480660EA
:10D01000012204210F4812F0F5FA01220321100326
:10D0200008F0BEFC012206210B4812F0EBFA0120A9
:10D030000A490870F8BD0020FCE70020FAE700006C
:10D0400036000020340000200C00002026000020C4
:10D0500014000020202000400804004004000020AC
:10D0600070470000F8B507460D4614461E4660207E
:10D070004D4908700020307028190121C9038842E9
:10D080007EDC002C7DDD881184427ADC47480580F7
:10D09000474807602846E917890E09188911890150
:10D0A000691A444A1180104600884021081A4249F2
:10D0B00008802046E117890E09188902090C3F4AA9
:10D0C0001180E117890E091889118901611A3C4AFA
:10D0D00011803A480088002827D136480088001976
:10D0E00040281ADD01203749088033480088201A7B
:10D0F00084B22046E117890E091889112F4A118040
:10D10000E117890E091889118901611A2C4A1180C9
:10D11000294800882C49088029E0002029490880F6
:10D12000274800882849088021E0012025490880F7
:10D1300020480088002803D140202349088016E0B9
:10D140001D480088201A84B22046E117890E09186C
:10D1500089111A4A1180E117890E0918891189016C
:10D16000611A174A11801448008817490880174827
:10D17000066001220421164812F044FA012201E05F
:10D1800010E00DE00321100308F00AFC0122062143
:10D19000104812F037FA02200F4908700120F8BD3C
:10D1A0000020FCE70020FAE73600002034000020D1
:10D1B0000C000020280000202A0000202C00002065
:10D1C0003000002032000020260000201400002043
:10D1D00020200040080400400400002070B50446F0
:10D1E0000E4615462046002805DBC206D20E012158
:10D1F0009140144A116000BF3146204617F04EFDA1
:10D20000012D0ED12046002809DB00BF00BFC20659
:10D21000D20E012191400C4A116000BF00BF00BF37
:10D220000FE0204600280ADBC206D20E0121914001
:10D23000054A80321160BFF34F8FBFF36F8F00BF7D
:10D2400000BF70BD80E200E000E100E0F7B588B00B
:10D25000154600247F20C00507900C20069000BFD3
:10D2600009E0A001694A11580898FBF79FFB00D814
:10D2700005E0601CC4B20698401EA042F1DC00BF6D
:10D2800063492846FBF792FB3CD8A1015F4A891805
:10D2900048690999FBF7A7F805900999FBF7A3F8E6
:10D2A0000646A001594A801801690898FBF79BF8C7
:10D2B00003900999FBF797F8A101544A8918059042
:10D2C000C8680999FBF78FF80390A0014F4A8018AE
:10D2D00081680898FBF787F8A20101904B48101865
:10D2E00041680198FBF726F802900399FBF722F8B2
:10D2F00004900599FBF71EF807463146FBF71AF82C
:10D3000007907DE043492846FBF750FB3CD8A1013C
:10D310003E4A8918886A0999FBF765F805900999CA
:10D32000FBF761F80646A001384A8018416A089860
:10D33000FBF759F803900999FBF755F8A101334A17
:10D3400089180590086A0999FBF74DF80390A00128
:10D350002E4A8018C1690898FBF745F8A201019090
:10D360002A48101881690198FAF7E4FF029003999E
:10D37000FAF7E0FF04900599FAF7DCFF074631461B
:10D38000FAF7D8FF07903BE0A101204A8918C86B43
:10D390000999FBF728F807460999FBF724F8A20139
:10D3A00005901A481018816B0898FBF71CF8039039
:10D3B0000999FBF718F80746A20114495118486B60
:10D3C0000999FBF710F80390A001104A8018016B2F
:10D3D0000898FBF708F80190A0010C4A8018C16A70
:10D3E0000198FAF7A7FF02900399FAF7A3FF3946CD
:10D3F0000490FAF79FFF06460599FAF79BFF0790FE
:10D4000028460799FAF7EFFF0BB0F0BD440800205B
:10D41000000050410000D04110B5C046C046C04693
:10D42000C04610BD10B52E2001F072FD01280AD1B2
:10D43000092010F091FF002805D12E2001F07AFD7F
:10D44000022002F009FC10BDF0B589B004460E467A
:10D450000027002006900590049003900290019010
:10D460000A2E01DA09B0F0BD0025CEE1A90060580E
:10D470000021FBF7A5FA06D8A9006058FB49096806
:10D48000FBF794FA0CD3A90060580021FBF78EFA41
:10D490007ED2A9006058F6490968FBF791FAF7D2E5
:10D4A0000498401CC0B20490781CC7B2022F70D1FF
:10D4B000012D49D1ED49A0680968FBF781FA05D92A
:10D4C000EB49A0680968FBF771FA7DD8E749E06885
:10D4D0000968FBF775FA05D9E549E0680968FBF7C3
:10D4E00065FA0BD8E14920690968FBF769FA27D981
:10D4F000DF4920690968FBF759FA21D90021E06862
:10D50000FBF754FA0BD1D94920690968FBF758FA9F
:10D5100016D9D74920690968FBF748FA10D9D349C9
:10D52000E0680968FBF74CFA05D9D149E068096859
:10D53000FBF73CFAC9D800212069FBF737FA43D141
:10D5400005950120069063E10F2DF8D1C749E06AE7
:10D550000968FBF735FA05D9C549E06A0968FBF7A0
:10D5600025FAB2D8C149206B0968FBF729FA05D919
:10D57000BF49206B0968FBF719FA0ED8BB49606BED
:10D580000968FBF71DFA2CD9B949606B096801E0FD
:10D5900038E12CE0FBF70AFA23D90021206BFBF7D6
:10D5A00005FA0BD1B149606B0968FBF709FA18D984
:10D5B000AF49606B0968FBF7F9F912D9AB49206BE9
:10D5C0000968FBF7FDF900E0FAE005D9A849206BEE
:10D5D0000968FBF7EBF9ADD80021606BFBF7E6F9C2
:10D5E000ADD102200690681EC0B2059010E1032F55
:10D5F0007EDB0D2F7CDCF01EA84261DD691C8900FA
:10D6000060589A490968FBF7DBF907D9691C89005A
:10D61000605897490968FBF7C9F951D8A91C8900D6
:10D62000605892490968FBF7CBF907D9A91C890012
:10D6300060588F490968FBF7B9F90FD8E91C8900D0
:10D6400060588A490968FBF7BBF935D9E91C89009C
:10D65000605887490968FBF7A9F92DD9A91C8900E9
:10D6600060580021FBF7A2F90FD1E91C890060582E
:10D670007E490968FBF7A4F91ED9E91C89006058A6
:10D680007B490968FBF792F916D9A91C89006058F3
:10D6900076490968FBF794F907D9A91C89006058F5
:10D6A00073490968FBF782F90AD8E91C89006058B8
:10D6B0000021FBF77BF903D1059501200690A7E037
:10D6C000052D7DDBE91E8900605868490968FBF774
:10D6D00077F907D9E91E8900605865490968FBF7A1
:10D6E00065F96DD8291F890060586049096800E014
:10D6F0004EE0FBF765F907D9291F890060585C499E
:10D700000968FBF753F90FD8691F8900605857491A
:10D710000968FBF755F935D9691F890060585449E4
:10D720000968FBF743F92DD9291F890060580021AA
:10D73000FBF73CF90FD1691F890060584B49096814
:10D74000FBF73EF91ED9691F8900605848490968EE
:10D75000FBF72CF916D9291F89006058434909683D
:10D76000FBF72EF907D9291F89006058404909683D
:10D77000FBF71CF947D8691F890060580021FBF7A7
:10D7800015F940D102200690A81EC0B205903FE0D6
:10D790000E2F38D13549A06B0968FBF711F905D96F
:10D7A0003349A06B0968FBF701F910D82F49E06BEA
:10D7B0000968FBF705F907D92D49E06B096800E016
:10D7C00021E0FBF7F3F802D80320069020E0274978
:10D7D00020680968FBF7F4F805D92549206809682D
:10D7E000FBF7E4F80FD8214960680968FBF7E8F80F
:10D7F00005D91F4960680968FBF7D8F803D80420E9
:10D80000069005E00027681CC5B2B54200DA2DE697
:10D8100000BF0698002863D1089020E0002515E09D
:10D820006A1C9200A158AA00A058FBF7C9F80BD2B5
:10D83000A80020580390681C80002058A900605060
:10D84000691C890003986050681CC5B2701E089955
:10D85000401AA842E4DC0898401CC0B20890701E30
:10D8600008998842DADC022007900EE05C03002071
:10D87000600300200798800021580298FAF75AFDAB
:10D8800002900798401CC0B20790B01E07998842CA
:10D89000F0DC301FFAF7B4FF014600900298FAF767
:10D8A000DFFD029009F0C4FB0A2818D10498032870
:10D8B00015DB00210298FBF783F804D29449029803
:10D8C000FBF774F809D300210298FBF76FF806D232
:10D8D00090490298FBF774F8F9D20020029014E105
:10D8E000069801284DD10598401CC0B205900598B6
:10D8F000301AC6B2002509E0059828188000215882
:10D900000298FAF717FD0290681CC5B2B542F3DB26
:10D910003046FAF780FF014600900298FAF7A0FD22
:10D92000019000210198FBF74BF804D27A49019845
:10D93000FBF73CF809D300210198FBF737F819D21F
:10D9400076490198FBF73CF814D27548FAF7C2FC07
:10D95000962808D872480C30FAF7BCFC962802D8F2
:10D9600000200290D1E08321C9050298FAF778FDE2
:10D970000290CAE08321C9050298FAF771FD02906E
:10D98000C3E00698022845D1002507E0A8002158E9
:10D990000298FAF7CFFC0290681CC5B20598854240
:10D9A000F4DB0598FAF737FF014600900298FAF782
:10D9B00057FD019000210198FBF702F804D2564967
:10D9C0000198FAF7F3FF09D300210198FAF7EEFF67
:10D9D00019D252490198FAF7F3FF14D25048FAF7D6
:10D9E00079FC962808D84E480C30FAF773FC962834
:10D9F00002D80020029088E08321C9050298FAF736
:10DA00002FFD029081E08321C9050298FAF728FDD5
:10DA100002907AE0069803283AD1E16BA06BFAF7FE
:10DA200089FC0290012189070298FAF719FD0190FB
:10DA300000210198FAF7C4FF04D237490198FAF798
:10DA4000B5FF09D300210198FAF7B0FF19D2334985
:10DA50000198FAF7B5FF14D23148FAF73BFC962843
:10DA600008D82F480C30FAF735FC962802D8002049
:10DA700002904AE08321C9050298FAF7F1FC02906E
:10DA800043E08321C9050298FAF7EAFC02903CE0E2
:10DA90000698042839D161682068FAF74BFC029097
:10DAA000012189070298FAF7DBFC01900021019817
:10DAB000FAF786FF04D218490198FAF777FF09D3DD
:10DAC00000210198FAF772FF19D214490198FAF768
:10DAD00077FF14D21248FAF7FDFB962808D81048B1
:10DAE0000C30FAF7F7FB962802D8002002900CE0E1
:10DAF0008321C9050298FAF7B3FC029005E083215F
:10DB0000C9050298FAF7ACFC02900298AAE400005A
:10DB10008FC2753D8FC275BD0AD7233D0AD723BD7D
:10DB200060190020FEB504460E4600200290142E17
:10DB300000DD1426276820680190002518E0A80061
:10DB400021580198FAF73CFF02D2A8002058019012
:10DB5000A80021583846FAF729FF01D2A800275813
:10DB6000A80021580298FAF7E5FB0290681CC5B29C
:10DB7000B542E4DB39460298FAF72DFC0090019992
:10DB8000FAF729FC0290B01EFAF73AFE014600901F
:10DB90000298FAF765FCFEBDF3B597B00E4600207B
:10DBA000169014901390002515E0AA001799895833
:10DBB0002846EA0F12185210920003AB9950691CC4
:10DBC0008A0017998958EA0F1218521092000BAB6D
:10DBD0009950A81CC5B2B542E7DB00253AE0002405
:10DBE0002FE0621C920003AB9958A2009858FAF7F4
:10DBF000E7FE0DD2A00003A908581590601C800014
:10DC00000858A10003AA5050611C89001598505073
:10DC1000621C92000BAB9958A2009858FAF7D0FEFC
:10DC20000DD2A0000BA908581590601C8000085860
:10DC3000A1000BAA5050611C890015985050601C1F
:10DC4000C4B2F10F89194910491E491BA142C8DC11
:10DC5000681CC5B2F10F89194910491EA942BEDCE2
:10DC600001270FE0B80003AA11581498FAF762FBD5
:10DC70001490B8000BAA11581398FAF75BFB139095
:10DC8000781CC7B2F10F89194910491EB942E9DC65
:10DC9000301FFAF7B5FD029013991498FAF74AFB72
:10DCA00001900299FAF7DCFB1690169819B0F0BDB6
:10DCB000F3B589B000200890002500260790069053
:10DCC0000590049003900290019000274C48006852
:10DCD000002804D14B48076838460BB0F0BD00243B
:10DCE00007E0A00046490858002800D104E0601C65
:10DCF000C4B20A988442F4DB00BF0894089C012C4B
:10DD000005D13F4807683F4807603846E5E73C488B
:10DD1000006804903A4800680390002415E0A000D1
:10DD2000374909580498814203D3A0003449085860
:10DD30000490A000324909580398814203D8A000FA
:10DD40002F4908580390601CC4B208988442E6DB4F
:10DD5000002425E0A0002A4909580498401A02909E
:10DD600029490298884207D8681CC5B2A0002449F6
:10DD70000958069808180690A000214909580398E8
:10DD8000081A019020490198884207D8701CC6B231
:10DD9000A0001B490958059808180590601CC4B2DA
:10DDA00008988442D6DBB5420ED103990498401AF4
:10DDB0001549884205D829460698FAF7ABF907466F
:10DDC00015E01048076812E0B54208DD0A9506988C
:10DDD00007900A990798FAF79DF9074607E00A960F
:10DDE000059807900A990798FAF794F90746002FC3
:10DDF00002D00448076001E00248076838466CE733
:10DE0000A81F00207804002047E10000F7B59EB06D
:10DE100005461746002600201D901C901B901A9066
:10DE20001990189017901690159028210BA8FAF7C2
:10DE30002AFA282101A8FAF726FA286819902868F2
:10DE40001890012F0BD1286815904B491598086040
:10DE50001F98006849490860159821B0F0BD00245A
:10DE600011E0A00029581998814202D3A000285837
:10DE70001990A00029581898814202D8A00028586B
:10DE80001890601CC4B2BC42EBDB002430E0A00060
:10DE900029581998401A17903949179888420CD870
:10DEA000A1001F984058B1000BAA5050701CC6B278
:10DEB000A00029581B9808181B90A00029581898F2
:10DEC000081A16902E49169888420FD8A1001F985C
:10DED00041581D98800001AA11501D98401CC0B2E5
:10DEE0001D90A00029581A9808181A90601CC4B2F6
:10DEF000BC42CCDB1D98864214D10A2E0AD1314691
:10DF00001B98FAF707F9159028220BA91B48FAF776
:10DF1000A1F925E018480068159028211748FAF75C
:10DF2000B2F91DE01D9886420DDD37461B981C9006
:10DF300039461C98FAF7EEF8159028220BA90F48DD
:10DF4000FAF788F90CE01D9F1A981C9039461C9826
:10DF5000FAF7E0F81590282201A90848FAF77AF9AB
:10DF60001598002803D004491598086002E002487B
:10DF700000681590159870E77C040020A81F002009
:10DF800047E10000F0B587B004460E4600270020A8
:10DF900006902068059020680490032E2FDD002550
:10DFA00019E0A90060580599FAF70AFD02D8A800FF
:10DFB00020580590A90060580499FAF7F7FC02D898
:10DFC000A80020580490A80021583846FAF7B2F962
:10DFD0000746681CC5B2B542E3DBB01EFAF710FC79
:10DFE000039038460499FAF7F6F901900599FAF783
:10DFF000F2F902900399FAF733FA069003E0701EE3
:10E00000800020580690069807B0F0BD10B500209B
:10E01000C7494870022088700021C548C170062198
:10E020000171002141718171DD20C149C871E52173
:10E03000BF480172D6214172CA218172BD49C172A5
:10E04000090A01730020BA4948730021B848817356
:10E05000C1730121017407214174192181740020C9
:10E06000B349C8740021B248017541750121817519
:10E070000721C175992101760F2141760021817612
:10E080000020AB49C876012008770721A8484177CE
:10E09000192181770021C17730211C3001710121C4
:10E0A0004171022181710721C1711921017201465B
:10E0B0000931A148FAF726F901219D482030417223
:10E0C000002109304170142181708C21C17005211B
:10E0D00008380173002141739849801C0173090AB3
:10E0E00041730121C01E417404211130417063212C
:10E0F00081707421C1706E210171622141715121C1
:10E100000F3041714921401D41704E2181704721DE
:10E11000C17044210171412141714F2181714A2116
:10E12000C1714921017243214172482181722D211F
:10E13000C1724E210173472141734E2181734221E7
:10E14000C1730021401F4175153041708170C1704D
:10E15000017141718171153801771C3041708170F6
:10E16000C1700171417181710121001DC1700021D7
:10E17000C01C41708170C1700171332141717821DF
:10E1800081710021C01E81720421C17218210B30DF
:10E19000417000218170AA21C170002101710B38EA
:10E1A00001744174014612310020FAF7ABF860495E
:10E1B00076310020FAF7A6F85D497A310120000493
:10E1C000FAF7A0F85A497E3101200004FAF79AF8CC
:10E1D0005749823101200004FAF794F854498631F6
:10E1E00001200004FAF78EF851498A310120000419
:10E1F000FAF788F84E498E3101200004FAF782F8C8
:10E200005A214B4880308174C174002004E0002200
:10E21000474994310A54401C2028F8DB0F21444818
:10E2200080300175AA2114300172552181721121AB
:10E230004173232181737F21C17302210174322133
:10E240004174002181740521C1740175002141755B
:10E25000072181751421C175B7210C30017500218A
:10E2600041753749801C0175090A41750821801ED6
:10E270000176102141760F2181760421C176052196
:10E280001B30417001211B384177E1218901801C3D
:10E290000177090A417728211E3001700021417061
:10E2A000811C0020FAF72EF800212148C03081712E
:10E2B000C171014608310020FAF724F81C49D03119
:10E2C0000020FAF71FF81A49D4311E48FAF71AF855
:10E2D0001749D8310020FAF715F81549DC3100202C
:10E2E000FAF710F800211248D0300182418201462D
:10E2F00014311548FAF706F80D489430017C763051
:10E3000001717638417C763041717638817C763087
:10E31000C1707638C17C763081717638017D733872
:10E320000173090A41737330417D7630C17110BDAC
:10E33000F025002033160000B80B00005203000047
:10E340001A2B0000E0D14D000000404010B514F041
:10E350000BFE0B480078002804D0012803D00228C7
:10E3600007D103E009E000F017F806E000F0A4F997
:10E3700003E000200249087000BF00BF10BD00008C
:10E380002A05002003480078002801D101207047A9
:10E390000020FCE72B05002010B5BB4800780828BA
:10E3A0007CD007DC030016F06AFC0812447C7C5B1E
:10E3B0008EAAB07C162872D004DC092870D00A28F6
:10E3C0006FD1F7E017286DD01828F9D11DE101F0C1
:10E3D0000DFE01282CD1AD48C07A401CAB49C87253
:10E3E000C87A0A21F9F7ACFEC8B2A849C872E1217F
:10E3F0000901242011F0D6F8A5480088401CA44942
:10E4000008800D2000F08EFD0002000EAA2801D128
:10E410000EF058FC55219F488170232000F08AFDA2
:10E42000482000F087FD0BF0EDFF012096490870B1
:10E430001BE10CF053FA002803D004209249087025
:10E440000DE00CF041FA002809D093480DF0BCF81B
:10E450009249252011F0A6F804208B49087004E1A8
:10E460000CF03CFA00281ED001F0CCFD092806D1A2
:10E4700002208B49087006208349087022E08948F1
:10E48000027BC37A10021843014600228548C01D52
:10E490000BF0AAFE05207C49087013E04FE0A2E0D3
:10E4A00060E0DEE0A9E07C480078A52804D02520C3
:10E4B000FDF76EFB002805D1F12079490870062090
:10E4C00071490870D1E00020FEF718F9002806D045
:10E4D00001207349087006206B4908700EE06E48F1
:10E4E0000078A52804D02520FDF752FB002805D18F
:10E4F000F1206B490870062063490870B5E002F00E
:10E5000085FB072060490870AFE0674A67496448A7
:10E51000007801F093FF01F0EBFD01280ED101F02E
:10E5200001FE012803D108205749087006E0322176
:10E53000262011F037F80A205349087095E00CF0B6
:10E54000C3F901280DD1544B002257480188574880
:10E550000DF06EFE6421262011F024F809204A49AE
:10E56000087082E0232000F0D3FC012804D026208C
:10E57000FDF70EFB00280FD1232000F0DBFC02206A
:10E580004749087000214348417001200BF0BEFE4E
:10E5900007203D4908700CE03F480078A52808D1C5
:10E5A00032213C48417003203D490870072036491C
:10E5B00008705AE0482000F0ABFC002806D0482044
:10E5C00000F0B8FC3221262010F0ECFF2620FDF7E9
:10E5D000DFFA002806D101F061FD012802D11620E2
:10E5E0002949087041E00CF06FF9002804D011F0BF
:10E5F000CDF817202449087037E00CF065F90028A1
:10E6000002D01820204908702FE0FEF7C7FA012831
:10E6100026D10D2000F086FC0002000EAA280FD1A2
:10E6200000211C48763881700020214908700B4673
:10E630000122962117487438FEF714FD00F0F0FE11
:10E640000BF08CFE14F056F9FDF798FCFDF788FBF3
:10E6500000211048817000200B490870154908708E
:10E6600003E000200849087000BF00BFFFF78AFEE2
:10E67000002807D12420FDF78BFA002802D11820AA
:10E680000149087010BD00002B050020172900204B
:10E6900032050020FA26002022050020B80B0000D9
:10E6A00034050020F0250020200500201727002039
:10E6B000380500202A05002010B5FD480078030029
:10E6C00016F0DDFA190E3D5EF175A0DBF2EFEEED0E
:10E6D000F1F1ECEBEAE9E8E7E6E5E4E3E2E1F10099
:10E6E00001F084FC012829D1F248C07A401CF1498C
:10E6F000C872C87A0A21F9F723FDC8B2ED49C87279
:10E70000E1210901242010F04DFFEB480088401C56
:10E71000E94908800D2000F005FC0002000EAA283F
:10E7200001D10EF0CFFA232000F004FC482000F0C5
:10E7300001FC0BF067FE0120DD49087090E20CF04F
:10E74000CDF800280DD01BF0E9FB002805D00DF016
:10E7500013FB0220D649087011E00420D449087048
:10E760000DE00CF0B1F8002809D0D4480CF02CFFD3
:10E77000D349252010F016FF0420CD4908706FE220
:10E780000CF0A2F8012811D11BF0C8FB012803D11D
:10E790000520C749087009E0C8480CF015FFC849B2
:10E7A000252010F0FFFE0420C149087058E20CF04B
:10E7B00095F8002812D0002104201CF0C1FEC148A9
:10E7C000027BC37A1002184301460022BD48C01DD7
:10E7D0000BF00AFD0520B649087012E0B748007832
:10E7E000A52804D02520FDF7D3F9002809D101215F
:10E7F00004201CF0A5FEF120B34908700620AC49A6
:10E8000008702DE20020FDF779FF002825D01BF0CD
:10E8100085FB012805D1AC4908700620A449087081
:10E820002AE007201BF08EFB01280FD100210720D2
:10E830001CF086FE01201BF085FB044621462620A5
:10E8400010F0B0FE0A209A49087015E001209E4998
:10E8500008700620964908700EE098480078A528B0
:10E8600004D02520FDF794F9002805D1F120964920
:10E87000087006208E490870F2E102F0C7F90720FF
:10E880008B490870ECE1BBE1B2E1A7E18BE180E1EB
:10E890005EE142E12EE1F8E0F1E0D8E0B4E059E0D9
:10E8A00033E01FE000E0D7E1884A894986480078D4
:10E8B00001F0BCFE01F026FC012812D101F038FC69
:10E8C000012803D108207A4908700AE001201BF0D2
:10E8D00039FB04462146262010F064FE0A207449C4
:10E8E0000870BDE10BF0F0FF01280DD1734B002241
:10E8F0007648018876480DF09BFC6421262010F0B4
:10E9000051FE09206A490870AAE1232000F000FBAB
:10E91000012804D02620FDF73BF900280FD1232041
:10E9200000F008FB00206B4908700220664908705F
:10E9300000216948417007205D49087009E05F487F
:10E940000078A52805D103205F49087007205849A1
:10E95000087085E1482000F0DBFA00280BD0482041
:10E9600000F0E8FA01201BF0EDFA044621462620CB
:10E9700010F018FE47E02620FDF70AF9002842D1E2
:10E9800001F08CFB01283ED101F030FB01280FD1B2
:10E990004848C07A401C4749C872C87A0A21F9F72A
:10E9A000CFFBC8B24349C8720520414908702AE02C
:10E9B0001BF0B4FA012815D147487638007B802136
:10E9C000084000280AD044487638007B8007800F32
:10E9D000002803D014203649087014E00D20344973
:10E9E000087010E006201BF0ADFA012808D10420C1
:10E9F0001BF0A8FA002803D10D202D49087002E071
:10EA000016202B4908702BE101F048FB01281DD18D
:10EA10000BF05AFF002819D000202B4908702E480F
:10EA20002238827E437E10021843014601222A4882
:10EA30000D380BF0D9FB01201BF084FA0446214667
:10EA4000262010F0AFFD0E201949087008E10120C2
:10EA5000FDF754FE002806D001201B4908700F2046
:10EA6000134908700AE02620FDF792F8002805D126
:10EA7000F120154908700F200D490870F0E002F0F0
:10EA8000B9F810200A490870EAE0104A10490E4807
:10EA9000007801F053FB01F021FB012829D101F09E
:10EAA0003BFB01281AD111200149087021E0000028
:10EAB0002B05002017290020320500202205002008
:10EAC000B80B0000F02500203405002020050020B0
:10EAD0001727002035050020FA26002001201BF012
:10EAE00031FA04462146262010F05CFD13206349CC
:10EAF0000870B5E00BF0E8FE01280DD1604B012253
:10EB00006048018860480DF093FB3221262010F008
:10EB100049FD122059490870A2E0232000F0F8F9BD
:10EB2000012809D1232000F005FA02205749087076
:10EB30001020524908700AE02620FDF729F8002825
:10EB400005D103205149087010204C49087087E016
:10EB5000482000F0DDF9002803D113F0D1FE012890
:10EB60000AD1482000F0E6F901201BF0EBF9044639
:10EB70002146262010F016FD2620FDF709F8002872
:10EB800006D101F08BFA012802D116203B4908700A
:10EB900066E00BF099FE012804D10DF0D9F815209C
:10EBA000364908705CE00BF08FFE012815D11BF090
:10EBB000B5F902280ED101213548017213F09AFEF1
:10EBC000FDF7DCF9FDF7CCF800202C49087031493D
:10EBD000087002E016202949087041E00BF074FE2D
:10EBE000002804D010F0D2FD17202449087037E027
:10EBF0000BF06AFE002802D01820204908702FE090
:10EC0000FDF7CCFF012826D10D2000F08BF9000282
:10EC1000000EAA280FD100211D48763881700020EF
:10EC20001D4908700B460122962119487438FEF7D9
:10EC300019FA00F0F5FB0BF091FB13F05BFEFDF70A
:10EC40009DF9FDF78DF800211148017200200B4954
:10EC500008701049087003E000200849087000BFE0
:10EC600000BFFFF78FFB002807D12420FCF790FF9F
:10EC7000002802D118200149087010BD2B05002082
:10EC80002205002020050020172700203405002041
:10EC9000FA2600202A05002038050020F0B58BB0A8
:10ECA00005460E4600242A480A900020099020219B
:10ECB00001A8F9F7E8FA274F012D0ED0022D0CD04C
:10ECC000042D0AD0062D08D0082D06D00C2D04D016
:10ECD0000420099009980BB0F0BD1E48006A01217C
:10ECE0004902884371020122520211400843194926
:10ECF0000862002407E0A000174908586843A100F3
:10ED000001AA5050641C082CF5D300241CE01048C4
:10ED10000A9011E00A98411E0A9100280AD00F4873
:10ED20000C49C8620E48C862A00001A90858A10099
:10ED3000785001E00720CEE7A0003858A10001AAD2
:10ED400051588842E6D1641C082CE0D30998C2E7E8
:10ED5000FFFFFF000000024068C402005A5A000092
:10ED6000A5A5000010B501460020084A084BDA624C
:10ED7000084ADA621A46126A0C239A438B000C2462
:10ED800023401A43024B1A6210BD00005A5A000079
:10ED900000000240A5A5000070B504464721090601
:10EDA0002046F9F70DFE01D2002070BD8F21C90564
:10EDB0002046F9F718FB0546F9F756FDF5E7000080
:10EDC00010B5002408F050F8044609480088201ABD
:10EDD00080B208490860064804800846006805219A
:10EDE0000902884203D3032000020249086010BDD3
:10EDF000D8030020D403002070B53D4800780028D7
:10EE000006D0012805D0032862D006286AD123E065
:10EE10006CE0FDF7C3FE01281DD1364800781628A6
:10EE20000FD0482234493548F9F714FA344B4822B8
:10EE30000D2189013148FEF715F903202C4908708E
:10EE400009E02F4B48222D490D208001FEF7C4F820
:10EE500006202749087049E0FDF7A0FE012836D1B9
:10EE6000012500241EE0A100244A8818F9F732FA8F
:10EE70000021C943884201D1002515E0A1001F4AA5
:10EE80008818F9F727FA1F49884207D8A1001B4ABA
:10EE90008818F9F71FFA1C49884201D2002503E0BF
:10EEA000601CC4B2122CDEDB00BF002D0BD1482247
:10EEB00011491248F9F7CEF9114B48220D21890169
:10EEC0000E48FEF7CFF803200949087000BF0DE097
:10EED000FDF764FE012804D10C49087000200449A4
:10EEE000087003E000200249087000BF00BF70BD39
:10EEF00016050020F0250020ECC80200933C0020FD
:10EF0000150500209919010066E60000170500208C
:10EF100001465B2902DA0248405C70470020FCE7AA
:10EF20001837002001468800014A10587047000039
:10EF30004C25002001465B2904DA0020024A505487
:10EF4000012070470020FCE71837002070B5064606
:10EF5000002406F023F8C4B2E007C00F00280ED04A
:10EF6000B848007802218843801CB64908700846DA
:10EF7000C078402188434030B249C8700BE0B148A6
:10EF8000007802218843AF4908700846C0784021C4
:10EF90008843AC49C8700220204002280ED1A948FD
:10EFA0000078202188432030A64908700846C078A0
:10EFB000202188432030A349C8700BE0A148007885
:10EFC000202188439F4908700846C0782021884343
:10EFD0009C49C87004202040042807D199484078F3
:10EFE00040084000401C9749487005E0954840782B
:10EFF000400840009349487008202040082807D165
:10F000009048407804218843001D8E49487005E0EF
:10F010008C484078042188438A4948702020204049
:10F02000202807D18748407802218843801C8549E1
:10F03000487005E083484078022188438149487040
:10F040004020204040280ED17E48007840084000F3
:10F05000401C7C4908700846C07880218843803075
:10F060007849C8700BE0774800784008400075493F
:10F0700008700846C078802188437249C870802093
:10F08000204080280ED16F480078402188434030CE
:10F090006C4908700846C07804218843001D6949FE
:10F0A000C8700BE0674800784021884365490870C4
:10F0B0000846C078042188436249C870FCF7F8FD0F
:10F0C000012807D15F4840781021884310305D49FE
:10F0D000487005E05B4840781021884359494870E2
:10F0E0001020204010280ED156480078082188436F
:10F0F0000830544908700846C07810218843103001
:10F100005049C8700BE04F480078082188434D49AA
:10F1100008700846C078102188434A49C8700DF02D
:10F12000ADFE0A2807D14748407820218843203087
:10F130004449487005E043484078202188434149CC
:10F14000487040484078C02188433E49487014F0D8
:10F1500025FF0446032C03D0042C01D0052C07D135
:10F1600038484078C021884340303649487009E02B
:10F17000012C01D0022C05D132484078C0218843AF
:10F180003049487030484078002806D02D484078F3
:10F19000C0218843C0302B4948700FF075FA012810
:10F1A0000ED12848007804218843001D25490870A5
:10F1B0000846C0780821884308302249C8700BE00F
:10F1C00020480078042188431E4908700846C0780A
:10F1D000082188431B49C870FCF730FD012807D17E
:10F1E000184840780821884308301649487005E0DF
:10F1F0001448407808218843124948701148C07863
:10F2000040084000401C0F49C870084680784008FC
:10F210004000401C887009201AF094FE0949897842
:10F220000843084988700DF02FFE0546C00F4019AD
:10F23000C005000E0349087105223046F9F70AF8A7
:10F2400070BD0000440B0020192600200348007800
:10F25000002801D1012070470020FCE7540700205E
:10F2600010B50CF0C7FD11F0BFFE10BD5B2802DA2F
:10F270000121014A115470471837002070B5044627
:10F280000E460025FE20207060706820A0701020BF
:10F29000E0705E484078102809D100BF04E05C4867
:10F2A000415D281D21546D1C072DF8DB24E05948D1
:10F2B000407801280DD1002056494870002505E00E
:10F2C0005448801C415D281D21546D1C072DF7DB1F
:10F2D00009E0002505E04E480E30415D281D21540F
:10F2E0006D1C072DF7DB49484078112804D14948A7
:10F2F000417A201DFCF740F844484078492811D055
:10F3000006DC11280BD045280AD046284CD108E04D
:10F31000512808D0542807D0642845D105E000BF03
:10F3200000BF00BF00BF00BF00BF38488078E07258
:10F3300039480078001D20733448007960733348E1
:10F340004079A07331488079E0733048007A2074A6
:10F35000002505E03148415D2846113021546D1CDF
:10F360002D4800888542F5DB28484078912805D152
:10F370002648017A20461130FBF7FEFF2348027A27
:10F38000207B0B30C1B2A01C0FF04EFA2249098835
:10F3900011316054162120480088123021541E4833
:10F3A0000088133030802FE018488078E0721A48C7
:10F3B0000078C01C207315480079607313484079A9
:10F3C000A07312488079E073002505E01348415D81
:10F3D0002846103021546D1C0F4800888542F5DB0B
:10F3E000207B0B30C1B2A01C15F00AFF0A49098826
:10F3F0001031605416210848008811302154064805
:10F4000000881230308000BF00BF70BDBF400020B8
:10F4100045260020B5400020BC0B0020CC40002039
:10F420001FB51520AB490860AB48F8F753FFA94951
:10F430004860A948001DF8F74DFFA6498860A64816
:10F440000830F8F747FFA349C860A3480C30F8F725
:10F4500041FFA0490861A0481030F8F73BFF9D49E3
:10F4600048619D481430F8F735FF9A4988619A48F9
:10F470001C30F8F72FFF9749C86197487238007F12
:10F4800095497239497F0902084393497239897F46
:10F49000090408438F4908628F485638007A8E491C
:10F4A0005639C979090208438B49563989790904C3
:10F4B0000843884948628948886287481238C0787A
:10F4C00085490F3949780902084383490F398978FA
:10F4D0000904084380490F39C978090608437D4962
:10F4E000C8627D480F3800797B490F394979090294
:10F4F000084379490F398979090408437549086334
:10F5000075480E30007D744922314978090208435C
:10F51000714922318978090408436F492231C97839
:10F52000090608436B4948636B48223000796A49F1
:10F53000223149790902084367492231897909044E
:10F54000084365492231C97909060843614988633E
:10F5500061482230007A60492231497A0902084321
:10F560005D492231897A090408435B492231C97A0D
:10F57000090608435749C86357482230007B56495B
:10F580002231497B0902084353492231897B09040E
:10F59000084351492231C97B090608434D49086493
:10F5A0004D487238C07F4C495639097909020843E1
:10F5B0004949563949790904084346494864464847
:10F5C0001830F8F787FE434988646846FFF7BEFCA9
:10F5D00001990098039102906946487A897A090254
:10F5E00008433C4948653C482E30807D3A494431C7
:10F5F0004978090208433749886537482E30417DEC
:10F60000027D080210433349C86533482E30007E1E
:10F61000086631482E30407E48662F487238807820
:10F620002D497239C978090208432B497239097981
:10F6300009040843284972394979090608432549CC
:10F64000886725480E30807CC86723480E30C17C0F
:10F650002048803001602048723841781D48803051
:10F6600041601D482E30817E1A48803081601A48E2
:10F670003030417F027F08021043164980314861D3
:10F6800015484E3041780278080210431149803104
:10F6900088610AF05FFC0F498031C8610E48223052
:10F6A000017C763001717638417C76304171763854
:10F6B000817C7630C1707638C17C76308171763845
:10F6C000017D73380173090A41737330417D7630CF
:10F6D000C1711FBD4C25002062260020170027B2F3
:10F6E00000200149087070477C0B00200020014970
:10F6F00008707047BF0B0020002001490870704758
:10F70000D00B002030B589B004460D4611488178F1
:10F71000684681750F480179684601760D48417940
:10F72000684641760B48C17A6846C17709488179B5
:10F73000684681760748C1796846C17606480088E0
:10F74000064901AA31C2009105A80FC800F008F8C7
:10F7500009B030BDB73F00206E0B0020B73D002040
:10F76000FFB581B00D9F0B9E0C9C0025FE202070E4
:10F7700060706820A0701020E07000BF04E058485E
:10F78000415D281D21546D1C072DF8DB68468079EA
:10F79000E0726846C07B2073FB2E45DC301D607331
:10F7A0006846007AA0736846407AE0736846807ABB
:10F7B00020746846C07A60743246204612300A9936
:10F7C000F8F748FD6846C07BC007C00F00280FD07F
:10F7D000627B444B21460E310020F9F797FA607B9B
:10F7E000C117090F09180911491C0907090E61738E
:10F7F0000021607B0E302154022509E0607B0E3031
:10F80000205C615D4018C1B2607B0E3021546D1CDC
:10F81000607B0E30A842F1DC1621607B0F30215452
:10F82000607B1030388058E0301D81B2009168460E
:10F830000078607368464078A0736846007AE07389
:10F840006846407A20746846807A60746846C07A58
:10F85000A0743246204613300A99F8F7FBFC68463C
:10F86000C07BC007C00F002816D069460A881D4B10
:10F8700021460F310120F9F749FA69460888C11776
:10F88000090F09180911491C09050A0C009269465B
:10F89000487860730878A0730021684600880F30AC
:10F8A000215402250BE0684600880F30205C615D22
:10F8B0004018C1B2684600880F3021546D1C68465C
:10F8C00000880F30A842EEDC162168460088103010
:10F8D0002154684600881130388005B0F0BD000022
:10F8E000532600205B0B002030B589B004460D463E
:10F8F00011488178684681750F480179684601761C
:10F900000D484179684641760B48C17A6846C1770F
:10F9100009488179684681760748C1796846C17689
:10F9200006480088064901AA31C2009105A80FC8FF
:10F93000FFF716FF09B030BDCC440020C20B0020F9
:10F94000CC4200200148007870470000840200206B
:10F950001CB50721684615F0E9FF01216846417092
:10F96000C1706A460221C02005F0B4FF03220221C3
:10F97000C02005F085FF012203210846FDF72EFC7B
:10F980001CBD000010B500F00FF91348F8F7A2FCF9
:10F990001249884205D1002203210A20FDF71EFCEE
:10F9A0000AE00D48F8F796FC0D49884204D1002280
:10F9B00003210B20FDF712FC0748F8F78BFC03210D
:10F9C00001610548F8F786FC142101600021072039
:10F9D00010F0DCFD10BD00006013002000080040A6
:10F9E0000048004010B500F025F81148F8F772FC07
:10F9F00000694021884344180D48F8F76BFC046106
:10FA00000B48F8F767FC0069202188434418084830
:10FA1000F8F760FC04610648F8F75CFC0069042113
:10FA20008843041D0248F8F755FC046110BD00002E
:10FA30006013002038B580200EF0A6F900F06AF8B7
:10FA40000121072010F0A2FD2F493048F8F75AFC99
:10FA50002D48F8F73FFC00684021884304462A48B7
:10FA6000F8F738FC04602849091D0020F8F74AFC23
:10FA7000254908310420F8F745FC234910310220BC
:10FA8000F8F740FC1021684601701F481030F8F765
:10FA900021FCC1B2684641701B480830F8F71AFCD7
:10FAA000C1B26846C1701848001DF8F713FCC1B216
:10FAB000684681701448F8F70DFC044669460FF05B
:10FAC0000BFE1148F8F706FC1149884205D10122C6
:10FAD00003210A20FDF782FB0AE00B48F8F7FAFB46
:10FAE0000A49884204D1012203210B20FDF776FB4D
:10FAF0000548F8F7EFFB00684021884344180248A6
:10FB0000F8F7E8FB046038BD6013002000480040AF
:10FB1000000800401CB50721684615F007FF0021CA
:10FB2000684641706A46C02005F0D4FE02220021DA
:10FB3000C02005F01DFF01220021C02005F030FF8C
:10FB4000012118480FF0E2FD6A460121C02005F0AE
:10FB5000C1FE02220121C02005F00AFF002201217E
:10FB6000C02005F01DFF6A460421C02005F0B2FE4A
:10FB700002220421C02005F0FBFE00220421C02047
:10FB800005F00EFF01216846417001716A460321AC
:10FB9000C02005F09FFE02220321C02005F0E8FEF0
:10FBA0001CBD0000004800401CB50721684615F048
:10FBB000BDFE0020694648706A460121C02005F05C
:10FBC00089FE00220121C02005F0D2FE0022012181
:10FBD000C02005F0E5FE6A460421C02005F07AFE4B
:10FBE00000220421C02005F0C3FE00220421C02011
:10FBF00005F0D6FE6A460321C02005F06BFE002208
:10FC00000321C02005F0B4FE00220321C02005F02E
:10FC1000C7FE6A460021C02005F05CFE00221146A6
:10FC2000C02005F0A5FE01220021C02005F0B8FE8D
:10FC30001CBD00000148007870470000DA03002076
:10FC40000020014908707047DA03002001200149B3
:10FC500008707047DA03002070B505460024002DB7
:10FC600004D0012D24D0022D7DD167E000203F4932
:10FC700008703F4908703F4908603F4908603F49A4
:10FC8000F8F740FB3D49091D0020F8F73BFB002435
:10FC900008E00020A1003A4A5050A100394A5050D3
:10FCA000601CC4B2962CF4DB0120374908705BE07D
:10FCB00035480078012840D100203349087010F001
:10FCC00095FE2B480078002837D0294801782C4829
:10FCD000FEF758F927490860254801782948FEF7BA
:10FCE00051F9254908608121C90522480068F8F7C3
:10FCF00067FE12D38121C9051F480068F8F760FE2E
:10FD00000BD322491B480068F8F750FE05D31F4962
:10FD100019480068F8F74AFE04D200201549086027
:10FD200015490860154913480068F8F7EBFA1349BC
:10FD3000091D11480068F8F7E5FA15E0002012499E
:10FD400008701348F8F7C6FA06460C49F8F7DAFACD
:10FD50000F48001DF8F7BEFA06460849091DF8F7D6
:10FD6000D1FA01E0FFE700BF00BF70BD68040020CA
:10FD7000690400206C040020700400202C1900206D
:10FD8000D01A0020281D002074040020000080C02C
:10FD9000061A002070B504460025552C03D10EF03C
:10FDA0003BFB054613E0012C04D1012005F080F84F
:10FDB00005460CE0022C04D1022005F079F8054636
:10FDC00005E0032C03D1032005F072F80546284610
:10FDD00070BD000070B504460025112C12D13A48C0
:10FDE0000EF0FCFA00280BD03748007800040543D9
:10FDF000354840780002054333488078054361E088
:10FE0000324D5FE0222C12D131480EF0E7FA002883
:10FE10000BD02F480079000405432D48407900029B
:10FE200005432B48807905434CE0284D4AE0012CDE
:10FE300004D10020FFF776F8054643E0022C04D1F8
:10FE40000A20FFF76FF805463CE0042C04D10B2094
:10FE5000FFF768F8054635E0032C04D10C20FFF7C6
:10FE600061F805462EE0052C04D106200DF050FF68
:10FE7000054627E0062C04D107200DF049FF054672
:10FE800020E0072C04D108200DF042FF054619E0C0
:10FE9000082C04D109200DF03BFF054612E0092C87
:10FEA00004D10A200DF034FF05460BE00A2C04D1E2
:10FEB0002720FFF737F8054604E00B2C02D11BF092
:10FEC000A7FB0546284670BD40040020EEEEEE007C
:10FED0004704002070B50646002428480578012E06
:10FEE00027D108202840082801D1044303E0082135
:10FEF00020468843044604202840042801D10443B6
:10FF000003E00421204688430446022028400228BA
:10FF100001D1044303E002212046884304464020E7
:10FF20002840402802D10120044325E064086400F1
:10FF300022E0022E20D110202840102801D10443B5
:10FF400003E0102120468843044601200AF0AAF964
:10FF5000002802D08020044303E08021204688430B
:10FF6000044607484078002802D04020044303E0BC
:10FF70004021204688430446204670BD2B040020C3
:10FF80001926002038B504460025022C03D105F0BF
:10FF900037F8054622E0012C04D10C2005F030F89A
:10FFA00005461BE00A2C04D10A2005F029F8054675
:10FFB00014E0042C04D1042005F022F805460DE0DD
:10FFC000072C04D1072005F01BF8054606E00E2C8F
:10FFD00004D110F0BDFC0090009838BD2846FCE725
:10FFE00002461068C840C007C00F70470448807AB6
:10FFF0000349C97A884201D0012070470020FCE7FC
:020000040001F9
:10000000172900200248C07A0149085C70470000A7
:1000100017290020024800780249096808707047D3
:1000200036000020140000200148007870470000CE
:10003000F602002010B580200DF09AFE04466006FE
:10004000040E40200DF094FE04436006040E2020B0
:100050000DF08EFE04436006040E10200DF088FEA5
:1000600004436006040E08200DF082FE044360067F
:10007000040E04200DF07CFE04436006040E0220F2
:100080000DF076FE04436006040E01200DF070FEB4
:1000900004436006040E204610BD000001480078AD
:1000A00070470000590700200148007870470000A1
:1000B000C40400200148407A7047000083340020C7
:1000C00010B50446042C05DAA100034A8818F8F795
:1000D00001F910BD0020FCE7701A002003480078E9
:1000E000002801D1012070470020FCE77D0B002093
:1000F00003480078002801D1012070470020FCE768
:100100007F0B002003480078002801D101207047B0
:100110000020FCE7D40B0020014800787047000065
:100120007E0B00200148007870470000800B002003
:100130000148007870470000D50B0020F0B591B061
:1001400005460E461746012D7ED10020069006205A
:1001500004F056FF81B2B2480170090A41700920CB
:1001600004F04EFF80B2AE498870000AC87010F0EB
:10017000EFFB059000210598F8F718FC1BD2E90762
:10018000059848400590A7490598F8F72CF90446CA
:10019000F8F76AFB81B2A2480171090A4171014670
:1001A0004879097900020843E90308439C4908712A
:1001B000000A487115E09B490598F8F714F90446C0
:1001C000F8F752FB80B296490871000A48714879E5
:1001D0000979000208434104490C91480171090A58
:1001E00041718F4948790979000208438C49887127
:1001F000000AC8710A2004F003FF04468849083148
:10020000F8F780F886490C318748F8F77BF887487B
:10021000F8F760F886490390F8F7E5F80490F8F7E6
:1002200023FB04467E491031F8F76CF87F491439F6
:100230004A7C0B7C11021943084679491431F8F7BE
:1002400061F87749183100E0E2E00020F8F75AF849
:1002500009F088FE00127249087709F083FEC1B2E6
:100260006F484177090A81770CF00EFE6C49C91C72
:100270000877000A487706A80AF002FB6846008B58
:10028000404281B2664821300170090A417006A8D7
:100290000AF004FB68461821415E00290EDA008B43
:1002A0004042C1B25E482030C170C0780121C9030C
:1002B0004018C1B25A482030C17005E06846008B32
:1002C000C1B257482030C1700AA80AF079FA5449DF
:1002D00025310020F8F716F800244BE00AA8005D4D
:1002E000002846D04E482530F7F7F4FF00014C496E
:1002F00025310490F8F706F80AA8005D39280DDCCE
:1003000047482530F7F7E6FF0AA9095D3039084369
:10031000434925310490F7F7F5FF2AE00AA8005D6C
:10032000662811DC0AA8005D61280DDB3C482530F9
:10033000F7F7D0FF0AA9095D573908433849253135
:100340000490F7F7DFFF14E00AA8005D462810DCF0
:100350000AA8005D41280CDB31482530F7F7BAFFC9
:100360000AA9095D373908432D4925310490F7F76B
:10037000C9FF641C0A2CB1DB0AF076FA2849203147
:10038000487203A8FEF7E2FD0499039809910890CA
:1003900008A8017822482030817408A841782048B4
:1003A0002030C17408A881781D48203001750221D1
:1003B0004175022004F07CFD07901D490798F8F76D
:1003C00012F80490F8F750FA044615493631F7F759
:1003D00099FF13493A310020F7F794FF672108A8E5
:1003E000817531210176A12141760321C177122146
:1003F00081763421C1763E20094901AAC1C200910B
:100400000DA80FC8FFF7ACF901200A49087002E0F7
:1004100002200849087000200749087011B0F0BD9B
:10042000444000200000C84227B20000D42600202B
:10043000000020417E0B00207D0B0020F0B591B024
:1004400004460D461646012C7ED1002071490870E5
:10045000022004F02DFD0C906F490020F7F752FFA9
:100460006E490C98F7F7BFFF0490F8F7FDF90746BF
:100470006949091FF7F746FF02A812F0E9FE02A832
:1004800007C809AB07C36946888C0A21F7F758FEED
:100490006149091F08720CF0F7FC5F49091F487297
:1004A000000A88726846018D5B48001FC172090A04
:1004B00001736846408D5849091F48730FA80DF015
:1004C0008DFF10A840785449091F887310A801783F
:1004D0005148001FC17308A8817F4F48001F017455
:1004E00008A8417F4C48001F417408A8017F4A4872
:1004F000001F817403A8FEF729FD049903980E914B
:100500000D9008A8007D4449091FC87408A8417DC2
:100510004148001F017508A8817D3F48001F4175B3
:1005200002218175092019F00DFD3B49091F897DC4
:1005300008433949091F88750A20FEF7F3FC0002B9
:10054000010E3548001F00E02DE001760A20FEF77D
:10055000E9FC000E3049091FC87510F0F9F907468B
:10056000F8F782F981B22C48001F4176090A81769A
:100570009A21684681750221017610214176032176
:10058000C177562181767821C1761B202249091F27
:1005900001AA61C2009105A80FC8FFF7E1F8012088
:1005A0001F49087030E0032C10D11A480078012848
:1005B00008DA18480078401C1649087001201849CC
:1005C000087021E00220164908701DE0F12C14D1BA
:1005D0001448007D002808DD0AF080F9002804D0C6
:1005E0000021012009F092FE03E032210D488A30FB
:1005F000417002200A49087006E00021012009F03C
:1006000085FE02200649087000200749087011B0D5
:10061000F0BD0000810B002086400020000020413A
:10062000800B0020702600207F0B0020F0B589B0E1
:1006300004460D461646FB480078152877D00CDC9A
:10064000022875D004DC002810D0012871D1C9E03F
:100650000A286FD01428F9D183E11E286BD01F28F7
:100660006AD0202869D02128F0D18EE2012C21D136
:100670000020ED490870ED490870ED48C079202848
:1006800002DB0021EA48C171E948C079002803D1A2
:100690001F21E748817105E0E548C079401EC1B2DD
:1006A000E3488171012104201AF036FF0120DD4961
:1006B000087096E0022C4CD1DB480078012827D145
:1006C00010F01EF8012102201AF026FF0020D74961
:1006D0000870D7482C38C07955280ED10F20FEF766
:1006E00021FC0004000EAA2803D11E20CD49087069
:1006F00077E00A20CB49087073E00021012009F05F
:1007000005FE0220CB4908700020C649087068E049
:10071000C54800780A2811D1012102201AF0FCFEF8
:100720000020C24908700A20BE49087059E095E1CE
:1007300074E03DE2BAE0CFE1DBE1EFE1BA480078F6
:100740001E284ED10020B94908702120B5490870F3
:1007500047E0032C03D11520B249087041E0F12C89
:1007600039D1B348C079202802DB0021B048C171DB
:10077000AF48C079002803D11F21AD48817105E041
:10078000AB48C079401EC1B2A9488171FFF73AFC5D
:10079000072803D0FFF736FC012804D101210846C1
:1007A0001AF0BAFE10E0FFF72DFC002806D1012157
:1007B00008461AF0B1FE0FF08BFF05E0FFF722FCB0
:1007C000032801D10FF084FF02209A49087000200D
:1007D0009449087005E0022096490870002091496C
:1007E0000870ECE194480078002816D1FCF7D6F99F
:1007F000002812D08E4989799B225143012252034D
:10080000891888B28D4B9B228D49FCF7E5FB0120AE
:1008100085490870022083490870D0E1FCF7BEF9D1
:10082000002842D001200DF08DFD002836D08048F0
:10083000A43881798348C1767D48A438C17981483C
:100840001B3041707A48A438017A7E481B30817091
:1008500008A881787B481B30C17008A84178794886
:100860001B30017108A8017876481B3041712021A6
:10087000817108A80DF0A0FD07A804F0BBFB0020C3
:1008800005E007990A5C6E499B310A54401CC02858
:10089000F7DBFF2063306C49088002E09B206A4947
:1008A000088014205F49087000BF88E1674800781D
:1008B000002855D1FCF772F9002851D000205F497B
:1008C0000870FF215A488171C7790CE05848801C94
:1008D000F7F700FD0121B9400840002802D0544834
:1008E000877102E07F1E002FF0DA00BF5048807948
:1008F000FF2814D11F270CE04D48801CF7F7EAFCB5
:100900000121B9400840002802D04948877105E01C
:100910007F1E4748C079401EB842EDDB00BF444807
:100920008079FF2806D102204249087000203D4905
:10093000087015E03E4989799B22514301225203F8
:10094000891888B23D4B9B223D49FCF745FB9B2013
:100950003D4908800A203449087014203149087044
:100960002DE1FCF71BF900285BD00F20FEF7DAFA27
:10097000C0B2AA282AD19A2035498870022008716D
:10098000102048710320C87232480088401C314949
:100990000880084600782E4988712E480088001289
:1009A000C8711B202849088012F088FE264800885C
:1009B00029490D2201AB61C30091254905A8F7F72C
:1009C00049FC05A80FC8FEF7CBFE24E067202049AC
:1009D000887043200871A12048710320C8721D4807
:1009E0000088401C1B490880084600781849887117
:1009F000184800880012C8711348008810490D2259
:100A000001AB61C30091124905A8F7F723FC05A8C3
:100A10000FC8FEF7A5FE0120064908700020014915
:100A20000870CCE0D40B0020D90B0020D80B00209C
:100A3000B0260020D50B0020DD0B0020C00B0020CD
:100A4000F544002035460020D60B0020E80B00209E
:100A5000D9440020D20B0020B94700205948007823
:100A6000012810DA57480078401C5649087056484B
:100A700000781E2803D12020544908702BE0142050
:100A80005249087027E05048007801281DD1FFF72F
:100A9000B9FA072803D0FFF7B5FA012804D10121DC
:100AA00008461AF039FD10E0FFF7ACFA002806D12D
:100AB000012108461AF030FD0FF00AFE05E0FFF7AD
:100AC000A1FA032801D10FF003FE0220404908706B
:100AD00000203E49087072E0FCF760F8002807D05B
:100AE0001E20394908700EF061FE1F20374908703A
:100AF00065E00EF0CDFF0FF0C3F801280DD13548A9
:100B00000078002803D020203049087005E002203A
:100B10002F49087000202D49087050E0FCF73EF87E
:100B2000002831D09B202C498870012008711020AA
:100B300048710320C87229480088401C2749088052
:100B40000846007824498871244800880012C8713A
:100B5000204800780C214843401C21490880084661
:100B6000008820490D2201AB61C300911A4905A8F4
:100B7000F7F770FB05A80FC8FEF7F2FD0120144936
:100B8000087000201149087019E0FCF707F80028E8
:100B90000DD0154915480068F7F7B4FB144B062231
:100BA000C2211148FCF75EFA1E200849087006E0D1
:100BB00002200749087000200449087000BF00BFE8
:100BC00009B0F0BDD80B0020D90B0020D40B0020B9
:100BD000D50B0020DC0B0020D9440020D20B0020D4
:100BE000D60B0020D4470020B2260020EC0B0020BA
:100BF000C00B002001200349087000200249087042
:100C0000704700007D0B00207E0B00200020024971
:100C10000870024908707047D40B0020D50B0020E3
:100C2000014800687047000064070020FEB50024FA
:100C30000026FE480078002802D001287ED10BE073
:100C400000F010FEFA49086008460068042802D047
:100C50000120F6490870C6E2F5480078C007C00FC9
:100C600000286CD00020F349087100F015FE002028
:100C7000F14908700B2019F0BDF902A800F018FE28
:100C800001A804F0DFF8684604F0F8F8002432E226
:100C9000A00002990858A100E84A5050A00001990C
:100CA0000858A100E64A5050A000009A115820466A
:100CB00010F01AF8A000E149085C0006A100DF4A24
:100CC0005158FF221202114009020843A100DB4AD9
:100CD0005158FF2212041140090A0843A100D74AC3
:100CE0005158090E0843A1005050FAF7A7FF0128F8
:100CF00008D1D448F7F7EEFAA100D04A515840186D
:100D0000A1005050A000CE49085801210906084012
:100D100088427DD1A000C9490858C00FC0070121F1
:100D2000C907884215D1A000C449085840004008AE
:100D3000A100C24A5050A000114601E052E204E274
:100D40000858C043401CA10050500A2019F052F925
:100D500002E0172019F04EF9A000B8490858002801
:100D600004D0A0000858B84988420CD9A000B34963
:100D700008580121C907884209D3A000AF49085883
:100D8000B249884203D84D2019F034F936E0A0006A
:100D9000AA490858AD49884209D9A000A74908586E
:100DA000AB49884203D8072019F024F926E0A000B7
:100DB000A2490858A649884211D9A0009F4908585D
:100DC000A44988420BD8A0009C490858400040081C
:100DD00001218904081AA100984A50500EE0002C05
:100DE00005D19648C06BA100944A505006E0601EA1
:100DF000800092490858A100904A5050A1008F4AA3
:100E000050580EF0DFFC212019F0F4F8162000E015
:100E100010E019F0EFF8582019F0ECF8002085499F
:100E2000487088700870C87000F028FD012000F03C
:100E300025FDF7E0A000824908580121C9060840B5
:100E4000884238D17B484078102804DB0020A1007C
:100E50007A4A505013E077484078401C75494870F2
:100E6000002C05D17548C06BA100744A505006E0B3
:100E7000601E800071490858A100704A5050A100BE
:100E80006E4A50580EF09EFC022019F0B3F817205D
:100E900019F0B0F84D2019F0ADF800206549087040
:100EA000C870212019F0A6F8002000F0E7FC01200E
:100EB00000F0E4FCB6E0A0006149085801214906B1
:100EC000084088423AD15B488078102804DB002033
:100ED000A1005A4A505013E056488078401C5549AA
:100EE0008870002C05D15548C06BA100534A505062
:100EF00006E0601E800051490858A1004F4A50503A
:100F0000A1004E4A50580EF05DFC082019F072F80E
:100F1000212019F06FF8022019F06CF8172019F051
:100F200069F84D2019F066F8002042490870C87031
:100F300000F0A4FC012000F0A1FC73E0A0004049F7
:100F4000085801218906084088421DD13948007897
:100F5000401C384908700846007803280EDC002C35
:100F600005D13648C06BA100344A505006E0601EDF
:100F7000800032490858A100304A5050A1002F4A41
:100F800050580EF01FFC4DE0A0002D4908580121DB
:100F900049070840884204D0A00029490858002881
:100FA00029D1032019F026F82248C078401C214995
:100FB000C870002C05D12148C06BA1001F4A5050B9
:100FC00006E0601E80001D490858A1001B4A5050D1
:100FD0001848C078102808DB00201649C870FDF7B3
:100FE000D1F9012801D100F069FCA100134A505841
:100FF0000EF0E8FB16E0212018F0FCFF002C05D1D4
:101000000E48C06BA1000D4A505006E0601E8000E3
:101010000A490858A100094A5050A100074A5058EF
:101020000EF0D0FBA0000649085815E03903002057
:101030003003002071030020CA0300205017002055
:1010400090170020161A0020333303000701008098
:10105000CCCC0080000004800121090708408842B0
:1010600044D1092018F0C6FF701CC6B2102E09D159
:10107000002405E00120A1005C4A5050601CC4B26D
:10108000102CF7DB002C15D15848C06B0121C90783
:1010900088420AD85548C06B5549884205D3534801
:1010A000C06BA100514A505023E00120A1004F4ADB
:1010B00050501EE0601E80004C4908580121C907AD
:1010C00088420ED8601E8000484908584849884226
:1010D00007D3601E800045490858A100434A50507C
:1010E00007E00120A100414A505002E0632018F0BF
:1010F00081FF601CC4B2102C00DAC9E504F046FB85
:101100000220FEF7DDFF07463A49F7F7FBF8032018
:10111000FEF7D6FF074637490C31F7F7F3F8FEF72D
:1011200095FD3448F7F7D6F807463349F7F7EAF85C
:1011300030480C30F7F7CEF807462F490C31F7F757
:10114000E1F800202D4908704BE02D48006802218D
:101150000840022845D12B480079401C29490871D4
:1011600000F09AFB00F078FB054626480079052838
:101170000BDB05202349087140211C48F7F783F851
:1011800040212148F7F77FF819E0002410E0002CF7
:1011900005D11648C06BA100144A505006E0601EED
:1011A000800012490858A100104A5050601CC4B277
:1011B000102CECDBA1000D4A50580EF003FBE807A1
:1011C000C00F002803D0012018F014FF06E0022011
:1011D0002840022802D1012018F00CFF0020074906
:1011E000087000E000BF00BFFEBD000050170020E7
:1011F00066660000601900201819002039030020DD
:1012000030030020710300209017002010B53448EF
:101210000078002802D001285FD14CE00120FDF7C2
:1012200077FE012846D1FDF785FE002405E0002069
:10123000A1002C4A5050601CC4B2102CF7DB2A4A83
:1012400000200146F7F767F828490020F7F75AF819
:101250002649091D0020F7F755F825490020F7F722
:1012600051F82349091D0020F7F74CF821490020C7
:10127000F7F748F800202049086020490860204915
:1012800008602049086000F043F8FBF787FC00285D
:101290000DD01D4B1622FF2101311C48FBF7E2FE49
:1012A00000200F490870FF2018F0A4FE02E0012082
:1012B0000B49087012E0FBF771FC00280CD0124BB0
:1012C0001622FF2101311148FBF7CCFE0020044912
:1012D0000870FF2018F08EFE00E000BF00BF10BDB8
:1012E000B1030020501700209D03002004190020A6
:1012F0004C1900207E030020007F0020047F002086
:10130000087F00200C7F0020F8030020F81900203F
:1013100010B577201D490870882048701C480DF0D2
:101320005DF81B48007819498870194841781748BA
:10133000C170174881781548017115480179134823
:1013400041711448F6F7C6FF04461049891DF6F7A7
:10135000D9FF1048001DF6F7BDFF04460B490A31BE
:10136000F6F7D0FF0B482830F6F7B4FF04460749DC
:101370000E31F6F7C7FF07482C30F6F7ABFF0446EF
:1013800002491231F6F7BEFF10BD0000F819002027
:10139000DB03002004190020F8B5B24800780300F0
:1013A00013F06DFC090627F9F3F2F1F0EFEEF2000D
:1013B000FBF7F4FB00281BD000240DE0A000AA4A94
:1013C00081180020F6F79EFFA000A84A811800208F
:1013D000F6F798FF601CC4B2122CEFDBA44B162268
:1013E000A449FF200130FBF7F7FD01209D4908705B
:1013F00035E19F480078FBF7C3FB01287ED1FBF75E
:10140000CDFB0128FAD19B480078772877D19948FD
:1014100040788828FAD1984800689849884229D1AC
:10142000042197480CF0CAFB012806D19148801D81
:10143000F6F750FF9249086005E08E49891D9048F3
:101440000068F6F75FFF04218E480CF0B7FB012817
:1014500006D188480A30F6F73DFF8A49086005E062
:1014600084490A3187480068F6F74CFF05207D491A
:10147000087002E007207B4908707E480E30F6F7BE
:1014800029FF05468121C905F7F79AFA1BD3794848
:101490001230F6F71FFF05468121C905F7F790FACC
:1014A00011D374480E30F6F715FF05467649F7F765
:1014B0007DFA08D36F481230F6F70CFF05467249E3
:1014C000F7F774FA0CD26B490E310020F6F71AFFC9
:1014D000684912310020F6F715FF052061490870B0
:1014E0006448801DF6F7F6FE05465F49091DF6F7CC
:1014F00009FF60480A30F6F7EDFE01E04AE02AE015
:10150000054659490831F6F7FDFE5A48801DF6F7A1
:10151000E1FE05465D49F6F7F5FE56480E30F6F752
:10152000D9FE054650492C31F6F7ECFE51481230F1
:10153000F6F7D0FE05464C493031F6F7E3FE4A484F
:10154000001DF6F7C7FE0746F7F7D8F90546504ADB
:10155000F6F7E1FE1EE04D490020F6F7D3FEFBF75B
:101560001DFB002813D0FFF7D3FE414B1622FF21AD
:1015700001314048FBF776FD03203A49087009E045
:1015800056E040E036E025E068E015E003E00220A8
:101590003449087063E0FBF701FB00280BD0FFF72C
:1015A000B7FE334B1622FF2101313248FBF75AFDBB
:1015B00003202C49087052E02D480078FBF7E0FA30
:1015C000012806D1FBF7EAFA012802D107202549B4
:1015D000087044E0FBF7E2FA00280AD0244B1022FE
:1015E000FF2107312348801DFBF73CFD03201D49E7
:1015F000087034E01520FDF795FC264908600120AD
:10160000254908702BE01A480078FBF7B9FA012841
:101610000DD1FBF7C3FA012809D1154B0C221F4944
:10162000FF205130FBF7D8FC08200E49087016E067
:101630000F480078FBF7A4FA01280ED1FBF7AEFAA9
:1016400001280AD1FAF7FAFA002803D11349083120
:10165000F6F758FE06200349087000E000BF00BFFF
:10166000F8BD0000C5030020001900204819002023
:10167000E2030020F8190020147F00206D5C4B3A33
:10168000007F0020047F0020000080C03503002080
:101690009D03002090030020C60300200E1A0020A6
:1016A00070B559480078002804D001280BD00628CE
:1016B00072D182E0E121090103200DF01BF8012025
:1016C000514908709DE003200CF046FE002819D017
:1016D0000BF08EFC012815D00320FDF719FC012822
:1016E00010D04A48007800280CD1FAF7A1FA012856
:1016F00008D012F014FF012804D000200FF060F988
:10170000012859D1FBF74AFA002855D000200FF0E4
:1017100061F903200CF020FE00282ED13C48F6F79A
:10172000D9FD05463B48F6F7D5FD06462946F6F7AE
:1017300052FE04467F21C9052046F7F741F904D33C
:1017400035492046F7F732F913D23248F6F7C2FD91
:1017500005462F49F6F7D6FDFFF7DAFD2F4B162287
:10176000FF2101312E48FBF77DFC06202649087039
:1017700022E00020244908701EE0FAF759FA0128F7
:101780000BD1002027490870274B0422FF21593133
:101790002648FBF767FC0FE032E000201B49087089
:1017A000FFF7B6FD1D4B1622FF2101311C48FBF748
:1017B00059FC06201449087023E0FBF7EFF90028D4
:1017C0001DD0FF2018F016FC0320FDF7A1FB012817
:1017D00005D10320FDF7AEFB0120154908700BF081
:1017E00007FC012803D012F09AFE012804D1012041
:1017F00008F0C8FB13F08EFA00200349087000E0DF
:1018000000BF00BF70BD0000C4030020B003002073
:101810006C03002004190020000080BFF9030020A1
:10182000F8190020C80300209C030020161A00208D
:10183000C703002010B5074800780A2807DA0548D2
:101840000078401C0349087000F038F801E003F00C
:10185000A3FE10BDCA0300200148007870470000B5
:101860008A020020014800787047000089020020A9
:1018700001480078704700008C020020072800DD36
:10188000704701218140034A12788A4301490A7056
:1018900000BFF5E78A020020042001490870704764
:1018A0008902002000200149087070478C02002046
:1018B00001490160704700009413002010B5FEF745
:1018C00047F8FEF7B7F800200F4908600F49086095
:1018D0000F4908700F4908700F4908700F490870C8
:1018E0000F4908700F4908700F4908700F490870B8
:1018F0000F4908600F4908600F4908600FF0BAF9F6
:101900000B49086010BD00007C020020800200200E
:101910008402002085020020860200208702002029
:10192000880200208D0200208B0200208C02002003
:10193000980200209002002094020020F8B504468E
:10194000002C0AD005200004844202D317488442A8
:1019500003D9062018F04EFB02E0422018F04AFBA3
:10196000002C07D003200004844203D2042018F086
:1019700041FB02E02C2018F03DFB0EF0E9FF07468A
:101980000B493846F7F71CF808D33846F6F7B6FF88
:1019900005460022074BF6F7C5FF03D2052018F0D5
:1019A00029FB02E0372018F025FBF8BD0000730C7E
:1019B00000005C420000E0BFF0B589B000250027C0
:1019C00000261720FDF7AEFAFE49086008460068B9
:1019D00003F089FBFC490860084601680020F6F71F
:1019E000FAFCFA49086000242DE0A000F8490858E4
:1019F0000121C90788421CD3A000F54908584000BE
:101A00004008A100F24A5050A100505803F06BFB6F
:101A100000210790F6F7E3FCA100EE4A5050A00029
:101A2000EB4908580121C9070843A100E84A505072
:101A300007E0A100E64A505803F055FBA100E54A33
:101A40005050601CC4B2102CCFDB05F0F1FA0A280C
:101A500073D10020E04908701021DE48FBF7F4FC48
:101A60000646DE48066000213046F6F79FFF08D2A2
:101A70000A20DB49087031460020F6F7ACFC064628
:101A800002E00120D64908703046FDF785F908903C
:101A9000089800F0B3FA07463846FDF77DF9D149BA
:101AA0000690F6F72FFCCF48F6F714FCCE490690C7
:101AB000F6F728FCCB48F6F70DFC0690FFF73EFF43
:101AC000CA48407901280BD1C9480078401CC84950
:101AD000087008460078F02805DB0020087002E056
:101AE0000020C3490870C048F6F7F4FB002805D071
:101AF000162018F07FFA582018F07CFA384608F0C3
:101B000075FA0746384601F047FD39460020F6F7DA
:101B10004DFF7DD0B748007800280FD1B648006847
:101B2000F6F779FE432109060590F6F799FC394648
:101B30000690F6F758FC054612E08EE1AF493846AC
:101B4000F6F751FC0746AC480068F6F764FE3946E4
:101B50000590F6F748FCAA490690F6F781FC054681
:101B6000A8492846F6F73FFCA7490690F6F778FC07
:101B70000546A6492846F6F773FC054698480078BE
:101B8000012813D1A248F6F7AFFB03910290284633
:101B9000F6F7B4FE01910090039B029AF6F79EFCC3
:101BA0009B4A05910490F6F7B6FBE0E01620FDF79E
:101BB000B9F9984988423BD19548F6F795FB0591CC
:101BC00004902846F6F79AFE03910290059B049A2A
:101BD000F6F7BCFE05D88E4A00200146F6F79BFBBF
:101BE00012E08B48F6F780FB039102902846F6F747
:101BF00085FE01910090039B029AF6F719FD844A35
:101C000005910490F6F787FB8148F6F76DFB00E03D
:101C1000A7E005910490F6F7ADFE734908390690E8
:101C2000F6F770FB70480838F6F754FB7A490860FD
:101C30006D48001FF6F74EFB78490690F6F7C0FE98
:101C400021D2294676480068F6F774FB744908608B
:101C50006C4973480068F6F7B3FE7BD26949704857
:101C60000068F6F7B8FB6E4908605F48001FF6F79A
:101C700031FB64490590F6F75DFB5B49091F06904F
:101C8000F6F740FB66E05848001FF6F723FB65496E
:101C90000690F6F795FE21D2294661480068F6F7CE
:101CA00049FB5F49086060495D480068F6F788FEB7
:101CB00050D25D495A480068F6F78DFB58490860D4
:101CC0004948001FF6F706FB57490590F6F732FB27
:101CD0004549091F0690F6F715FB3BE04248001FF7
:101CE000F6F7F8FA4649A0390690F6F769FE24D2CD
:101CF00029464B480068F6F71DFB494908607F21DB
:101D0000C90547480068F6F75BFE23D27F21C90565
:101D100043480068F6F75FFB414908603248001FFE
:101D2000F6F7D8FA7F21C9050590F6F703FB2E498F
:101D3000091F0690F6F7E6FA0CE02B48001FF6F7AD
:101D4000C9FA29460590F6F7F5FA2749091F0690C2
:101D5000F6F7D8FA2448001FF6F7BCFA33490860B2
:101D600005E02148001FF6F7B5FA304908603A4609
:101D70001B480178284612F029FE079001218907A7
:101D80000798F6F71DFE05D3032189070798F6F794
:101D90000DFE01D2002007901D48F6F7A5FA039129
:101DA00002900798F6F7AAFD01910090039B029A12
:101DB000F6F794FB164A05910490F6F7ACFA14482E
:101DC00036E00000580300205C0300206003002080
:101DD00050170020B819002070030020B403002021
:101DE000A5030020541900200C190020A41900207C
:101DF000CB030020C0030020D4030020643B7F3FBE
:101E0000002474490000C8420000614500007A4483
:101E10009D0300203C4D0000007F0020A3BBBE4C72
:101E2000A80300207696184B00002041047F002074
:101E3000F6F75AFA05910490F6F79CFD5C49069076
:101E4000F6F760FA5A48F6F745FA5A4908605A48D0
:101E500005605A485A490860A7E05A4800780128A6
:101E600004D100205749087019F08EFB1021564804
:101E7000FBF7EAFA06465548066000213046F6F7B9
:101E800095FD00D200263046FCF786FF08900898A2
:101E900000F0B4F807463846FCF77EFF4C4908606E
:101EA0004C48407901280BD14B480078401C4A49E6
:101EB0000870084600780F2805DB0020087002E053
:101EC000002045490870384608F090F80746384623
:101ED000FAF772FC384601F05FFB39460020F6F74E
:101EE00065FD51D0162018F085F8582018F082F8BA
:101EF0003A480068F6F78FFC432109060590F6F78B
:101F0000AFFA39460690F6F76EFA35490790F6F7BC
:101F1000A7FA05463348F6F7DDF929460690F6F7A5
:101F200009FA30490790F6F7EDF92F48F6F7DCF992
:101F3000059104902D492846F6F792FA0190F6F79C
:101F4000DDFC03910290059B049AF6F7C7FA264A36
:101F500007910690F6F7DFF92348F6F7C5F90591E2
:101F60000490F6F707FD12490790F6F7CBF91D48E4
:101F7000F6F7B0F91E4908601E4805600C48F6F7F0
:101F8000A9F90C4908600DE00948F6F7A3F90949D9
:101F900008600748001DF6F79DF917490860002002
:101FA0001449086005480649086009B0F0BD000002
:101FB00004190020007F0020187F00206D5C4B3A40
:101FC000147F002045030020B8190020B40300202E
:101FD0003C030020A4190020CB030020D4030020E0
:101FE000000010424C1900209D03002000007A449C
:101FF000087F00200C7F0020047F002001B59CB0EA
:1020000000201B901A9019901C9812F06FFB05206D
:102010000CF098F9002811D005200CF0C3F9FD4808
:102020000068FD49884203D90120FC49087002E09C
:102030000020FA4908700020F6490860F8491C9809
:102040000968884204D3012189041C98884202D37C
:1020500000201B90F5E3EF480068401CED49086044
:102060001C9803F040F81A90EE491A98F6F7BBF95D
:102070001A90F9F7E3FD01281AD1EB480068401CDB
:10208000E949086004200CF05DF9002813D0042011
:102090000CF088F9E4480068DF49884204D903F06D
:1020A0002DF80120E14908700020DF49086002E0B6
:1020B0000020DD490860DE480078002803D0DD48B4
:1020C0000068199002E00EF043FC19901998F6F799
:1020D00015FC0022D84B17911690F6F723FC0CD272
:1020E000D648F6F7F7F85F2807D9D4480C30F6F74A
:1020F000F1F85F2801D9D24819900BF001FED149BF
:102100000860D1481A99F6F76EF915901A99F6F702
:102110006AF91790CD481999F6F765F913901A994D
:10212000F6F761F91590CA481999F6F75CF911901C
:102130001999F6F758F91390C6481A99F6F753F912
:102140001190C5481999F6F74EF9C4490F90F6F762
:10215000F1F810901199F6F7EDF812901399F6F73F
:102160003AF914901599F6F7E5F816901799F6F7DD
:10217000E1F81890BA491898F6F718FC7ED80021B3
:102180001998F6F713FC04D3B6491998F6F718FC1A
:1021900003D2B548006D179028E01998F6F764FB54
:1021A000C0B215901598F6F736FB0D901999F6F711
:1021B00016F9149015988000AB4908580B901598A3
:1021C000401C800008580A900B99F6F704F90C900F
:1021D0001499F6F708F90D9015988000A24908584F
:1021E00001460C900D98F6F7A5F817901799084638
:1021F000F6F7F9F80C901A99F6F7F5F89B490D9057
:10220000F6F7F1F813901998129000211998F6F743
:10221000CDFB02D20020129006E095491998F6F7FE
:10222000CFFB01D29248129092481299F6F7DBF850
:102230000C9091481299F6F7D6F808901299F6F793
:10224000D2F80A908D481299F6F7CDF807901299B6
:10225000F6F7C9F808901299F6F7C5F809900A99A7
:10226000F6F768F80B900C99F6F7B5F884490D90DD
:10227000F6F760F811908348129900E0EAE1F6F76A
:10228000B2F80B9080481299F6F7ADF809901299C0
:10229000F6F7A9F80A900B99F6F74CF87B490C90E1
:1022A000F6F748F87A490D90F6F79DF810907848BF
:1022B0001099F6F798F80B901399F6F794F875497A
:1022C0000C90F6F790F80D901199F6F7C9F80F9069
:1022D00071491398F6F787F81B906D490F98F6F738
:1022E000BFF80E906D490E98F6F760FB55D26C481A
:1022F0000E99F6F778F80C906A480E99F6F773F88D
:1023000008900E99F6F76FF80A9067480E99F6F75D
:102310006AF805900E99F6F766F806900E99F6F7AA
:1023200062F8089061480E99F6F75DF802900E99F0
:10233000F6F759F803900E99F6F755F804900E99B0
:10234000F6F751F806905A480E99F6F74CF80190B6
:102350000E99F6F748F802900E99F6F744F80390B4
:102360000E99F6F740F804900E99F6F73CF80590B0
:102370000699F6F730F807900899F5F7DBFF099012
:102380000A99F6F728F80B900C99F5F7D3FF49490D
:102390000D90F5F7CFFF169051E147490E98F6F7EB
:1023A00005FB36D245480E99F6F71DF80C904448C7
:1023B0000E99F6F718F808900E99F6F714F80A90A7
:1023C00040480E99F6F70FF805900E99F6F70BF8BE
:1023D00006900E99F6F707F808903B480E99F6F725
:1023E00002F802900E99F5F7FEFF03900E99F5F7AB
:1023F000FAFF04900E99F5F7F6FF069033480E9910
:10240000F5F7F1FF01900E99F5F7EDFF02900E99A7
:102410005EE07DE0F0030020B8A10000C9030020C9
:102420005803002000007A43EC030020C80300207A
:1024300052030020540300200000E0BF18190020C0
:102440000000A041CC0300209F71E13C8D7F1F3D27
:10245000B43B243B0456BA40849E0D3EB29D3FC01F
:10246000000096420000C842C0C602005F2A0F3238
:1024700000005C4223DB5C421A516A3FA69BC4BB4E
:102480006606DF443B4A5B372684B3B64703803F8A
:1024900000007A4433333B412D86C143CDCCAC4060
:1024A0004B75013D61E28F3C1A53B03B3EF4553A07
:1024B000E93A4938C009653F00004842643B043BA3
:1024C0005762D838451E4D3632CE46330689982F8E
:1024D000F5F789FF03900E99F5F785FF04900E99A3
:1024E000F5F781FF05900699F5F775FF07900899B4
:1024F000F5F720FF09900A99F5F76DFF0B900C99FD
:10250000F5F718FFFE490D90F5F714FF169096E0C9
:10251000FC490E98F6F74AFA55D2FB480E99F5F7A2
:1025200062FF0C90F9480E99F5F75DFF08900E993F
:10253000F5F759FF0A90F6480E99F5F754FF059004
:102540000E99F5F750FF06900E99F5F74CFF08909D
:10255000F0480E99F5F747FF02900E99F5F743FF03
:1025600003900E99F5F73FFF04900E99F5F73BFFA6
:102570000690E9480E99F5F736FF01900E99F5F7A8
:1025800032FF02900E99F5F72EFF03900E99F5F7A2
:102590002AFF04900E99F5F726FF05900699F5F7A6
:1025A0001AFF07900899F5F7C5FE09900A99F5F703
:1025B00012FF0B900C99F5F7BDFED8490D90F5F779
:1025C000B9FE16903BE0D6480E99F5F70CFF0C903B
:1025D000D4480E99F5F707FF08900E99F5F703FF19
:1025E0000A90D1480E99F5F7FEFE05900E99F5F781
:1025F000FAFE06900E99F5F7F6FE0890CB480E9974
:10260000F5F7F1FE04900E99F5F7EDFE05900E99A1
:10261000F5F7E9FE06900E99F5F7E5FE07900899A3
:10262000F5F788FE09900A99F5F7D5FE0B900C99FD
:10263000F5F780FEBE490D90F5F77CFE16901699D1
:102640001B98F5F7D0FE1B9019A807C8FAF7FEFDF6
:102650001B90EEE3B7491998F6F7B2F97ED2B64966
:102660001898F6F7A3F97AD2B44800680146139097
:102670001A98F5F75FFE1590B04800680146119072
:102680001A98F5F757FE1390AC4800680146109071
:102690001A98F5F74FFE1190A848806A01461090ED
:1026A0001198F5F7A0FE12901399F5F79CFE14907F
:1026B0001599F5F798FE1790A0480068014610900C
:1026C0001A98F5F737FE12909C48006801460F9063
:1026D0001A98F5F72FFE10909848406A01460F901F
:1026E0001098F5F780FE11901299F5F77CFE139083
:1026F0001999F5F778FE15909048006801460E90FC
:102700001A98F5F717FE0F908C48006A01460E9054
:102710000F98F5F768FE10901999F5F764FE11907F
:102720001999F5F760FE13908448C0690D901999C6
:10273000F5F759FE0E901999F5F755FE0F90199976
:10274000F5F751FE11907D48006801460B901A98EC
:10275000F5F7F0FD0D907948006801E07DE171E04A
:1027600001460A901A98F5F7E5FD0B9073488069C9
:1027700001460A900B98F5F736FE0C900D99F5F787
:1027800032FE0F906D480068014609901A98F5F7DF
:10279000D1FD0A9069484069014609900A98F5F709
:1027A00022FE0B901999F5F71EFE0D906348006903
:1027B00008901999F5F717FE09901999F5F713FE86
:1027C0000B905E480068014606901A98F5F7B2FD36
:1027D00007905A48C068014606900798F5F703FE2F
:1027E00009905648806806901999F5F7FCFD079006
:1027F00052484068014606900798F5F79BFD0890FF
:102800000999F5F797FD0A900B99F5F793FD0C9050
:102810000D99F5F78FFD0E900F99F5F78BFD109040
:102820001199F5F787FD12901399F5F783FD149030
:102830001599F5F77FFD16901799F5F77BFD1B901D
:10284000F7E2F6E33D48C06A014613901A98F5F79F
:1028500071FD15903948C06A014611901A98F5F734
:1028600069FD13903548C06A014610901A98F5F733
:1028700061FD11903148406D014610901198F5F7B7
:10288000B2FD12901399F5F7AEFD14901599F5F776
:10289000AAFD17902948C06A014610901A98F5F7CA
:1028A00049FD12902548C06A01460F901A98F5F725
:1028B00041FD10902148006D01460F901098F5F7EA
:1028C00092FD11901299F5F78EFD13901999F5F775
:1028D0008AFD15901948C06A01460E901A98F5F7BE
:1028E00029FD0F901548C06C01460E900F98F5F722
:1028F0007AFD10901999F5F776FD119019991FE05E
:1029000070256B3F0000C843CB694B39C66FA735B4
:102910000D4FA03168681D2DF82DF527CB106F3FA6
:10292000574FED37D96F1233D9FBC82D6F73E1A71D
:102930004AA1713F00000C4200008C436807002050
:10294000F5F751FD1390FE48806C0D901999F5F73D
:102950004AFD0E901999F5F746FD0F901999F5F774
:1029600042FD1190F648C06A01460B901A98F5F79F
:10297000E1FC0D90F248C06A01460A901A98F5F7FA
:10298000D9FC0B90EE48406C01460A900B98F5F785
:102990002AFD0C900D99F5F726FD0F90E848C06AC6
:1029A000014609901A98F5F7C5FC0A90E448006CB6
:1029B000014609900A98F5F716FD0B901999F5F75D
:1029C00012FD0D90DE48C06B08901999F5F70BFDCC
:1029D00009901999F5F707FD0B90D948C06A01468F
:1029E00006901A98F5F7A6FC0790D548806B01462B
:1029F00006900798F5F7F7FC0990D148406B0690D0
:102A00001999F5F7F0FC0790CD48006B0146069048
:102A10000798F5F78FFC08900999F5F78BFC0A9059
:102A20000B99F5F787FC0C900D99F5F783FC0E9048
:102A30000F99F5F77FFC10901199F5F77BFC129038
:102A40001399F5F777FC14901599F5F773FC169028
:102A50001799F5F76FFC1B90EBE1BA491898F5F759
:102A6000A5FF7DD2B648806D014613901A98F5F700
:102A700061FC1590B248806D014611901A98F5F7E7
:102A800059FC1390AE48806D014610901A98F5F7E6
:102A900051FC1190AA4880300068014610901198AE
:102AA000F5F7A1FC12901399F5F79DFC1490159978
:102AB000F5F799FC1790A248806D014610901A987E
:102AC000F5F738FC12909E48806D01460F901A98D9
:102AD000F5F730FC10909A48C06F01460F9010989F
:102AE000F5F781FC11901299F5F77DFC1390199977
:102AF000F5F779FC15909248806D01460E901A9872
:102B0000F5F718FC0F908E48806F01460E900F98D5
:102B1000F5F769FC10901999F5F765FC1190199972
:102B2000F5F761FC13908648406F0D901999F5F701
:102B30005AFC0E901999F5F756FC0F901999F5F774
:102B400052FC11907E48806D01460B901A98F5F763
:102B5000F1FB0D907A48806D01460A901A9800E0CA
:102B60006DE0F5F7E7FB0B907548006F01460A90A2
:102B70000B98F5F738FC0C900D99F5F734FC0F9095
:102B80006F48806D014609901A98F5F7D3FB0A90BB
:102B90006B48C06E014609900A98F5F724FC0B902B
:102BA0001999F5F720FC0D906548806E08901999E9
:102BB000F5F719FC09901999F5F715FC0B90604889
:102BC000806D014606901A98F5F7B4FB07905C48B3
:102BD000406E014606900798F5F705FC09905848A5
:102BE000006E06901999F5F7FEFB07905448C06DEA
:102BF000014606900798F5F79DFB08900999F5F7AF
:102C000099FB0A900B99F5F795FB0C900D99F5F748
:102C100091FB0E900F99F5F78DFB10901199F5F738
:102C200089FB12901399F5F785FB14901599F5F728
:102C300081FB16901799F5F77DFB1B90F9E0404852
:102C400080304068014613901A98F5F773FB159091
:102C50003B4880304068014611901A98F5F76AFBAE
:102C60001390374880304068014610901A98F5F765
:102C700061FB119032488030C06A01461090119873
:102C8000F5F7B1FB12901399F5F7ADFB1490159978
:102C9000F5F7A9FB17902A4880304068014610904C
:102CA0001A98F5F747FB1290254880304068014696
:102CB0000F901A98F5F73EFB109021488030806AFB
:102CC00001460F901098F5F78EFB11901299F5F7C9
:102CD0008AFB13901999F5F786FB159018488030F8
:102CE000406801460E901A98F5F724FB0F9014489F
:102CF0008030406A01460E900F98F5F774FB1090F3
:102D00001999F5F770FB11901999F5F76CFB139071
:102D10000B488030006A0D901999F5F764FB0E900E
:102D20001999F5F760FB0F901999F5F75CFB119075
:102D300003488030406801460B901A9804E0000078
:102D40006807002000008C43F5F7F4FA0D90FD4869
:102D5000406801460A901A98F5F7ECFA0B90F9488A
:102D6000C06901460A900B98F5F73DFB0C900D9950
:102D7000F5F739FB0F90F3484068014609901A981F
:102D8000F5F7D8FA0A90EF488069014609900A9849
:102D9000F5F729FB0B901999F5F725FB0D90E948FC
:102DA000406908901999F5F71EFB09901999F5F7F4
:102DB0001AFB0B90E3484068014606901A98F5F715
:102DC000B9FA0790DF480069014606900798F5F7C1
:102DD0000AFB0990DB48C06806901999F5F703FBD8
:102DE0000790D8488068014606900798F5F7A2FA40
:102DF00008900999F5F79EFA0A900B99F5F79AFA57
:102E00000C900D99F5F796FA0E900F99F5F792FA46
:102E100010901199F5F78EFA12901399F5F78AFA36
:102E200014901599F5F786FA16901799F5F782FA26
:102E30001B90C5491898F5F7B9FD18D8C348006824
:102E40008830F5F747FA1690C04800689030F5F7DB
:102E500041FA14901B99F5F7C6FA15901699F5F7F3
:102E600069FA17901B99F5F7BEFA1B9053E0B84921
:102E70001898F5F79BFD18D8B44800685C30F5F752
:102E800029FA1690B14800686430F5F723FA1490D7
:102E90001B99F5F7A8FA15901699F5F74BFA1790C4
:102EA0001B99F5F7A0FA1B9035E0AA491898F5F799
:102EB0007DFD18D8A54800683030F5F70BFA16905C
:102EC000A24800683830F5F705FA14901B99F5F719
:102ED0008AFA15901699F5F72DFA17901B99F5F7C0
:102EE00082FA1B9017E099480068001DF5F7F2F987
:102EF0001690964800680C30F5F7ECF914901B9981
:102F0000F5F771FA15901699F5F714FA17901B99C1
:102F1000F5F769FA1B903F2109061998F5F746FD68
:102F200002D200201DB000BD8B491998F5F73EFD77
:102F30000CD28A48F5F7CEF95F2805D387480C30C4
:102F4000F5F7C8F95F2801D20020EBE7844919980A
:102F5000F5F72CFD06D200201999F5F727FD01D0D1
:102F60000020DFE7F8F76AFE012806D17D491B98AB
:102F7000F5F71CFD01D80020D4E77848F5F7AAF949
:102F80001590F5F763FC0022774B17911690F5F733
:102F9000C9FC0DD371480C30F5F79CF91590F5F785
:102FA00055FC0022704B17911690F5F7BBFC07D229
:102FB000412109061B98F5F7F9FC01D80020B1E77B
:102FC00000211B98F5F7F2FC01D200201B905E490E
:102FD0001998F5F7EBFC38D2412109061B98F5F753
:102FE000E5FC05D261491B98F5F7FDF91B908AE2D3
:102FF000412109061B98F5F7E3FC0AD85C491B98A8
:10300000F5F7D4FC05D25B491B98F5F7ECF91B905A
:1030100079E257491B98F5F7D3FC0BD856491B9812
:10302000F5F7C4FC06D251491B98F5F7DCF91B9063
:1030300069E26DE250491B98F5F7C2FCD7D84F49B9
:103040001B98F5F7D0F91B905DE23F491998F5F709
:10305000B7FC2FD84A491998F5F7A8FC2AD2494954
:103060001B98F5F7A3FC05D242491B98F5F7BBF96D
:103070001B9048E243491B98F5F7A2FC0AD83C494B
:103080001B98F5F793FC05D23F491B98F5F7ABF970
:103090001B9038E236491B98F5F792FCA7D83649C1
:1030A0001B98F5F783FCA2D234491B98F5F79BF9DE
:1030B0001B9028E232491998F5F782FC14D833495D
:1030C0001998F5F773FC0FD22E491B98F5F778FC89
:1030D0008DD82F491B98F5F769FC88D225491B9894
:1030E000F5F781F91B900EE228491998F5F768FC6D
:1030F0007AD828491998F5F759FC75D216491B98C2
:10310000F5F754FC05D224491B98F5F76CF91B9090
:10311000F9E111491B98F5F753FC45D81F491B9855
:10312000F5F744FC40D21E481B99F5F75CF91D49A0
:103130001690F5F7FFF817901B99F5F754F91B90C7
:10314000E1E10000E807002000005041CC0300202E
:103150000000D041000096420000A0401819002055
:10316000CDCCCC3D0000104100006840D7A3803F8B
:10317000000004424E62803F0000BE428941803F11
:10318000000088410000B8411283803F3333E3419F
:1031900000000C4214AE064252B87E3F000040418F
:1031A000008FA83AFD127D3FDE491B98F5F708FC19
:1031B0000AD8DD491B98F5F7F9FB05D2DB491B98C6
:1031C000F5F711F91B909EE1D9491B98F5F7F8FB2B
:1031D0000BD8D8491B98F5F7E9FB06D2D6491B98BE
:1031E000F5F701F91B908EE10AE0D2491B98F5F73B
:1031F000E7FB8DD8CD491B98F5F7F5F81B9082E1D8
:10320000CE491998F5F7DCFB62D8CD491998F5F746
:10321000CDFB5DD2CB491B98F5F7C8FB05D2CA4957
:103220001B98F5F7E0F81B906DE1C6491B98F5F780
:10323000C7FB12D8BB491B98F5F7B8FB0DD2C348A2
:103240001B99F5F7D0F8C2491690F5F773F8179067
:103250001B99F5F7C8F81B9055E1B2491B98F5F793
:10326000AFFB0AD8B0491B98F5F7A0FB05D2B949C6
:103270001B98F5F7B8F81B9045E1AD491B98F5F799
:103280009FFB0AD8AB491B98F5F790FB05D2B249D2
:103290001B98F5F7A8F81B9035E1A6491B98F5F7A0
:1032A0008FFB0AD8AD491B98F5F780FB05D2A949D9
:1032B0001B98F5F798F81B9025E1A8491B98F5F79E
:1032C0007FFB90D8A6491B98F5F78DF81B901AE163
:1032D0009B491998F5F774FB77D8A2491998F5F727
:1032E00065FB7ED297491B98F5F760FB05D296499E
:1032F0001B98F5F778F81B9005E192491B98F5F7B4
:103300005FFB12D887491B98F5F750FB0DD2964802
:103310001B99F5F768F895491690F5F70BF8179093
:103320001B99F5F760F81B90EDE07E491B98F5F7C7
:1033300047FB0AD87C491B98F5F738FB05D28C4926
:103340001B98F5F750F81B90DDE077491B98F5F7CF
:1033500037FB0AD887491B98F5F728FB05D2764931
:103360001B98F5F740F81B90CDE083491B98F5F7C3
:1033700027FB0AD86E491B98F5F718FB05D276494A
:103380001B98F5F730F81B90BDE069491B98F5F7DD
:1033900017FB0AD867491B98F5F708FB05D26D495A
:1033A0001B98F5F720F81B90ADE062491B98F5F7E4
:1033B00007FB0BD869491B98F5F7F8FA06D26F4955
:1033C0001B98F5F710F81B909DE00AE063491B98E5
:1033D000F5F7F6FA04D86A491B98F5F704F81B903C
:1033E00091E060491998F5F7EBFA09D855491B980F
:1033F000F5F7DCFA05D254491B98F4F7F4FF1B905B
:1034000081E050491B98F5F7DBFA12D845491B9823
:10341000F5F7CCFA0DD254481B99F4F7E4FF534961
:103420001690F4F787FF17901B99F4F7DCFF1B90B9
:1034300069E03C491B98F5F7C3FA0AD83A491B984A
:10344000F5F7B4FA05D24A491B98F4F7CCFF1B9064
:1034500059E035491B98F5F7B3FA0AD845491B9846
:10346000F5F7A4FA05D234491B98F4F7BCFF1B907A
:1034700049E041491B98F5F7A3FA0AD841491B983E
:10348000F5F794FA05D229491B98F4F7ACFF1B9085
:1034900039E03C491B98F5F793FA0AD824491B9860
:1034A000F5F784FA05D238491B98F4F79CFF1B9076
:1034B00029E01F491B98F5F783FA0AD81D491B9884
:1034C000F5F774FA05D22D491B98F4F78CFF1B9081
:1034D00019E018491B98F5F773FA0AD81F491B9889
:1034E000F5F764FA05D229491B98F4F77CFF1B9085
:1034F00009E01A491B98F5F763FA04D824491B9888
:10350000F4F771FF1B901B9817F008FB1B9000BF8E
:1035100020491B98F5F754FA01D21E481B901B98BE
:1035200000E500000000404100000C421283803F93
:103530000080D444004003458941803F14AE0642D8
:10354000000010420000A040A4707D3F6F12033BBA
:1035500048E17A3FD7A3803F4E62803F00002F456D
:103560002506813F00002C42B7D0153BA1837A3F4E
:103570009CC4803F0000484200009642E926813FFB
:10358000FCA9813F00009C4260E5803FC1CA813FA9
:10359000D34D823F00409245F0B585B004460027E8
:1035A0000020039002900190FAF7ECFE002802D16F
:1035B00001209749087097480078002806D0012814
:1035C00023D002282AD0032871D111E100212046FE
:1035D000F5F7ECF918D003F02BFD0A2805D18E4839
:1035E000F4F778FE8D49086004E08D48F4F772FE28
:1035F0008A49086003210C200BF07CF800208449E4
:103600000870012083490870FFE00C200AF0A4FE36
:10361000002802D102207F490870F6E000212046F0
:10362000F5F7C4F97ED103F003FD0A287BD17A486F
:10363000F4F750FE0546794801682846F4F7CBFEBA
:1036400007463F2109063846F4F7C5FE03907F215F
:10365000C9053846F4F7BFFE029072493846F4F7C0
:10366000BAFE019070490298F5F7AAF920D86F497F
:103670000298F5F79BF91BD86748F4F72BFE06462E
:103680006B490298F4F7AFFE31460090F4F7A7FEBD
:1036900005466149F4F736FE5F48F4F71BFE0090DB
:1036A000F5F72CF90546634AF4F735FE9AE0A8E0F1
:1036B00061490398F5F784F91FD860490398F5F735
:1036C00075F91AD85448F4F705FE06465849039888
:1036D000F4F789FE31460090F4F781FE05464E4925
:1036E000F4F710FE4C48F4F7F5FD0090F5F706F9F5
:1036F0000546504AF4F70FFE74E051490198F5F77A
:103700005FF96FD84F490198F5F750F96AD84048EA
:103710000078012866D14048F4F7DCFD06464A49A6
:10372000019801E063E014E0F4F75DFE314600909B
:10373000F4F755FE05463849F4F7E4FD3648F4F74A
:10374000C9FD0090F5F7DAF805463A4AF4F7E3FDCB
:1037500048E03348F4F7BEFD054630480168284686
:10376000F4F739FE074639493846F4F734FE03903A
:1037700037493846F4F72FFE029036490298F5F79C
:103780001FF915D834490298F5F710F910D82448D4
:10379000F4F7A0FD064626490298F4F724FE3146C8
:1037A0000090F4F71CFE05461D49F4F7ABFD19E047
:1037B0002A490398F5F704F914D829490398F5F72D
:1037C000F5F80FD81648F4F785FD06461849039812
:1037D000F4F709FE31460090F4F701FE0546104962
:1037E000F4F790FD00200A4908700A4908700CE0BF
:1037F00000212046F5F7DAF802D1002005490870CB
:1038000003E000200349087000BF00BF05B0F0BD11
:10381000E8030020E303002004190020E403002053
:103820004C19002000002041295C0FBD295C0F3D90
:10383000CDCC4C3E9D030020295C8FBC295C8F3C85
:10384000CDCC4CBFCDCC4C3F9A99593F0000FA43A8
:1038500000007A4400000CC200000C4200008CC141
:1038600000008C4103480078012800D170470020F7
:10387000FCE700008D02002010B5FCF769F8FCF7AA
:10388000D9F80020154908601549086015490870E5
:1038900015490870154908701549087015490870D0
:1038A0001549087004201549087000201449087053
:1038B00014490870144908701449086014490860D4
:1038C000144908600DF0D6F9104908601920FBF77B
:1038D00029FBC1B21048C17010BD00007C0200205D
:1038E0008002002084020020850200208602002041
:1038F00087020020880200208D020020890200201B
:103900008A0200208B0200208C02002098020020F6
:1039100090020020940200209A000020F8B50026B2
:103920000024FE480078232801D301F000F843006A
:103930007B449B885B009F4422005100A100F6005D
:1039400012012F015603D803FA0341045E047E04DA
:10395000CB042706DF060607AF07FA07C407E2070E
:103960004E016A018A01DA01FA07DD00E704070562
:103970005705B7050A06D4021D0375069506E849E2
:1039800001200006F4F7BEFCE5481C38C07810287A
:1039900003DD1021E2481C38C170E248007801289C
:1039A00002D10020DF4908700DF064F9DE4908609B
:1039B0000120DA490870DD4908700020DC490870F0
:1039C000DC4908700120DC4908600020DB49086000
:1039D000DB48DC490860FCF705F8C4E34E20FBF740
:1039E00097FA00282AD00DF045F9CF490968401A06
:1039F000D549884241D94E20FBF79CFACC48007843
:103A000001283AD10DF036F9C74908600020C849AD
:103A100008700220C14908700120C44908700220C2
:103A2000C54908600420C5490860C848C549086000
:103A3000C748C8490860FBF7D5FF1EE0BC480078BE
:103A400001281AD10DF016F9B74908600020B849CD
:103A500008700220B14908700120B44908700220A2
:103A6000B54908600420B5490860B848B549086000
:103A7000B748B8490860FBF7B5FFAEE7AD48007836
:103A8000012836D10020AB490870B148C078B2494E
:103A90004870084640780421084004280AD10020D4
:103AA000AE4908600DF0E6F89F49086019209B496F
:103AB00008701EE0A9480068401CA8490860084634
:103AC0000068FF212D3188420ED90020A3490860EB
:103AD0000220A3490870A348007801210843A149A6
:103AE0000870FDF7A7FE04E00120914908708B499A
:103AF000087072E700208E4908700320874908701B
:103B000001208A4908700DF0B5F887490860062041
:103B100089490860002089490860934889490860FC
:103B2000FBF760FF59E782480078012816D1002092
:103B30007F4908700DF09EF87B49086004207749A2
:103B400008700120794908707B49086000207B4992
:103B5000086086487B490860FBF744FF3DE77448EE
:103B60000078012817D10DF085F86F490860002012
:103B70006F49087005206949087001206B49087079
:103B800006206D49086000206C49086078486D493E
:103B90000860FBF727FF20E765480078012819D166
:103BA0000DF068F860490860002061490870142031
:103BB0005A49087001205D49087006205E49086076
:103BC00000205E4908606B4908706B485D490860D9
:103BD000FBF708FF01E756480078012816D10020BE
:103BE0005349087015204D4908700DF043F84E49AF
:103BF000086001204D4908704F49086000204F4976
:103C000008605E484F490860FBF7ECFEE5E648486F
:103C1000007801281AD10DF02DF8434908600020E2
:103C20004349087016203D49087001203F4908703B
:103C30000220414908600420404908604348414946
:103C40000860434843490860FBF7CCFEC5E63948A5
:103C5000007801284AD10020364908703C48C078D5
:103C60003D49C8700846C0780821084008281DD181
:103C700000203A4908602E4908700CF0FBFF2A49E1
:103C80000860172025490870012028490870022083
:103C900029490860042029490860394829490860F1
:103CA0002B482C490860FBF79DFE1FE02B4800685D
:103CB000401C2A49086008460068FF212D318842CF
:103CC0000ED90020254908600220254908702548A2
:103CD00000780121084323490870FDF7ABFD05E09A
:103CE00001201349087015200C49087075E6114829
:103CF000007801287DD100200E4908700C49087019
:103D00000CF0B8FF08490860114800781249C870E3
:103D10000F48407888700E48807833E08502002094
:103D2000B60000208B0200209802002086020020AE
:103D30008802002087020020800200207C020020F0
:103D400018BF02006402002050C30000EABE020057
:103D50006C020020680200205C000020900200201D
:103D6000890200208A020020D2BE020019BF020090
:103D7000D8BE020078020020DEBE02001CBF020096
:103D800006BF02004870F848C078087000201AE0AA
:103D9000014609318900F54A525C01460931890022
:103DA000F24BC91849785218014609318900C918DF
:103DB00089785218014609318900C918C978511803
:103DC0000C19411CC8B21028E2DB2106FF221202A6
:103DD000224012021143FF2212042240120A114310
:103DE000220E11430846E249F4F78CFA0024002021
:103DF0001BE075E001464F318900DC4A525C014608
:103E00004F318900D94BC9184978521801464F31B2
:103E10008900C9188978521801464F318900C9189C
:103E2000C97851180C19411CC8B22E28E2DB2106B2
:103E3000FF221202224012021143FF2212042240EA
:103E4000120A1143220E11430846C949091DF4F70D
:103E500059FA002004E0C749095C8E19411C88B258
:103E6000432109018842F6D33106FF221202324073
:103E700012021143FF2212043240120A1143320E81
:103E800011430846BA490831F4F73CFABA48F4F746
:103E900021FAB04210D00620B84908700120B84974
:103EA0000870B84908600020B7490860B748B849A9
:103EB0000860FBF797FD13E01F20B0490870012050
:103EC000AF4908700220AF4908600420AE4908607D
:103ED000B048AF490860A448AF490860FBF782FDCD
:103EE0007BE5AE480078012843D10020AB4908703B
:103EF000AB4908700CF0BEFEAA4908609A480078E9
:103F00009D49087098484078487097488078887034
:103F10009548C078C8709648F4F7DCF9054696488D
:103F2000F4F7D8F9854210D0072094490870012091
:103F300093490870934908600020934908609348AA
:103F400093490860FBF74EFD13E020208B49087071
:103F500001208B49087002208A49086004208A49A0
:103F6000086091488A4908607F488B490860FBF7E0
:103F700039FD32E589480078012833D1002087498E
:103F80000870874908700CF075FE8649086076480D
:103F90000078794908707448407848707248807891
:103FA00088707148C078C8707148001DF4F792F9A4
:103FB00005467148F4F78EF9854203D007206F4912
:103FC000087002E01E206D49087001206C490870DD
:103FD0006C49086000206C4908606C486C490860B6
:103FE000FBF700FDF9E46E48007801287CD100253C
:103FF00000206B4908700CF03DFE6A4908606B4870
:104000000068401E6A490978884235D95C206949B0
:10401000087067490878C10F09184910654A51703E
:1040200063490878C10F091849104900411AC907A6
:10403000090E917000BF09E05D480078C001401989
:104040004C49095CE81C5B4A11546D1C802DF3D36C
:1040500001204B49087083204A49086000204A49E2
:10406000086054484A490860FBF7BCFC5048007897
:10407000401C4F49087036E05C204E4908704C499E
:104080000878C10F091849104A4A51704849087800
:10409000C10F091849104900411AC907090E91704A
:1040A000002509E042480078C00140193149095C07
:1040B000E81C404A11546D1C3F4800688542F1D30A
:1040C00001202F4908703C480068C01C2D49086039
:1040D00000202D49086037482D490860FBF782FC15
:1040E00007202649087000BF77E42D480078012892
:1040F0001CD10CF0BFFD2B49086000202849087036
:1041000008201E49087001201D490870FF20FF305B
:104110001C49086000201C490860012018490870EB
:104120001248801C1A490860FBF75CFC55E41C48E7
:104130000078012816D10CF09DFD1A490860002076
:104140001749087009200D49087001200C490870B2
:104150000C49086000200C4908600C480C490860B4
:10416000FBF740FCE4E30EE26C020020620000205A
:10417000560200201DBF02005C00002085020020C6
:1041800086020020800200207C0200201ABF02006C
:104190006402002008BF020068020020870200209D
:1041A00088020020980200200ABF0200700200204E
:1041B000780200205414002074020020FE48007889
:1041C000012817D10CF056FDFC4908600020FA497F
:1041D00008700A20FA4908700120FA490870062080
:1041E000F94908600020F9490860F948F949086070
:1041F000FBF7F8FB9CE3F048007801281AD10CF09B
:1042000039FDEE4908600020EB4908700B20EC49AD
:1042100008700120EB4908700220EB490860042077
:10422000EA490860EC48EB490860EC48EC49086052
:10423000FBF7D8FB7CE3EB480078012847D100204E
:10424000E8490870E548C078E749C8700846C07872
:104250000221084002281AD10020E44908600CF02D
:1042600009FDD64908600020D34908700C20D449C4
:1042700008700120D3490870D34908600020D34951
:104280000860DB48D3490860FBF7ACFB1FE0D74868
:104290000068401CD549086008460068FF212D31A0
:1042A00088420ED90020D14908600220D149087007
:1042B000D148007801210843CF490870FDF7BAFAC8
:1042C00005E00120BC4908700A20BD4908702FE3B1
:1042D000B9480078012816D10CF0CCFCB749086029
:1042E0000020B54908701A20B54908700120B54969
:1042F0000870B54908600020B4490860BF48B54956
:104300000860FBF76FFB13E3AB48007801281AD174
:104310000CF0B0FCA94908600020A74908701B20D8
:10432000A74908700120A74908700220A649086023
:104330000420A6490860A848A6490860A748A849DB
:104340000860FBF74FFBF3E2A648007801284AD14A
:104350000020A4490870A148C078A349C870084645
:10436000C0780821084008281DD100209F49086016
:10437000914908700CF07EFC904908601C2090491F
:10438000087001208F49087002208F4908600420BE
:104390008E4908609A488F490860904890490860A3
:1043A000FBF720FB1FE091480068401C8F49086024
:1043B00008460068FF212D3188420ED900208B4924
:1043C000086002208B4908708B480078012108435F
:1043D00089490870FDF72EFA05E00120764908703A
:1043E0001A2077490870A3E27E48007801285AD144
:1043F00000207C490870704908700CF03BFC6F4944
:1044000008607648007878490870744840784870A9
:104410007248807888707148C078C8707948F3F71E
:1044200059FF05467048F3F755FF854227D0764877
:104430000068401C744908600846006803280DD9CC
:104440000020086002206B4908706B480078012149
:10445000084369490870FDF7EDF924E00720584941
:1044600008700120574908705749086000205749D3
:1044700008605F4857490860FBF7B4FA13E01D2055
:104480004F49087001204F49087002204E490860CA
:1044900004204E4908605D484E4908604F48504925
:1044A0000860FBF79FFA43E24E48007801284DD19F
:1044B00000204C490870404908700CF0DBFB3F4974
:1044C0000860464800784849087044484078487079
:1044D0004248807888704148C078C8704948001DBB
:1044E000F3F7F8FE05464048F3F7F4FE85421AD08C
:1044F00045480068401C4449086008460068032895
:104500000DD90020086002203A4908703A48007826
:104510000121084338490870FDF78CF909E00720AC
:104520002749087005E00020374908601E2024490B
:10453000087001202349087023490860002023499E
:1045400008602B4823490860FBF74CFAF0E11A4851
:104550000078012817D10CF08DFB18490860002065
:10456000154908700D20164908700120154908707A
:1045700006201549086000201449086024481549A0
:104580000860FBF72FFAD3E10B480078012848D1E7
:104590000CF070FB094908600020074908700120F1
:1045A000084908700849086000200849086019484F
:1045B0000849086030E000008802002098020020CE
:1045C0008502002086020020800200207C0200205C
:1045D000ECBE020064020020EABE02006C02002071
:1045E00068020020870200205C000020900200206A
:1045F0001ABF0200890200208A0200201CBF0200AC
:1046000008BF020056020020940200200ABF0200E8
:10461000F2BE020018BF0200FBF7E4F92120D549E1
:10462000087085E1D448007801281AD10CF022FBEB
:10463000D24908600020D04908702220CD49087076
:104640000120CF4908700220CE4908600420CE49DD
:104650000860CE48CE490860CE48CF490860FBF7D5
:10466000C1F965E1CD480078012844D10020CB494B
:104670000870C848C078CA49487008464078042184
:104680000840042817D10020C64908600CF0F2FA4F
:10469000BA4908600120BA490870BA490860002088
:1046A000B9490860C048BA490860FBF79BF90E2079
:1046B000B04908701FE0BB480068401CB949086059
:1046C00008460068FF212D3188420ED90020B549E7
:1046D00008600220B5490870B548007801210843F8
:1046E000B3490870FDF7A6F805E00120A24908705B
:1046F0002120A04908701BE19F480078012821D1A2
:104700000020AC4908709C4908700CF0B3FA9B4932
:104710000860A948C078A8491431C97848437D2168
:104720004843C117490E0918C8117D21C900F3F784
:1047300007FDC01C87B23946082009F0DBFF0F20B7
:104740008C490870F4E0082009F006FE00280BD11F
:104750000220964908709648007801210843944940
:104760000870FDF767F896E09248007801283ED17E
:1047700092480088FF2101310843904908800020B9
:104780008F4908708B4908708B48C0788A4914316A
:10479000C97848437D214843C117490E0918C811FB
:1047A0007D21C900F3F7CCFCC01C87B23946082034
:1047B00009F0A0FF0CF05EFA7049086012206D4904
:1047C000087001206E49087002206E4908607A481E
:1047D0001430C0780C2148436B49086079486C4913
:1047E000086079486C490860FBF7FCF853E07748AB
:1047F000007801280BD1F8F7D1F9012807D1002062
:104800006F490870714908705A49087043E0FDF714
:104810002FF801281AD1FDF745F8002068490870E3
:104820000CF028FA55490860102052490870012000
:104830005349087006205349086000205249086017
:10484000634853490860FBF7CDF824E0FDF710F802
:1048500002281AD1FDF726F80020594908700CF0FB
:1048600009FA46490860102042490870012044496D
:1048700008700620434908600020434908605548F5
:1048800043490860FBF7AEF805E001204C49087089
:104890000F20384908704BE03748007801280CD1C8
:1048A00000203E490870344908703649086036498E
:1048B00008600F202F49087002E010202D49087071
:1048C00036E036480078012815D1002033490870B9
:1048D00029490870132027490870012028490870C9
:1048E000284908600020284908602F4828490860A6
:1048F000FBF778F802E012201E49087018E01E4805
:10490000007801280FD10020244908701A49087046
:104910001C4908601C4908600120244908700F20C8
:104920001449087002E013201249087000E000BF2B
:1049300000BF104800780F281BD00E4800780028D0
:1049400017D00CF097F90D490968401A224988429E
:104950000FD3174800780221084315490870022038
:104960001249087000200849086006490860FCF7F1
:1049700061FFF8BD85020020880200209802002017
:1049800086020020800200207C020020EABE020095
:10499000640200206C0200206802002087020020D0
:1049A0005C000020900200201ABF02008902002053
:1049B0008A0200208402002086000020C00400201B
:1049C0008D020020F8BE0200941300208B0200200C
:1049D00012BF02000CBF0200B0AD01007047000022
:1049E00010B525480078002804D0012812D00228EC
:1049F0003ED12AE002F01CFB0A2805D107F080FC1A
:104A000002201D49087004E000F0B0F801201A49A6
:104A100008702EE002F00CFB0A2815D1002002F0ED
:104A20000BFA002015490870082000F08DF80020CE
:104A30001349086013490860134908601348144972
:104A4000086002200C49087013E002F0F1FA012816
:104A50000DD100200F49088000F088F8102000F0E8
:104A600073F80D480A49086001200349087000E006
:104A700000BF00BF10BD00007C03002052030020D7
:104A8000087F00200C7F0020187F00205A6B7C8D4F
:104A9000107F00201C7F00208D7C6B5AF8B52548C4
:104AA0000078002802D0012840D107E03C210520F1
:104AB00009F020FE01201F49087038E0052009F0A8
:104AC0004BFC002831D1022000F0F2F900901220B6
:104AD000FAF71EFA00281ED11748F3F7FBFB05462C
:104AE00029460098F3F777FC04461449F3F768FF6A
:104AF00011D21148F3F7EEFB04461149F3F702FC1B
:104B00000F48F3F7E7FB0646F3F7F8FE04460D4AB5
:104B1000F3F701FC06E01220FAF70CFA06490098B8
:104B2000F3F7F0FB00200349087000E000BF00BF6E
:104B3000F8BD0000340300203503002000001643B8
:104B4000041900209D030020082803D10121064AF2
:104B5000117008E0102803D10221034A117002E00D
:104B60000021014A117070478C020020F0B585B019
:104B700009F048F80546802102F022F90CF07AF895
:104B8000964908600421964809F018F8012817D0C2
:104B90000421944809F012F8012811D0002190480E
:104BA0000068F3F703FF0BD38F498D480068F3F7D4
:104BB00007FF05D300218B480068F3F7F7FE04D206
:104BC000002087490860874908600221874808F06B
:104BD000F5FF012802D10020844908804D20FAF712
:104BE00097F9002843D04D20FAF7A4F97F480088B0
:104BF000F3F711FE432109060290F3F731FC7C49DB
:104C00000390F3F797FB0746754801683846F3F7BA
:104C1000EAFB0646734801683046F3F78BFB05460E
:104C20007449F3F76FFB7448F3F754FB03906F4834
:104C30000088F3F7F0FD432109060090F3F710FC1C
:104C40006B490190F3F776FB029065480168029882
:104C5000F3F7C9FB07466949F3F702FC06460399D7
:104C6000F3F768FB05466449F3F74CFB3FE05F4808
:104C70000088F3F7D0FD432109060290F3F7F0FB1B
:104C800007465F49F3F756FB0390554801680398C0
:104C9000F3F7A9FB0646534801683046F3F74AFB91
:104CA00005465449F3F72EFB5348F3F713FB0390E3
:104CB0004E480088F3F7AFFD432109060090F3F753
:104CC000CFFB07464E49F3F735FB01904448016896
:104CD0000198F3F788FB49490290F3F7C1FB0646B8
:104CE0000399F3F727FB05464349F3F70BFB4248CB
:104CF000F3F7F0FA0746F3F701FE0546414AF3F7EA
:104D00000AFB00204049086001204049087000204B
:104D10003F4908703749091DF3F7F4FA354908315E
:104D20000020F3F7EFFA344908310020F3F7EAFAEC
:104D3000304930310020F3F7E5FA2E4934310020B4
:104D4000F3F7E0FA2B4938310020F3F7DBFA294971
:104D50003C310020F3F7D6FA264940310020F3F722
:104D6000D1FA002405E00020A1002A4A5050601C1E
:104D700084B2102CF7DB40212748F3F784FA002493
:104D800005E00020A100254A5050601C84B2102C80
:104D9000F7DB002405E00020A100214A5050601CF0
:104DA00084B2142CF7DB002405E00020A1001D4A8A
:104DB0005050601C84B21E2CF7DB00201A4908807A
:104DC0001A4908701A4908801A4908801A49087057
:104DD0001A4908601A49087005B0F0BD6403002044
:104DE0000C7F0020087F00200080BB441C7F002037
:104DF000666616404C1900200419002000007A4411
:104E00003333B33E9D030020187F00207D03002034
:104E1000520300205017002090170020D0170020C8
:104E200010180020601800204C0300204E030020C2
:104E300040030020420300204403002078030020A8
:104E4000450300200349C9788900034A8918016095
:104E5000704700009A0000209413002010B5022132
:104E6000C02000F02BFD012805D103490870022164
:104E7000C02000F0F7FC10BD840200200349C9786F
:104E8000C900034A89180160704700009A00002099
:104E90009413002005480078002804D0002003491E
:104EA0000870012070470020FCE70000C7030020C5
:104EB000F8B5044623000FF0E2FE0D6A080C2A3D07
:104EC00042474C51565B60656A003248F3F702FA7C
:104ED000F8BD30480838F3F7FDF905460021F3F72F
:104EE00065FD0FD22B4908390020F3F70BFA29484A
:104EF0000838F3F7EFF90746F3F700FD0546264AB1
:104F0000F3F709FA23480838F3F7E4F9E0E7214812
:104F1000001FF3F7DFF905460021F3F747FD04D240
:104F20001C49091F0020F3F7EDF91A48001FF3F799
:104F3000D1F9CDE71748001DF3F7CCF9C8E71548BC
:104F40000830F3F7C7F9C3E712480C30F3F7C2F99A
:104F5000BEE710481030F3F7BDF9B9E70D4814303B
:104F6000F3F7B8F9B4E70B481830F3F7B3F9AFE744
:104F700008481C30F3F7AEF9AAE706482030F3F7EB
:104F8000A9F9A5E703482430F3F7A4F9A0E7002026
:104F9000C0439DE70C1900209D0300200020144908
:104FA0000979134AD27852001143114A527992007A
:104FB00011430F4A5278D20011430D4A127A12015E
:104FC00011430B4A927852011143094AD279920156
:104FD0001143074A1278D2011143054A927912020D
:104FE0001143034A527A5202114388B270470000BB
:104FF000A419002001490160704700008E160020AE
:1050000070B5044623000FF03AFE0D4C080C111643
:1050100023282D3A3F444C494C002348F3F75AF9D2
:1050200070BD21480838F3F755F9F9E71E48001F0D
:10503000F3F750F9F4E70020FBF742F805461A4968
:10504000091DF3F75FF91848001DF3F743F9E7E787
:1050500015480830F3F73EF9E2E713480C30F3F750
:1050600039F9DDE70120FBF72BF805460E49103131
:10507000F3F748F90C481030F3F72CF9D0E70A4859
:105080001430F3F727F9CBE707481830F3F722F984
:10509000C6E705481C30F3F71DF9C1E7034800686F
:1050A000BEE70020C043BBE7541900203C030020AA
:1050B000FEB505460C462846F3F7ADFB07468F21A3
:1050C000C905F3F7CDF906462046F3F7A4FB3146B0
:1050D0000090F3F788F90746F3F7C6FB01900198B3
:1050E00000F094FDFEBD70B504462046F3F793FB37
:1050F00005468F21C905F3F7B3F970BD70B50024DB
:10510000F6F79CFD012827D12948F3F7E3F8C00FF3
:10511000C0070121C907884210D12548F3F7DAF802
:10512000C043461C3046FFF7DEFF054621480168B4
:105130002846F3F7FFF81F4908600DE01C48F3F715
:10514000C9F80646FFF7CFFF05461A48016828460A
:10515000F3F745F917490860164800680121C907A7
:105160004840044614492046F3F720FC04D3134971
:105170002046F3F725FC00D270BD00212046F3F74E
:1051800015FC0CD20120C00744402046F9F704FE6C
:10519000401EC54306492846F3F7B4F806E020460A
:1051A000F9F7FAFD05460249F3F7ACF800BFE3E76B
:1051B000161A0020B40300200AD723BD0AD7233DC6
:1051C0000148006870470000107F002010B50D48AE
:1051D0000078002813D10C48007800280FD10B4824
:1051E000007801280BD10A480078002807D1FCF785
:1051F00039FB04210840042801D1012010BD002002
:10520000FCE70000B8030020B1030020C403002025
:105210003903002010B50020284988704870C870F4
:1052200008702749087027490870274908702749DE
:1052300008702749087005E0F7F728FDFAF710F81D
:10524000FCF7AAF8234800780028F5D0042122486A
:1052500008F0B4FC01280BD000211F480068F3F7C8
:10526000A5FB05D31D491C480068F3F7A9FB02D232
:105270001B48194908601B4800681B4988420AD02E
:10528000184800681949884205D017481549086030
:10529000134811490860134800681449884206D130
:1052A0001020FFF751FC0020F9F7E0FF04E0002098
:1052B0000F4908600F49086010BD0000A4190020C4
:1052C0007C03002039030020B1030020C403002028
:1052D00034030020C6030020387F00200000704205
:1052E0000000A041107F00205A6B7C8D8D7C6B5A92
:1052F000087F00200C7F0020F8B507460C46384692
:10530000F3F789FA05461549F2F7FCFF1348F2F75F
:10531000E1FF0090F3F7F2FA0546114AF2F7FBFFBE
:105320000E48F2F7D7FF05460E49F2F7EBFF0B48A0
:10533000F2F7D0FF0C4908602046F3F76CFA0546F7
:105340000649091DF2F7DEFF0448001DF2F7C2FF0F
:1053500006490860012006490870F8BD04190020BC
:105360009D0300207E030020007F0020047F00209A
:10537000B0030020FEB5FFF733FBFBF757FC08F046
:10538000D1FC01F055FE0A2856D172480078002859
:1053900002D001284FD122E008F0CEFF08210840BA
:1053A00008281BD1FAF746FC012817D1032008F082
:1053B000EBFFFAF745FCF9F703FD0BF05BFC6649E0
:1053C000086066480078FCF7F7FAF8F7DBFF00287A
:1053D00004D10120624908705E4908702BE0FAF799
:1053E00029FC012826D1032008F0CEFFFAF728FC7B
:1053F000F9F7E6FC0BF03EFC57490968401A594999
:1054000008600BF037FC544908605648006856495C
:10541000884202D955485349086050480078FCF743
:10542000CBFAF8F7AFFF012804D1002049490870F2
:105430004B49087000BF84E001F0FAFD012819D142
:10544000FAF7F2FD012815D10BF014FC4849086069
:10545000FAF7F0FB012874D1FAF7F2FBF6F788FCB3
:10546000F9F7AEFC3D480078FCF7A6FA2220F9F7E0
:1054700061FD66E001F0DCFD012862D10BF0FAFB72
:105480003B490968401A3B4988425AD32220F9F720
:105490003FFD002852D1F8F775FF012851D1364859
:1054A0000088F3F7B8F9432109060290F2F7D8FF14
:1054B00007463249F2F73EFF06463148016830465A
:1054C000F2F791FF05462F4801682846F2F732FFB0
:1054D00004462D49F2F716FF2C48F2F7FBFE029026
:1054E00025480088F3F797F9432109060090F2F761
:1054F000B7FF22490190F2F71DFF074620480168D7
:105500003846F2F770FF06462149F2F7A9FF054633
:105510000299F2F70FFF04461C49F2F7F3FE1B480D
:10552000F2F7D8FE0646F3F7E9F90446194AF2F70E
:10553000F2FE022004F026FD0FF0ECFB2220F9F72A
:10554000F9FCFBF763FEFCF7ABF8FFF7A7FAF7F7F8
:1055500069FFFEBDB8030020BC03002070030020DB
:10556000C0030020D40300208096980080841E0091
:1055700064030020E0C810001C7F00203333B33EDA
:105580000C7F0020087F00204C1900200419002007
:1055900000007A449D030020012003490870002088
:1055A00002490870704700008D020020850200202B
:1055B000FEB505466248066807686248057062489D
:1055C0000570002D68D02E20F9F7A2FC002802D02B
:1055D0000020FAF741FB002405E00020A1005B4A0F
:1055E0005050601C84B2102CF7DB002405E0002032
:1055F000A100574A5050601C84B2142CF7DB0024E1
:1056000005E00020A100534A5050601C84B21E2CBB
:10561000F7DB002050490870504908805049088045
:105620005049088050490870504908605049087036
:105630005049F2F767FE50490020F2F763FE4E49E9
:1056400028310020F2F75EFE4B492C310020F2F7A2
:1056500059FE494930310020F2F754FE45493431B2
:105660000020F2F74FFE434938310020F2F74AFE9E
:10567000002405E00020A100314A5050601C84B293
:105680000A2CF7DB00203D4908703D4908703D4970
:1056900008703D49086051E02E20F9F74BFC0120CD
:1056A000FAF7DAFA36480078032840DD00241EE0D5
:1056B000A100234A50583146F3F782F902D8A000DE
:1056C0001F490E58A1001E4A50583946F3F76EF98B
:1056D00002D8A0001A490F58A000194A11582A48A8
:1056E0000068F2F727FE28490860601C84B224484D
:1056F00000788442DCDB22490978881EF3F780F8C1
:105700003146029020480068F2F765FE3946009065
:10571000F2F761FE01900299F2F7A2FE1A490860C1
:1057200000201749087001201649087006E0002083
:10573000134908701349087013490860FEBD000042
:10574000D81800207D03002051030020D01700202E
:1057500010180020601800204E0300204C03002089
:10576000400300204203002044030020780300206F
:10577000450300200C190020541900204F0300207D
:1057800050030020520300205403002010B50522CE
:105790000D490E480BF042FB00F02AF80C48027845
:1057A0000C490D48F8F732FB0C49086008480178AD
:1057B0000B48F8F77DFA0B49086006220A490B48A6
:1057C000F3F75AFB10BD0000941F0020801F00203B
:1057D0005C040020A81A0020801A00206004002029
:1057E000A81F002064040020581A0020401A00203E
:1057F00010B51748F2F76EFD164909688900164A78
:10580000505013480C30F2F765FD124909688900C1
:10581000124A50500F480068401C0E490860084664
:1058200000680A2808D00E4800680A2807D00846F1
:1058300000680B49086002E00A20094908600A2153
:1058400004480068F2F766FC0248016010BD0000E1
:105850005819002058040020801A0020A81A00209F
:105860005C04002070B504460D460449601800220F
:10587000294609F0C7FE002070BD0000100E02404E
:10588000F8B504460E4615460548A9004018071904
:1058900001223146384609F0B5FE0020F8BD00006F
:1058A000300D024070B504460D4603496018294684
:1058B000FAF796FB70BD0000040D024070B5044677
:1058C0000D46034960182946FAF78AFB70BD0000AF
:1058D000000E024070B504460E4615462149601878
:1058E0000022314609F08EFE00201F496118B200E7
:1058F00088502A781B49091F6018314609F082FE3A
:105900006A7818490C396018314609F07BFEAA788C
:10591000144910316018314609F074FEEA781149D3
:1059200014316018314609F06DFE2A790D4918319D
:105930006018314609F066FE6A790A49203160181C
:10594000314609F05FFE094880680121C903884398
:10595000A979C9030122D203114008430349886091
:10596000002070BD0C0D0240000C0240000F0240F0
:1059700010B50346024818188C000251002010BDD3
:10598000000C024070B504460D460449601801221F
:10599000294609F037FE002070BD00000C0D0240C2
:1059A00070B504460D46164603496018324629462E
:1059B00009F028FE002070BD080D024001460429B0
:1059C00001D1024800E00248704700000002004098
:1059D000004000400146002906D0012907D00229D5
:1059E00007D0032909D106E00120800706E004481A
:1059F00004E0044802E0044800E000BF00BF704734
:105A000000010040006000400064004070B588B0B4
:105A1000044600250026042C01D0052C71D110214C
:105A200068460FF083FF2046FFF7C8FF0546362182
:105A300061435D4A891808461030F2F74BFC81B289
:105A40006846418036216143574A89180846143018
:105A5000F2F740FCC1B268464170362060435249BB
:105A600040180830007E01281AD10020694688803D
:105A70000AF054FD0290362161434B4A89180846CA
:105A80001C30F2F727FC81B26846C18036216143A1
:105A9000454A891808460830F2F71CFC039013E0C9
:105AA0000320C002694688804B21490202910121EE
:105AB00089026846C180362161433B4A89180846FD
:105AC0000830F2F707FC039036206043364940184F
:105AD0000830407E69460870284601F03FFA0021F0
:105AE000284601F005FA0121284601F001FA0021BB
:105AF000284601F01CFA0121284601F004FA51E081
:105B0000FFE7102104A80FF011FF2046FFF762FF06
:105B1000064636216143244A891808461030F2F7B8
:105B2000D9FB81B268464182362161431E4A8918F9
:105B300008461430F2F7CEFBC1B2684641740AF051
:105B4000EDFC069036216143174A891808461C303F
:105B5000F2F7C0FB81B26846818236216143124A66
:105B6000891808460830F2F7B5FB079036206043E5
:105B70000D4940180830417E6846017404A930463A
:105B80000CF0F4FB002130460CF0BAFB012130464A
:105B90000CF0B6FB002130460CF0D1FB0121304661
:105BA0000CF0B9FB08B070BD100E002070B50446B3
:105BB0000A212046F2F7C4FA06010A212046F2F72C
:105BC000BFFA7018C5B2284670BD08B50020009015
:105BD00000BF00980028FCD008BDF8B50446002599
:105BE00000270FE00A212046F2F7AAFA8EB23046CB
:105BF000B840284385B2381DC7B20A212046F2F7C3
:105C00009FFA84B2002CEDD12846F8BDF8B50446C1
:105C1000002500270EE00A212046F2F77BFA0E4607
:105C20003046B8400543381DC7B20A212046F2F776
:105C300071FA0446002CEED12846F8BD10B500F0EC
:105C400089F810BD10B5C046C04610BD70B50446F9
:105C50000D460126002229462046083009F0D2FCD4
:105C60000026304670BD014601208A6808239A4309
:105C70008A60002070470000F8B505460C460127F1
:105C8000244885420CD12448806A10218843224947
:105C900088620846806A102108431F4988620BE029
:105CA0001D48806A202188431B4988620846806A13
:105CB00020210843184988620020A860207AA86043
:105CC000606800012168884201D90120F8BD207A6E
:105CD000402814D10120286061682068F2F71AFA80
:105CE000C008401EC6B2092E03DA0021284600F083
:105CF0001FF83146284600F016F8074608E0002055
:105D00002860607A4000A17A08436072607A286156
:105D10003846DBE700040040002000400146002038
:105D2000CA68D0B270470246012051600020704717
:105D300070B504460D46012601222946204608304A
:105D400009F060FC0026304670BD02460120D1609B
:105D50000020704710B5F74800780F2871D00CDC90
:105D60000C284FD004DC00280FD00B286AD117E094
:105D70000D2856D00E28F9D192E0153803000EF008
:105D80007EFF05FDFCFBFAF961000521EA48006889
:105D9000FFF75CFF0421E8480068FFF7C9FF9DE2B8
:105DA000E5480068406908280FD10521E2480068ED
:105DB000FFF74CFF0421E0480068FFF747FFA221EE
:105DC000DD480068FFF7C1FF1BE0DB480068406961
:105DD000182816D10C20D74908700521D64800682C
:105DE000FFF734FF0421D4480068FFF72FFFD348A2
:105DF0000088FF22120210400112CF480068FFF70E
:105E0000A4FF6BE2CC4800684069282808D10D2027
:105E1000C8490870C9480178C7480068FFF795FF6E
:105E20005CE2C5480068406928280CD10521C248B9
:105E30000068FFF77DFF0421BF480068FFF706FFF9
:105E40002DE09CE03CE2BC480068406910281ED16F
:105E50000521B9480068FFF7F9FE0421B64800683B
:105E6000FFF7F4FEA321B4480068FFF76EFFB448C3
:105E70000088012805D10221AF480068FFF7E6FE3F
:105E80000DE00221AC480068FFF752FF07E0AA4886
:105E900000684069402802D10E20A64908701DE222
:105EA000A54800684069502831D1A54800880028DD
:105EB0005FD0A1480068FFF731FFA2490968087068
:105EC000A0480068401C9F49086005219A48006866
:105ED000FFF7BCFE042198480068FFF7B7FE98481A
:105EE0000088401E9649088008460088012808D18D
:105EF0000F209049087002218F480068FFF7A6FE26
:105F000037E002218C480068FFF712FF31E08A4831
:105F10000068406958282CD187480068FFF7FEFECA
:105F200088490968087087480068401C85490860EE
:105F300083480088401E824908800846008800285F
:105F400017D105217C480068FFF780FE04217A48BC
:105F50000068FFF7EDFE0AF08DFE7B4908607B4884
:105F6000007810218843103078490870002071496A
:105F70000870B3E18CE1C0E078E068E032E06E48A0
:105F80000068406958282CD16B480068FFF7C6FEAE
:105F90006C49096808706B480068401C69490860D2
:105FA00067480088401E6649088008460088002827
:105FB00017D1052160480068FFF748FE04215E48BC
:105FC0000068FFF7B5FE0AF055FE5F4908605F48BC
:105FD00000781021884310305C4908700020554932
:105FE00008707BE100205A490880534800684069E6
:105FF00008280FD1052150480068FFF727FE04212B
:106000004D480068FFF722FEA2214B480068FFF7C9
:106010009CFE1BE0484800684069182816D11620ED
:1060200044490870052144480068FFF70FFE042129
:1060300041480068FFF70AFE40480088FF2212022C
:10604000104001123C480068FFF77FFE46E13A48E5
:1060500000684069282808D1172036490870374859
:10606000017835480068FFF770FE37E13248006874
:106070004069282840D132480088401E34490988A8
:10608000884221D10AF0F6FD324908602D480068A7
:106090002F4A1288815C28480068FFF756FE2E4878
:1060A000008801280CD12D480088002808D12C48F0
:1060B0000088002804DD2A480088401E28490880FE
:1060C00018201C49087017E01D480088401E204910
:1060D0000988884210DD17201649087019480068A1
:1060E0001B4A1288815C14480068FFF72EFE18488E
:1060F0000088401C16490880F0E00F48006840699D
:10610000282816D11448008800282BD10949087086
:106110000E4800781021884310300C490870052182
:1061200005480068FFF792FD042103480068FFF767
:10613000FFFDACE006000020380000203400002005
:10614000260000200800002020000020360000204B
:10615000240000201C000020320000202800002025
:106160002C00002060480088002830D05F4800885C
:106170005F49098840185D4908805E4800685C49AD
:10618000098840185B4908605B480088002803DDE7
:1061900040205A49088006E059480088574908803D
:1061A00000205749088000204F4908801920554990
:1061B0000870012054490880052154480068FFF701
:1061C00045FD042151480068FFF7B2FD5FE04A48F1
:1061D000008800281DDD454800884030434908807C
:1061E00044480068403043490860402043490880E3
:1061F000192044490870012043490880052143487B
:106200000068FFF723FD042140480068FFF790FD78
:106210003DE03B480088002821DD344800884030BC
:1062200032490880334800684030324908603448B9
:1062300000883249088000203149088019203149FE
:106240000870012030490880052130480068FFF7B8
:10625000FDFC04212D480068FFF76AFD17E028487F
:106260000088002813D12A48007810218843103074
:106270002749087000202349087005212348006839
:10628000FFF7E4FC042121480068FFF751FD25E0F9
:106290001E4800684069102811D11520194908705E
:1062A00005211A480068FFF7D1FC0421174800684F
:1062B000FFF7CCFCA22115480068FFF746FD0DE072
:1062C000002010490870052110480068FFF7BEFC47
:1062D00004210E480068FFF72BFD00BF00BF0B48EC
:1062E0000068FFF7C0FC10BD28000020340000202B
:1062F0002A000020080000202C000020260000209A
:1063000030000020060000202E0000203800002071
:106310003600002002480078C006C00F7047000019
:1063200036000020024800788006C00F7047000049
:10633000360000201CB50220F5F7CCFB072168468B
:106340000FF0F4FA002168464170012181700021AC
:10635000C17001714171012181716A4603210020E0
:10636000FFF7B8FA002203211046FFF701FB0122D4
:1063700003210020FFF714FB1CBD10B500F004F84A
:106380000220F5F799FB10BDF0B587B007216846EC
:106390000FF0CCFA142102A80FF0C8FA00216846C9
:1063A00041706A4603210020FFF794FA042203217A
:1063B0000020FFF7DDFA012108200AF0E7F80021AC
:1063C000684601724173C17201218173017300211A
:1063D0008172417202A90220F5F78AFB0AF09EF849
:1063E00007460D49F1F796FE84B201200004001B18
:1063F00085B229460220F5F717FB01200004001B97
:1064000086B231460220F5F71FFB01210220F5F785
:1064100041FB07B0F0BD0000E02801001CB50021E1
:1064200008200AF0B3F80220F5F754FB01220221FC
:10643000C802FFF7B5FA072168460FF077FA002186
:1064400068464170012181700021C1700171417164
:10645000012181716A460B218020FFF73BFA00225F
:106460000B218020FFF79CFA6A460C218020FFF761
:1064700031FA01220C218020FFF792FA6A460321AB
:106480000020FFF727FA002203211046FFF770FAD9
:10649000012203210020FFF783FA1CBD0148007888
:1064A000704700009405002003480078002801D1BF
:1064B000012070470020FCE78F0400201CB5FFF787
:1064C00063FF072168460FF031FA002168464170EA
:1064D000012181700021C17001710121417181711F
:1064E0006A460221C802FFF7F5F901220221C8021B
:1064F000FFF756FA0BF075F90020034908702920C0
:10650000F8F7B4FE1CBD00008F04002010B52B4826
:106510000078002804D0012821D0022848D129E0A1
:106520002920F8F7F5FC00280BD02920F8F702FD08
:106530004B21C900112009F035F801201F490870CE
:106540000CE000F077F8012808D100F087F8C821A6
:10655000112009F027F80120184908702CE00420C8
:106560000AF0BEFF012804D10BF03BF902201349C9
:10657000087021E01120F5F70BFB002817D104204B
:106580000AF0AEFF012812D100F052FD0A280ED108
:10659000F9F78AFD00280AD1F8F758FE012806D13C
:1065A0000BF0E0F800F05AF800200449087003E00E
:1065B00000200249087000BF00BF10BD8F040020FA
:1065C00010B507480078012808D11020F5F7E0FA47
:1065D000002803D102490870FFF7ACFE10BD00008F
:1065E0003C00002010B500240AF044FB054909686E
:1065F000441A05480068844201D3002010BD0120E0
:10660000FCE70000B0020020AC02002010B500241E
:106610000AF030FB05490968441A054800688442BD
:1066200001D3002010BD0120FCE70000A8020020DB
:10663000A4020020014800787047000051040020A7
:106640000146024800780840704700004F040020CF
:1066500001480078704700009F0200200020014997
:1066600008707047510400200146034800788843B1
:10667000014A1070012070474F040020002801DDFE
:10668000082800DD7047421E01239340D9B2034A17
:1066900012788A43014B1A7000BFF3E79F02002073
:1066A00003480078002801D1012070470020FCE752
:1066B0009D02002003480078002801D10120704786
:1066C0000020FCE74E04002010B50AF0E7F803F0C4
:1066D0000BFC10BD002003490870034908700349F2
:1066E000087070474E0400204F0400205004002022
:1066F00010B586480078002802D001286FD1EEE05E
:10670000FFF7A6FF824908700846007803000EF0E4
:10671000B6FA09065067CBBBCBCBCB97CB000D208D
:10672000F8F700FC000E7B490978884215D00D204F
:10673000F8F7F8FB000E774908700D20F8F7F2FB28
:10674000000EAA2803D12C20F8F790FD05E00022C6
:10675000062141208001FFF723F92C20F8F7D8FB10
:10676000002822D00D20F8F7DDFB000EAA281CD14E
:106770002C20F8F7DFFB0AF0D9F8002811D100220D
:1067800003210220F6F72AFD002206214120800184
:10679000FFF706F90A21202008F004FF01205B49D9
:1067A000087000205C49087002E00020574908701A
:1067B00093E00120FFF762FF002055490870574819
:1067C0000078012108435549087001205449087098
:1067D0005A20F8F74BFD00204C4908707DE092E00C
:1067E0000220FFF74BFF00204949087000F014FC1D
:1067F000FF21053188420ED11F20F8F793FB0028B6
:1068000009D0464800780821084344490870002010
:106810003E49087013E000F0FFFB4249884205D171
:106820003E480078202108433C4908703B480078E6
:1068300002210843394908700020344908704CE0AF
:106840000420FFF71BFF0020314908700DF0A6FB64
:10685000042803D00DF0A2FB032811D12E480078A4
:1068600002280DDA4C20F8F701FD2C480078202191
:1068700008432A49087028480078401C26490870B7
:1068800000202249087028E00320FFF7F7FE0020CF
:106890001F49087021480078042108431F490870E7
:1068A00000201A49087018E00120FFF7E7FE0220D7
:1068B000FFF7E4FE0320FFF7E1FE0420FFF7DEFE12
:1068C0000520FFF7DBFE0620FFF7D8FE0720FFF7C5
:1068D000D5FE0820FFF7D2FE00BF00BF14E0202045
:1068E000F5F756F901280DD101220621412080013A
:1068F000FFF756F8012203210220F6F76FFC002073
:106900000249087000E000BF00BF10BD4E04002027
:106910005004002052040020530400204F040020A3
:10692000510400200203000010B5F848007803006D
:106930000EF0A5F90A064C9EBEFAF9F8F7F6F5F442
:10694000F3480078002812D00020F1490870222076
:10695000F5F71EF900280AD12320F5F719F90128C7
:1069600005D1EC48007808210843EA490870F5F79A
:1069700079F9E949087008460078002814D00846DB
:10698000007800F0D0F9012805D1F5F7FDF90020D5
:10699000DE49087019E0F5F7F7F9022000F0F2F986
:1069A0000120DA49087010E03220F8F7B1FA002827
:1069B00008D03220F8F7BEFA0020D84908802C20F1
:1069C000F8F754FC0020D14908709CE1FFF71EFE47
:1069D000002849D1D048007800F0A5F9012806D157
:1069E000022000F0CFF90220C84908703FE0CC48EF
:1069F0000078401CC0B2CA49087001282DDBC64887
:106A00000078022818D1C5480088401CC349088076
:106A1000084600881E2816DD00220621412080013C
:106A2000FEF7BEFFBB48007804210843B94908704F
:106A30000020B649087010BDB84800881E2802DD45
:106A40003220F8F713FCB348007801210843B1491C
:106A500008700320AD49087002E00120AB490870BE
:106A6000022000F08FF902E00120A84908704AE1F5
:106A7000FFF7CCFD002817D1A748007800F053F9A4
:106A8000012808D10020A6490870F5F77DF90020FB
:106A90009E4908700BE0F5F777F9022000F072F9D3
:106AA00001209A49087002E00220984908702AE102
:106AB000FFF7ACFD00285BD19748007800F033F970
:106AC000012806D1022000F05DF904208F490870EA
:106AD00051E093480078401CC0B291490870C82822
:106AE0003FDB8D48007802281FD18C480088401C6D
:106AF0008A490880084600881E281DDD00220621DC
:106B000041208001FEF74CFF8248007804210843B1
:106B10008049087000207D4908708CE7EFE0D4E0E0
:106B2000A6E08EE070E044E026E07C4800881E2865
:106B300002DD3220F8F79AFB7648007802210843FC
:106B4000744908700120724908700021222008F061
:106B500029FD9621232008F025FD05206B490870AA
:106B600002E0032069490870022000F00BF902E0FE
:106B7000032066490870C6E0FFF748FD002814D1DD
:106B80006548007800F0CFF8012805D1002064495D
:106B900008705E4908700BE0F5F7F6F8022000F087
:106BA000F1F803205949087002E0042057490870A1
:106BB000A9E0FFF72BFD002822D15748007800F00C
:106BC000B2F8012806D1022000F0DCF806204F4977
:106BD000087018E0FFF73CFD02210840002808D1AA
:106BE0004F4908701E2000F0BBF807204749087085
:106BF00009E0022000F0C6F805204449087002E0D0
:106C00000520424908707EE0FFF700FD002814D1FE
:106C10004148007800F087F8012805D1002040495C
:106C200008703A4908700BE0F5F7AEF8022000F062
:106C3000A9F805203549087002E00620334908709C
:106C400061E0FFF7CFFC00280BD1354908703148CF
:106C50000078042108432F49087000202B49087050
:106C600005E0022000F08EF80820284908704AE06C
:106C7000FFF7CCFC002824D12748007800F053F817
:106C8000012806D1092021490870022000F07AF875
:106C90001AE023480078401CC0B2214908706428DB
:106CA0000BDB002008701B480078022108431949BB
:106CB000087007201549087006E00720134908707E
:106CC00002E00820114908701DE0FFF79FFC002832
:106CD00011D11148007800F026F8012805D10020D4
:106CE0000F4908700949087008E0F5F74DF80720CA
:106CF0000649087002E009200449087003E00020FA
:106D00000249087000BF00BF00BF94E69D0200204A
:106D1000A00200209F020020B4020020B602002042
:106D20009E020020704710B50446022C04D10A21AF
:106D3000802000F007F810BD0B210120000300F0B7
:106D400001F8F8E770B504460D4629462046FEF7DF
:106D5000A9FD002801D0012070BD0020FCE7000043
:106D600010B50446044860430449086009F082FFF6
:106D70000349086010BD000040420F00AC02002033
:106D8000B002002010B504467D20C00060438100A1
:106D900040180349086009F06DFF0249086010BD02
:106DA000A4020020A8020020704710B5C046C046CB
:106DB00010BD10B502F038FFC046C04610BD00003F
:106DC0003EB504460D460A2168460EF0AFFD01218E
:106DD000092009F0DBFB0721684601700021C17022
:106DE0008170002C03D003206946487002E0022025
:106DF0006946487000216846017141710121817125
:106E00000804401B81B2684601816946094802F0C6
:106E10004CFF084802F024FF0121064802F033FF2E
:106E2000012203211120F6F7D9F90121014802F0CE
:106E300020FF3EBD000F004010B50446012C08D1D4
:106E40000121092009F0A2FB0121064802F011FFEF
:106E500007E00021092009F099FB0021014802F018
:106E600008FF10BD000F00400149096888B2704753
:106E7000400F00403EB504460A2168460EF056FD1C
:106E80000121242009F082FB0721684601700021BE
:106E9000C1708170002C03D003206946487002E065
:106EA0000220694648700021684601714171817174
:106EB00001816946094802F0F8FE084802F0D0FE58
:106EC0000021064802F0DFFE012203211120F6F71F
:106ED00085F90121014802F0CCFE3EBD400F004083
:106EE00010B502F0B3FE10BD10B502F0B4FE10BD37
:106EF00070B504460D46002229462046143008F09D
:106F000081FB002070BD70B504460D460022294665
:106F1000201D08F077FB002070BD70B504460D46BB
:106F200001222946201D08F06DFB002070BD70B5C0
:106F300004460D4601222946201D08F063FB00206F
:106F400070BD70B504460D46002629462046103017
:106F5000F9F746F80646304670BD0000F0B587B038
:106F600005460C460127224A07CA04AB07C3002086
:106F70000390002C02D1042007B0F0BD002068600F
:106F8000608861780843E1880843A1880843217834
:106F9000084368602078402802D02078C02824D197
:106FA000E088C117C90D09184912890004AA515A6D
:106FB0008EB2E168B1400846F1F72DFC0290A0685E
:106FC000F1F729FC01900299F1F74AFA03903F2169
:106FD00009060398F1F7AEF90290F1F745FC80B28B
:106FE000A86104212846FFF798FF00273846C3E729
:106FF00088C4020001460868C0B2704702461068A3
:10700000000A0002CBB2184310600020704710B590
:1070100002F0B6FE10BD00000348007800020349EC
:10702000097808437047000023040020240400204E
:1070300003480078042801D1012070470A20FCE7AA
:107040002304002010B501201749087017490020BB
:10705000F1F758F91321002001F0F6FB132101206C
:1070600001F0F2FB1321022001F0EEFB13210320BB
:1070700001F0EAFB1321042001F0E6FB13210520B7
:1070800001F0E2FB1321062001F0DEFB13210720B3
:1070900001F0DAFB1321082001F0D6FB13210920AF
:1070A00001F0D2FB10BD0000C3020020C40200208A
:1070B000032803D0072801D0082833D14F49096A93
:1070C00082004F4B9A58120991434C4A1162810039
:1070D0004C4A5158090982004B4B9A5812091143E6
:1070E000464A526A8A4345494A628100474A515892
:1070F00009098200464B9A58120911433F4A926A85
:107100008A433E498A628100424A515809098200F5
:10711000414B9A5812091143384AD26A8A43374977
:10712000CA626AE002283CD13449C96A8200394BFC
:107130009A5812099143314AD1621146896A8200F4
:10714000324B9A58120991432C4A91621146496A6E
:1071500082002C4B9A5812099143284A51621146D9
:10716000096A8200264B9A5812099143234A1162F8
:10717000114649688200244B9A5891431F4A516036
:107180001146C9688200244B9A5891431B4AD1602A
:107190001146896882001E4B9A589143174A9160A4
:1071A0002BE0164909688200154B9A589143134AFF
:1071B00011608100134A51588200134B9A581143B1
:1071C0000E4A52688A430D494A6081000F4A51585D
:1071D00082000F4B9A581143084A92688A43074924
:1071E0008A6081000B4A515882000B4B9A58114318
:1071F000024AD2688A430149CA607047405C004035
:10720000C8C30200A0C30200F0C3020078C302009A
:1072100040C4020050C3020018C40200F8B505467D
:107220000C462B000DF02BFD140B2532485E7287A7
:10723000A1B0CFF4F2F1F0EFEEEDECEBEAE9A00053
:10724000D4490858A100D44A515808430090A000DE
:10725000D24E3058A600D24FBE5930430246A0004D
:10726000D04E3358A000D04E3158204602F0FEFBDD
:107270008EE100200090A000CA490B58A000C74929
:107280000A580021204602F0F1FB81E1A000C1492B
:1072900008580090A000C34E3058A600C34FBE59F6
:1072A00030430346A000BE4E3258A000BE4E3158B7
:1072B000204602F0DBFB6BE1A000B64908580090C5
:1072C000A000B84E3058A600B84FBE593043034610
:1072D000A000B24E3258A000B34E3158204602F002
:1072E000C5FB55E1A000AC4908580090A000AD498D
:1072F0000858A100AD4E715808430346A000A749A5
:107300000A580021204602F0B1FB41E1A000A1494A
:107310000858A100A04A515808430090A000A34E6D
:107320003358A0009D4E3258A0009F4E3158204641
:1073300002F09CFB2CE1A00096490858A100964A57
:10734000515808430090A000944E3058A600944F26
:10735000BE5930430246A000944E3358A000924ECE
:107360003158204602F082FB12E1A00089490858FA
:107370000090A0008B490B58A00088490A580021B2
:10738000204602F073FB03E1A00082490858A100E7
:10739000814A515808430090A000824E3058A60000
:1073A000824FBE5930430346A0007C4E3058A600A1
:1073B0007B4FBE5930430246A0007B4E31582046D9
:1073C00002F054FBE4E0A00072490858A100724AA0
:1073D000515808430090A000724E3058A600734FD9
:1073E000BE5930430346A0006C4E3258A0006E4E8A
:1073F0003158204602F03AFBCAE0C8E0C3E0B7E0EB
:10740000A5E08CE078E062E048E034E01DE0FFE7D2
:10741000A00060490858A1005F4A515808430090F5
:10742000A00060490858A100604E71580843034607
:10743000A0005A490858A100594E71580843024605
:107440000021204602F012FBA2E0A0005249085899
:107450000090A000514E3058A600514FBE59304305
:107460000246A000514E3358A0004F4E31582046DE
:1074700002F0FCFA8CE0A00046490858A100464AF8
:10748000515808430090A000454B1A58A000464BA5
:1074900019580023204602F0E9FA79E00020009014
:1074A000A000404E3058A600404FBE59304303461E
:1074B000A0003A4E3058A600394FBE59304302461C
:1074C000A000394E3158204602F0D0FA60E0A0000A
:1074D00030490858A100304A515808430090A00094
:1074E000324E3358A0002E4E3258A0002E4E315846
:1074F000204602F0BBFA4BE0A00026490858A10044
:10750000254A515808430090A00028490B58A00074
:1075100023490A580021204602F0A8FA38E0A000CA
:107520001C490858A1001C4A515808430090A0006B
:107530001C490858A1001D4E715808430346A0007D
:1075400017490A580021204602F090FA20E0A000D6
:10755000114908580090A000144E3358A000104E56
:107560003258A000104E3158204602F07FFA0FE04A
:1075700000200090A0000D490B5800221146204623
:1075800002F074FA04E02046FFF792FD00E000BF2D
:1075900000BFF8BD50C3020018C40200A0C302001F
:1075A000F0C3020078C30200C8C3020040C4020056
:1075B00010B5FDF7F3FC51490870514800780028D8
:1075C00002D0012878D145E005F058FC4D490978F2
:1075D000884206D005F052FC4A490870012048490B
:1075E00008704648007820210840474909788842B9
:1075F00008D0424800782021084043490870012003
:107600003F49087013F03CF940490978884206D098
:1076100013F036F93D49087001203949087013F01C
:107620000BF93B490978884206D013F005F938492F
:1076300008700120324908700CF0B6FC3549097811
:10764000884206D00CF0B0FC3249087001202C4969
:10765000087050E005F012FC0A2803D1012001F067
:10766000CDFB02E0002001F0C9FB2748007820286C
:1076700003D1012001F006FB02E0002001F002FB33
:1076800022480078012802D101F086F802E00020AB
:1076900001F082F81E480078012802D101F0EAF8D2
:1076A00002E0002001F0E6F81B480078002804D131
:1076B000012001F043F803E019E0002001F03EF85A
:1076C00014480078032807D012480078042803D013
:1076D00010480078052803D1012001F06FFB02E07B
:1076E000002001F06BFB00200549087003E000203A
:1076F0000349087000BF00BF10BD00002B0400202C
:107700002004002025040020260400202704002057
:10771000280400202A04002029040020F3B583B0A7
:107720000E46092700BF0398029000210298F1F746
:107730003DF903D2F90702984840029033000DF05A
:107740009EFA06040F1C2937455358480299F0F752
:107750004AFE029001F072FB019001F0ABF84BE0A1
:1077600053480299F0F73FFE029001F067FB514940
:107770000843019001F09EF83EE04F480299F0F76F
:1077800032FE029001F05AFB4C490843019001F08F
:1077900091F831E04A480299F0F725FE029001F095
:1077A0004DFBE121C9040843019001F083F823E077
:1077B00044480299F0F717FE029001F03FFB612167
:1077C00009050843019001F075F815E03E4802995B
:1077D000F0F709FE029001F031FB21214905084331
:1077E000019001F067F807E00298029001F026FB93
:1077F000019001F05FF800BF00BF0298F1F748F870
:1078000004460D4620462946002358405940084367
:1078100020D016E00A22002320462946F0F7A4FCD7
:10782000D0B239467A1E57B20190C8B2019901F020
:107830000BF80A22002320462946F0F795FC04465F
:107840000D460021084661406840014306D0002FE4
:10785000E0DA03E00021092000F0F6FF002E15DD3C
:10786000062E13DA01F0EAFA0121C906B1400843F5
:10787000019001F01FF806E039467A1E57B2C8B2EF
:10788000002100F0E1FFF01CB842F5DD002F0BDB1A
:1078900000210398F1F78AF806D239467A1E57B2CA
:1078A000C8B2122100F0D0FF05B0F0BD0024744929
:1078B0000050C3470000C20700401C460000840778
:1078C00000007A440000C84200002041F8B5074695
:1078D0000C460825002F16D010E00A213846F0F794
:1078E00019FC009129466A1E55B2C8B2009900F0F1
:1078F000ABFF0A213846F0F70DFC0746002F19D0E0
:10790000002DEADA16E00620001BC6B208E0294680
:107910006A1E55B2C8B2002100F096FF701EC6B2B2
:10792000002E01D0002CF2D1002C03D10021082020
:1079300000F08AFF23000DF0A2F905040A131C25AC
:107940002E0001F07BFA009000F0B4FF29E001F076
:1079500075FA012149040843009000F0ABFF20E0D4
:1079600001F06CFA012189040843009000F0A2FFA5
:1079700017E001F063FA0121C9040843009000F008
:1079800099FF0EE001F05AFA012109050843009021
:1079900000F090FF05E001F051FA009000F08AFF3E
:1079A00000BF00BFF8BD0000F8B50446FFF74AFB72
:1079B00023000DF064F906CE042B7998CBCE01207C
:1079C000400200F077FF02206B49087008460078FB
:1079D000F8F7E0F9694908600846006800906849CE
:1079E0000098F0F7E3FF08D266490098F0F738FDF9
:1079F00005460121FFF792FE07E062490098F0F783
:107A00002FFD05460321FFF789FEB3E05E4800F035
:107A100051FF03205849087008460078F8F7BAF972
:107A20005649086008460068009058490098F0F7E9
:107A3000BDFF0BD253490098F0F712FD0121C90791
:107A4000484005460321FFF769FE2CE050490098A5
:107A5000F0F7ACFF0BD24B490098F0F701FD012184
:107A6000C907484005460421FFF758FE1BE0494975
:107A70000098F0F79BFF0BD242490098F0F7F0FC1A
:107A80000121C907484005460521FFF747FE0AE0E6
:107A90003C490098F0F7E4FC0121C907484005463D
:107AA0000621FFF73BFE65E00720400200F002FFE1
:107AB00001203149087008460078F8F76BF92F4922
:107AC000086008460068F0F7A6FE07468F21C90542
:107AD000F0F7C6FC06462A49F0F7C2FC054601212C
:107AE000FFF71CFE46E00120C00200F0E3FE552037
:107AF0002149087008460078F8F74CF91F490860DA
:107B0000084600680A280DD20021072000F09CFEDC
:107B10000021062000F098FE002118480068FFF7B9
:107B2000D5FE12E015480068642809D2002106201D
:107B300000F08AFE002111480068FFF7C7FE04E04C
:107B400000210E480068FFF7C1FE13E000F044FE7C
:107B500010E00E21022000F077FE0E21032000F03D
:107B600073FE0A21042000F06FFE0121052000F0C1
:107B70006BFE00BF00BFF8BD2C04002030040020C5
:107B800000007A440000C842000200080024744942
:107B90008096184B20BCBE4CFEB50446FFF752FA47
:107BA00001F04CF9054600F085FE23000DF067F862
:107BB0000FFD0945819FD0FCFBFAF9F8F7F6F5F4C3
:107BC000FD001120FE49087008460078F8F702F918
:107BD000FC490860084600680002010F012000F01F
:107BE00033FEF84800680003010F022000F02CFE6D
:107BF0001221032000F028FEF24800880004010F43
:107C0000042000F021FEEF4800880005010F052048
:107C100000F01AFE1221062000F016FEE948007856
:107C20000006010F072000F00FFEE648007801076C
:107C3000090F082000F008FE56E32220E0490870F2
:107C400008460078F8F7C6F8DE490860084600687C
:107C50000002010F012000F0F7FDDA480068000380
:107C6000010F022000F0F0FD1221032000F0ECFDD6
:107C7000D44800880004010F042000F0E5FDD1483D
:107C800000880005010F052000F0DEFD122106200E
:107C900000F0DAFDCB4800780006010F072000F065
:107CA000D3FDC84800780107090F082000F0CCFD7B
:107CB0001AE30121084600F0C7FD1221022000F05E
:107CC000C3FD0120BE49087008460078F8F782F825
:107CD000BC490860096809090A225143B94A127867
:107CE0001207120F88180021FFF7F0FDFCE20221B5
:107CF000012000F0A9FD1221022000F0A5FD0220C4
:107D0000AF49087008460078F8F764F8AD49086094
:107D10000120C00400F0CEFDAA480068010F052034
:107D200000F092FDA74800680001010F062000F056
:107D30008BFDA44800680002010F072000F084FDBD
:107D4000A04800680003010F082000F07DFDCBE291
:107D50000321012000F078FD1221022000F074FDC3
:107D600003209749087008460078F8F733F89549DA
:107D70000860084600680002010F032000F064FD5F
:107D8000904800680003010F042000F05DFD8D485D
:107D900000880004010F09E07CE149E116E1EBE015
:107DA000C7E0A3E07FE05BE019E09CE2052000F083
:107DB0004BFD844800880005010F062000F044FDBB
:107DC000804800780006010F072000F03DFD7D4847
:107DD00000780107090F082000F036FD84E2042036
:107DE0007749087008460078F7F7F4FF754908608E
:107DF00008460068010F012000F026FD7148006868
:107E00000001010F022000F01FFD6E480068000213
:107E1000010F032000F018FD6A4800680003010FFD
:107E2000042000F011FD674800880004010F0520C0
:107E300000F00AFD634800880005010F062000F0ED
:107E400003FD604800780006010F072000F0FCFCED
:107E50005C4800780107090F082000F0F5FC43E2B8
:107E60000421012000F0F0FC1221022000F0ECFCC3
:107E700005205349087008460078F7F7ABFF5149D1
:107E8000086008460068F0F7E1FC00224E4B0191C3
:107E90000090F0F73DFC0546F0F76CFD0746032126
:107EA000FFF73CFC20E20521012000F0CDFC12216F
:107EB000022000F0C9FC06204149087008460078FD
:107EC000F7F788FF3F49086008460068F0F7BEFCF6
:107ED00000223D4B01910090F0F71AFC0546F0F7A7
:107EE00049FD07460321FFF719FCFDE106210120AA
:107EF00000F0AAFC1221022000F0A6FC0720304965
:107F0000087008460078F7F765FF2E4908600846B4
:107F10000068F0F79BFC054600222B4BF0F7F8FBBE
:107F200001910090F0F726FD07460321FFF7F6FBCD
:107F3000DAE10721012000F087FC1221022000F085
:107F400083FC08201E49087008460078F7F742FFB6
:107F50001C49086008460068F0F778FC00221A4BBC
:107F600001910090F0F7D4FB0546F0F703FD0746BA
:107F70000321FFF7D3FBB7E10821012000F064FCE7
:107F80001221022000F060FC09200D49087008460B
:107F90000078F7F71FFF0B49086008460068F0F704
:107FA00055FC0022084B01910090F0F7B1FB05460B
:107FB000F0F7E0FC07460321FFF7B0FB94E1000077
:107FC0002D040020340400200000F040092101208D
:107FD00000F03AFC1221022000F036FC0A20C349CE
:107FE000087008460078F7F7F5FEC14908600120DF
:107FF000C00400F05FFCBE4800880004010F0520AB
:1080000000F022FCBA4800880005010F062000F0AD
:108010001BFCB74800780006010F072000F014FC95
:10802000B34800780107090F082000F00DFC5BE160
:108030000A21012000F008FC1221022000F004FCBB
:108040000220AA49087008460078F7F7C3FEA8493D
:1080500008600120C00400F02DFCA5480088000441
:10806000010F052000F0F0FBA14800880005010F7A
:10807000062000F0E9FB9E4800780006010F07206B
:1080800000F0E2FB9A4800780107090F082000F091
:10809000DBFB29E10B209549087008460078F7F7CB
:1080A00099FE9349086008460068019008460078E8
:1080B000012836D10B21002000F0C6FB122101203F
:1080C00000F0C2FB68460179022000F0BDFB1221DE
:1080D000032000F0B9FB694648790A21F0F730F82F
:1080E000C5B22946042000F0AFFB694648790A2151
:1080F000F0F726F8CDB22946052000F0A5FB1221A5
:10810000062000F0A1FB68468179072000F09CFB67
:108110001221082000F098FB6846C179092000F080
:1081200093FB73480078022836D10B21002000F021
:108130008BFB1221012000F087FB684601790220A9
:1081400000F082FB1221032000F07EFB6946487993
:108150000A21EFF7F5FFC5B22946042000F074FBB1
:10816000694648790A21EFF7EBFFCDB22946052091
:1081700000F06AFB1221062000F066FB6846817958
:10818000072000F061FB1221082000F05DFB68462B
:10819000C179092000F058FB55480078032878D1B0
:1081A0001221002000F050FB694648796421EFF766
:1081B000C7FFC5B22946012000F046FB6946487951
:1081C0000A21EFF7BDFF06460A21EFF7B9FFCDB24E
:1081D0002946022000F038FB694648790A21EFF76A
:1081E000AFFFCDB22946032000F02EFB6946887907
:1081F0008021084000281CD01221042000F024FB1C
:10820000694689794806400E0A21EFF799FFC5B201
:108210002946052000F018FB694689794806400E7A
:108220000A21EFF78DFFCDB22946062000F00CFBA6
:1082300017E01321042000F007FB694688790A2122
:10824000EFF77EFFC5B22946052000F0FDFA69462A
:1082500088790A21EFF774FFCDB22946062000F095
:10826000F3FA1321072000F0EFFA6946C8790A21D2
:10827000EFF766FFC5B22946082000F0E5FA694627
:10828000C8790A21EFF75CFFCDB22946092000F03A
:10829000DBFA17480078042824D10B21002000F0D5
:1082A000D3FA1221012000F0CFFA6846417902206A
:1082B00000F0CAFA1221032000F0C6FA6946887954
:1082C0000A21EFF73DFFC5B22946042000F0BCFAB1
:1082D000694688790A21EFF733FFCDB22946052098
:1082E00000F0B2FA00E000BF00BFFEBD2D04002088
:1082F0003404002070B50446FEF7A4FE00F09EFD95
:10830000054600F0D7FA012C02D0022C79D14DE0BD
:108310000121084600F098FA1221022000F094FA98
:1083200001204B49087008460078F7F7D3FD49490A
:108330000860084600784007C00F002804D00121DB
:10834000052000F081FA03E00021052000F07CFA0E
:10835000404800780007C00F002804D00121062003
:1083600000F072FA03E00021062000F06DFA3948AF
:108370000078C007C00F002804D00121072000F0BA
:1083800063FA03E00021072000F05EFA314800782C
:108390008007C00F002804D00121082000F054FA03
:1083A00003E00021082000F04FFA4FE002210120F5
:1083B00000F04AFA1221022000F046FA0220244975
:1083C000087008460078F7F785FD224908600846DE
:1083D0000078C006C00F002804D00121052000F05D
:1083E00033FA03E00021052000F02EFA1948007846
:1083F0008006C00F002805D00121062000F024FAD5
:1084000004E022E00021062000F01EFA1148007866
:108410004006C00F002804D00121072000F014FA04
:1084200003E00021072000F00FFA0A480078000658
:10843000C00F002804D00121082000F005FA03E055
:108440000021082000F000FA00E000BF00BF70BD6E
:108450002E04002038040020F0B587B00546FEF752
:10846000F1FD2B000CF00BFC07FD052755A8E3FCE4
:10847000FD00A848407A552804D10120400200F0B0
:1084800019FA03E00520C00100F014FA0220A24905
:10849000087008460078F7F775FDA049086008469F
:1084A000006805909E490598EFF7DAFF064601211E
:1084B000FFF734F92AE19748407A552804D107207C
:1084C000400200F0F7F903E01D20C00100F0F2F9CE
:1084D00001209149087008460078F7F753FD8F494D
:1084E000086008460068F0F7B1F9064600228D4B97
:1084F000F0F70EF900228C4B01910090F0F708F98B
:1085000003910290F0F736FA01210490FFF706F983
:10851000FCE08048407A552804D10120C00200F0D8
:10852000C9F903E01120C00100F0C4F90A207A491A
:10853000087008460078F7F725FD78490860084676
:1085400000680121C907884219D37448006888432C
:108550007249086008460068F0F778F9064600227C
:10856000704BF0F7D5F80022704B01910090F0F7B6
:1085700067F803910290F0F7FDF9044613E06748AD
:108580000068F0F763F906460022664BF0F7C0F882
:108590000022674B01910090F0F752F8039102908E
:1085A000F0F7E8F9044663492046EFF759FF06461D
:1085B0000021FFF7B3F8A9E05648407A552804D1C6
:1085C0000120C00200F076F903E01120C00100F0A4
:1085D00071F90121084600F037F91221022000F05C
:1085E00033F904204C49087008460078F7F7CAFCB4
:1085F0004A49086008460068F0F728F90646002254
:10860000484BF0F785F80022494B01910090F0F7B4
:1086100017F803910290F0F7ADF904464649204659
:10862000EFF71EFF06460021FFF778F86EE03948A5
:10863000407A552804D10120C00200F03BF903E044
:108640001120C00100F036F90221012000F0FCF8F1
:108650001221022000F0F8F807202F49087001E0ED
:1086600023E042E008460078F7F78CFC2B490860CD
:1086700008460068F0F7EAF806460022294BF0F7B2
:1086800047F800222A4B01910090EFF7D9FF0391A0
:108690000290F0F76FF9044627492046EFF7E0FE15
:1086A00006460021FFF73AF830E01A48407A55288C
:1086B00003D1202000F0FEF802E0A02000F0FAF83C
:1086C0000F21012000F0C0F80E2013490870084661
:1086D0000078F7F757FC11490860084600680590D4
:1086E00003210598FFF71AF810E00E21032000F08F
:1086F000ABF80E21042000F0A7F80A21052000F0B5
:10870000A3F80421062000F09FF800BF00BF07B0C7
:10871000F0BD0000FA2600202F0400203C040020B9
:108720000050C3470000F04000408F40000039C0B7
:10873000000039400000C84200401C461249087041
:1087400012490978104A127891421BD00E490978D3
:108750000E4A117001210E4A1170002809D00A4AF0
:1087600011700C49097804229143091D094A1170BE
:1087700008E00021044A1170064909780422914357
:10878000044A117070470000C1020020C20200209C
:10879000C3020020C402002001210C4A11700028ED
:1087A00009D00B4A11700B49097849084900491C46
:1087B000084A117008E00021054A1170054909783E
:1087C00049084900034A117070470000C3020020A5
:1087D000BF020020C402002010B501201749087014
:1087E00017491848EFF78EFD0821002000F02CF8FB
:1087F0000821012000F028F80821022000F024F8C8
:108800000821032000F020F80821042000F01CF8C3
:108810000821052000F018F80821062000F014F8BF
:108820000821072000F010F80821084600F00CF895
:108830000821092000F008F810BD0000C302002044
:10884000C4020020FFFFFF0F0A280EDA0122824037
:10885000064B1B881A43054B1A80142902DA044A76
:10886000115402E01322024B1A547047BA0200203E
:10887000D714002001210C4A1170002809D00B4A9E
:1088800011700B49097802229143891C084A117022
:1088900008E00021054A1170054909780222914338
:1088A000034A117070470000C3020020C00200207C
:1088B000C402002070B504460120464908704648AD
:1088C0000078002807D140222146914308464349B9
:1088D000EFF718FD09E040480078012805D1402154
:1088E000214308463D49EFF70DFD3D48007800283B
:1088F00009D03A48EFF7EEFC102108430546374906
:10890000EFF700FD08E03548EFF7E4FC102188435D
:1089100005463249EFF7F6FC32480078002809D0C6
:108920002E48EFF7D7FC0821084305462B49EFF7FF
:10893000E9FC08E02948EFF7CDFC0821884305460B
:108940002649EFF7DFFC28480078002809D02348A3
:10895000EFF7C0FC0121084305462049EFF7D2FCA0
:1089600008E01E48EFF7B6FC45086D001B49284695
:10897000EFF7C8FC1D480078002809D01748EFF72A
:10898000A9FC0221084305461449EFF7BBFC08E0A7
:108990001248EFF79FFC0221884305460F49EFF785
:1089A000B1FC13480078002809D00C48EFF792FC7E
:1089B0000421084305460949EFF7A4FC08E00748ED
:1089C000EFF788FC0421884305460449EFF79AFC39
:1089D00070BD0000C3020020BC020020C4020020C1
:1089E000BD020020BE020020BF020020C002002005
:1089F000C102002010B59E48007800281CD101203B
:108A00009B490870FCF7DCFB9A4988420AD1042094
:108A10009949087001209949087008460078FFF7C5
:108A20001BFD23E101209449087094490870084611
:108A30000078FEF7B9FF19E10220FDF701FE0028DA
:108A400034D000208E4908700220FDF70DFE8A48C0
:108A50000078042810D18948007803280CD101201F
:108A600085490870002085490870FEF7EBFA8248B6
:108A7000007800F027F9F9E07F4800780428D0D08A
:108A800003217D480078EFF75BFBC8B27A49087094
:108A900008460078401C0870002078490870FEF7EE
:108AA000D1FA7548007800F00DF9DFE00120FDF7FC
:108AB000C7FD00285AD0002071490870FEF7C2FA9D
:108AC0000120FDF7D1FD6C48007801280FD1052168
:108AD0006A480078EFF734FBC8B268490870084666
:108AE0000078401C087008460078FEF75DFF624879
:108AF000007802280FD10E2160480078EFF720FBA4
:108B0000C8B25E49087008460078401C08700846E4
:108B10000078FFF741F858480078032811D15749E9
:108B20000878C10F091849104900411A534A1170B9
:108B300010460078401C1146087008460078FFF780
:108B4000D9FB4D480078042895D106214B48007880
:108B5000EFF7F6FAC8B24949087008460078401C99
:108B6000087008460078FFF777FC7FE00420FDF7E7
:108B700067FD002815D00020414908700420FDF74A
:108B800073FD3D480078042870D0FEF75BFA0120A1
:108B9000394908703949087008460078FEF704FF23
:108BA00064E00820FDF74CFD002819D0002034496E
:108BB0000870FEF747FA0820FDF756FD04202E49FD
:108BC000087000202D4908702B48007800F07AF8D2
:108BD00000F034F9802108430446FFF76BFE45E0BE
:108BE0001120F6F795F9002812D0002024490870CA
:108BF000FEF728FA1120F6F79DF901201E490870AA
:108C000005201E49087008460078FEF7CDFE2DE0CD
:108C10000020F6F77DF9002812D0002018490870CE
:108C2000FEF710FA0020F6F785F9042012490870C3
:108C300001201249087008460078FFF70DFC15E086
:108C40001020F6F765F9002810D000200C490870B4
:108C5000FEF7F8F91020F6F76DF9012006490870C3
:108C60000649087008460078FEF79EFE10BD000019
:108C7000220400208D7C6B5A230400202404002051
:108C80002104002001210C4A1170002809D00B4A50
:108C900011700B490978082291430831084A117074
:108CA00008E00021054A117005490978082291431E
:108CB000034A117070470000C3020020BE0200206A
:108CC000C402002070B50446FEF7BCF9002C17DD85
:108CD000052C15DA00F0B2F80546FFF7EBFD12217E
:108CE0000320FFF7B1FD0A210420FFF7ADFD214667
:108CF0000520FFF7A9FD12210620FFF7A5FD0FE0D3
:108D00000E210320FFF7A0FD0E210420FFF79CFD9C
:108D100012210520FFF798FD0A210620FFF794FD98
:108D200070BD000010B521480078002802D001284D
:108D300036D123E01E480078012803D11D48007871
:108D4000012807D11A480078022803D01848007873
:108D5000032807D13C21012005F0CCFC0120134958
:108D600008700AE012480078042806D11249012050
:108D700005F0C0FC01200D49087015E0012005F048
:108D8000EBFA00280BD10120094908700949087045
:108D900008460078FEF708FE00200449087003E04A
:108DA00000200249087000BF00BF10BD2104002050
:108DB0002304002024040020302A000001210C4A52
:108DC0001170012809D10B4A11700B490978402212
:108DD00091434031084A117008E00021054A1170A2
:108DE0000549097840229143034A117070470000F9
:108DF000C3020020BC020020C402002001210C4A52
:108E00001170002809D00B4A11700B490978102203
:108E100091431031084A117008E00021054A117091
:108E20000549097810229143034A117070470000E8
:108E3000C3020020BD020020C402002010B5024879
:108E4000EFF748FA10BD0000C402002010B5092158
:108E50000020FCF797FD0A210020FCF793FD0B2171
:108E60000020FCF78FFD0C210020FCF78BFD042176
:108E70008020FCF787FD05218020FCF783FD002181
:108E80004020FCF77FFD01214020FCF77BFD022103
:108E90004020FCF777FD0C2101200003FCF772FD58
:108EA0000D2101200003FCF76DFD0E2101200003C0
:108EB000FCF768FD0A214020FCF764FD0B214020EF
:108EC000FCF760FD0C214020FCF75CFD0D214020EB
:108ED000FCF758FD0E214020FCF754FD0F214020E7
:108EE000FCF750FD0821C020FCF74CFD0921C020F3
:108EF000FCF748FD0A21C020FCF744FD0B21C020EF
:108F0000FCF740FD06218020FCF73CFD0721802076
:108F1000FCF738FD08218020FCF734FD0921802072
:108F2000FCF730FD08210020FCF72CFD0321402038
:108F3000FCF728FD04214020FCF724FD05214020FA
:108F4000FCF720FD06214020FCF71CFD10BD0000B1
:108F500007480078002809D106480078002805D184
:108F600005480088002801D1012070470020FCE757
:108F7000B8020020C3020020BA0200200D48007889
:108F8000022805D10C480078022801D10020704742
:108F900008480078042805D107480078002801D047
:108FA0000020F4E705480078002801D00020EEE713
:108FB0000120ECE7230400202404002020040020EA
:108FC0001FB5082102A80CF0B1FC082168460CF07E
:108FD000ADFCFFF73BFF0121162007F0D7FA2E4822
:108FE0000090001401900F214905019888430190D9
:108FF00001210903019888430190019800090001AB
:1090000001904900019888430190490001988843E4
:1090100001904900019888430190490001988843D4
:109020000190890001988843019049000198884384
:1090300001904900019888430190684600F0D8FDEE
:109040000121684601720321417200218172C172BF
:109050000321017301214173002181730121C17337
:1090600002A800F067FD00F057FD00200B490870D2
:109070000B4908800B4908700B4908700B490870B0
:109080000B4908700B4908700B4908700B490870B0
:109090000B49EFF737F91FBD0000FFFFB8020020B2
:1090A000BA020020BC020020BD020020BE02002047
:1090B000BF020020C0020020C1020020C302002025
:1090C000C402002010B50020154908701549087029
:1090D00015490870FCF774F81449884206D1042039
:1090E0001349087001201349087004E00120104959
:1090F00008701049087001200F49087000200F49BE
:1091000008700F4908700F4908700F490870012056
:109110000E49087000200E4908600E49086010BD15
:109120002004002021040020220400208D7C6B5AA2
:10913000230400202404002025040020260400200D
:1091400027040020280400202A04002029040020ED
:10915000300400203C04002010B5022005F0FCF88B
:10916000002814D10121022005F0C4FAFEF720FAEC
:10917000FFF7D8FD00F012FCF5F704F9012803D140
:109180000020FFF7DBFA02E00120FFF7D7FAFFF734
:1091900031FC10BD10B5FE480078002806D001282B
:1091A00014D002287ED003287DD1FFE2F948007850
:1091B000002803D1F8480088002806D00120F4498F
:1091C000087007F057FDF5490860D4E3F1480078CE
:1091D000002869D0F2480078C107C90FF1484078EB
:1091E0008006C00F81420BD0EE4840782021884392
:1091F000EB4909784901202211400843E9494870A8
:10920000E74800788007C10FE64840780007C00FA4
:1092100081420DD0E348407808218843E04909782D
:109220008907C90FC900082211400843DD49487069
:10923000DB4800784007C10FDA48203080784007CB
:10924000C00F81420FD0D748203080780421884356
:10925000D34909784907C90F8900042211400843FE
:10926000D04920318870CE4800780007C10FCD4822
:1092700040784007C00F81420DD0CA484078042191
:109280008843C74909780907C90F8900042211409A
:109290000843C4494870C2480078C006C00FC1499D
:1092A000097B02E07EE265E3AAE18907C90F8842F3
:1092B0000DD0BC48007B02218843B9490978C90612
:1092C000C90F4900022211400843B6490873B44847
:1092D00000788006C00FB34909798907C90F884211
:1092E0000DD0B048007902218843AD49097889063C
:1092F000C90F4900022211400843AA490871A84831
:1093000000784006C00FA749097A8907C90F88422B
:109310000DD0A448007A02218843A1490978490662
:10932000C90F49000222114008439E4908729C4817
:109330000078C0099B49097A4907C90F88420DD0B6
:109340009848007A04218843954909780906C90F8D
:1093500089000422114008439249087290484078DD
:109360008007C00F8F4909788907C90F88420DD03F
:109370008C48007802218843894949788907C90FB8
:109380004900022211400843864908708448407809
:109390004007C00F834909784907C90F88420DD09B
:1093A00080480078042188437D4949784907C90FDE
:1093B00089000422114008437A49087078484078AF
:1093C0000007C00F774909794907C90F88420DD0B6
:1093D0007448007904218843714949780907C90F05
:1093E00089000422114008436E4908716C48807856
:1093F0008007C10F6B484078C007C00F81420AD078
:109400006848407840084000654989788907C90F55
:10941000084364494870624880784007C00F61493A
:10942000097BC907C90F88420AD05E48007B400803
:1094300040005B4989784907C90F084359490873B7
:10944000574880780007C00F5649097AC907C90FE5
:1094500088420AD05348007A400840005049897831
:109460000907C90F08434F4908724D488078C00664
:10947000C00F4C490979C907C90F88420AD0494829
:1094800000794008400046498978C906C90F084359
:1094900044490871424880788006C00F41490978E4
:1094A000C907C90F88420AD03E48007840084000EA
:1094B0003B4989788906C90F08433A4908703848FA
:1094C00080784006C00F374909784906C90F88429D
:1094D0000DD03448007840218843314989784906C5
:1094E000C90F89014022114008432E4908702C48B9
:1094F0008078C1092B4820304078C00981420FD0C4
:1095000028482030407880218843254989780906F9
:10951000C90FC901802211400843224920314870F7
:109520001F48C078C107C90F1E4820304078800608
:10953000C00F81420DD01B48203040782021884345
:109540001749C978490120221140084315492031A3
:1095500048701348C0788007C00F12490978C906BF
:10956000C90F88420DD00F480078102188430C495C
:10957000C9788907C90F0901102211400843094918
:1095800008700748C0784007C00F0649097B0BE008
:10959000B8020020C3020020BA020020C802002046
:1095A000C4020020405C00404907C90F88420DD02A
:1095B000F248007B04218843F149C9784907C90F63
:1095C0008900042211400843EC490873EC48C07834
:1095D0000007C10FE9484078C00981420DD0E74833
:1095E000407880218843E649C9780907C90FC90135
:1095F000802211400843E14948700020E149087089
:10960000E148008800287DD0DF480078C007C00FFF
:1096100000280DD0DC48008840084000DA49088066
:109620000020FDF745FDD94908780021FDF7F6FD3A
:10963000D54800880221084000280CD0D248008874
:109640008843D14908800120FDF732FDCF49487891
:109650000121FDF7E3FDCC480088042108400028E3
:109660000CD0C94800888843C74908800220FDF70C
:109670001FFDC64988780221FDF7D0FDC248008849
:109680000821084000280CD0BF4800888843BE4904
:1096900008800320FDF70CFDBC49C8780321FDF7C5
:1096A000BDFDB94800881021084000280CD0B648FC
:1096B00000888843B44908800420FDF7F9FCB349C9
:1096C00008790421FDF7AAFDAF4800882021084051
:1096D00000280CD0AC4800888843AB49088005209E
:1096E000FDF7E6FCA94948790521FDF797FDA64855
:1096F00000884021084000280ED0A34800888843F5
:10970000A14900E046E008800620FDF7D1FC9F4912
:1097100088790621FDF782FD9B480088802108405A
:1097200000280CD098480088884397490880072073
:10973000FDF7BEFC9549C8790721FDF76FFD9248FA
:109740000088FF210131084000280CD08E48008895
:1097500088438D4908800820FDF7AAFC8B49087AC8
:109760000821FDF75BFD8848008801214902084077
:1097700000280CD084480088884383490880092049
:10978000FDF796FC8149487A0921FDF747FD002045
:109790007D49088002207E49087007F06BFA7D49F8
:1097A0000860E8E003207A490870E4E07448007833
:1097B000C107C90F714840788006C00F81427DD132
:1097C0006F4800788007C10F6C4840780007C00FD1
:1097D0008142F4D16A4800784007C10F67482030C1
:1097E00080784007C00F8142E9D1654800780007C2
:1097F000C10F624840784007C00F81425ED1604887
:109800000078C006C00F5D49097B8907C90F8842EF
:1098100054D15B4800788006C00F58490979890700
:10982000C90F88424AD1564800784006C00F5349B4
:10983000097A8907C90F884240D151480078C00988
:109840004E49097A4907C90F884237D14C484078B8
:109850008007C00F494909788907C90F88422DD16F
:10986000474840784007C00F444909784907C90F65
:10987000884278D1424840780007C00F3F490979B3
:109880004907C90F88426ED13D4880788007C10FD3
:109890003A484078C007C00F814264D13848807888
:1098A0004007C00F3549097BC907C90F88425AD103
:1098B000334880780007C00F304900E053E0097A50
:1098C000C907C90F88424ED12D488078C006C00F05
:1098D0002A490979C907C90F884244D128488078A4
:1098E0008006C00F25490978C907C90F88423AD1B7
:1098F000234880784006C00F204909784906C90FDF
:10990000884230D11E488078C1091C4820304078F8
:10991000C009814227D11A48C078C107C90F17482A
:10992000203040788006C00F81421CD11448C07896
:109930008007C00F11490978C906C90F884212D1A2
:109940000F48C0784007C00F0C49097B4907C90F71
:10995000884208D10A48C0780007C10F07484078FC
:10996000C009814202D00120064908700020084940
:10997000087000E000BF00BF10BD0000405C004068
:10998000C4020020C3020020BA020020D714002025
:10999000B8020020C80200207047000010B5284817
:1099A000007801280FD12748007800280BD02648DE
:1099B0000078F6F7EFF925490968884203D0214875
:1099C0000078FDF7F1FF1E48007802280FD11D48EE
:1099D000007800280BD01E480078F6F7FBF91D49E7
:1099E0000968884203D017480078FEF7D5F8144874
:1099F000007803280FD11348007800280BD01648B0
:109A00000078F6F767FA15490968884203D00D48CF
:109A10000078FEF76FFC0A48007804280FD1094847
:109A2000007800280BD00E480078F6F7ABFA0D4905
:109A30000968884203D003480078FEF70DFD10BD89
:109A400023040020240400202C04002030040020E3
:109A50002D040020340400202E04002038040020AF
:109A60002F0400203C0400207047000070B5049CC7
:109A70008DB2002D05D0274D2D688EB23543254E71
:109A8000356095B2002D05D0224D6D6896B23543F4
:109A9000204E75609DB2002D05D01E4DAD689EB262
:109AA00035431C4EB560A5B2002D05D0194DED68AB
:109AB000A6B23543174EF5600D0C2D04002D06D0CF
:109AC000144D2D6A0E0C36033543124E3562150CBB
:109AD0002D04002D06D00F4D6D6A160C360335434C
:109AE0000C4E75621D0C2D04002D06D0094DAD6A7B
:109AF0001E0C36033543074EB562250C2D04002D90
:109B000006D0044DED6A260C36033543014EF5624E
:109B100070BD0000405C004000210549002004E0C9
:109B200000220A60091D421CD0B21028F8DB7047E1
:109B3000405C00402D490968072252029143027897
:109B4000520207235B021A401143284A1160114652
:109B50000968DA10914342789201DB101A401143F0
:109B6000224A1160114609682022914382785201ED
:109B700020231A4011431D4A11601146096818221A
:109B80009143C278D20018231A401143174A11603A
:109B900011460968062291430279520006231A40B1
:109BA0001143124A11601146496892159143427956
:109BB0001202FF2301331A4011430C4A516011462F
:109BC0004968802291438279D20180231A4011434F
:109BD000064A51601146096849084900C279D2070E
:109BE000D20F1143014A116070470000005C004031
:109BF000024A0168D160416811617047005C004011
